:020000040800F2
:1000000000040020A51F0008F71F0008F71F0008C4
:10001000F71F0008F71F0008F71F00080000000086
:10002000000000000000000000000000F71F0008B2
:10003000F71F000800000000F71F0008AD2A0208A3
:10004000452C0208472C0208492C02084D2C0208B6
:100050007D2C02087F2C0208812C0208A52C0208A6
:10006000C92C0208ED2C0208112D0208352D0208BA
:10007000372D0208392D02083B2D02083D2D0208BC
:100080003F2D0208412D0208432D0208F71F0008EA
:10009000F71F0008F71F0008F71F0008452D02088A
:1000A000912D0208932D0208952D0208972D020824
:1000B000992D02089D2D0208C92D0208392E02082B
:1000C0003B2E02083D2E02083F2E0208412E020858
:1000D000452E0208B52F0208DD2E020879300208ED
:1000E00035310208F9310208FB310208FD310208FE
:1000F00001320208693202086B3202086D320208CE
:100100006F32020871320208733202087532020837
:10011000793202084D3302084F3302085133020886
:100120005D3402085F340208613402086334020857
:1001300000000000000000000000000000000000BF
:1001400000000000000000000000000000000000AF
:10015000000000000000000000000000000000009F
:10016000000000000000000000000000000000008F
:10017000000000000000000000000000000000007F
:10018000000000000000000000000000000000006F
:10019000000000000000000000000000000000005F
:1001A000000000000000000000000000000000004F
:1001B000000000000000000000000000000000003F
:1001C000000000000000000000000000000000002F
:1001D000000000000000000000000000000000001F
:0401E0005FF8E0F1F3
:1001E800032A70B404460D4626D941EA000313F0E9
:1001F800030F13D020782B78984208BF294606D0E1
:100208001EE014F8010F11F8013F984218D1012A95
:1002180002F1FF32F5D1002070BC70470B4604464E
:1002280051F8045B50F8046BAE4204D1043A04461A
:10023800032A0B46F2D81D461046002ADAD1EBE70E
:10024800C01AE9E7032A2DE9F00109D82AB10023E9
:10025800CC5CC45401339342FAD1BDE8F001704735
:100268000B468218014603E02478013301F8014B5C
:1002780011F0030F1C46F7D113F003055DD06E4251
:10028800C5F1040CED009B594FEACC0C08E004348E
:10029800A7593B4607FA0CF748EA070741F8047BD9
:1002A800571A23FA05F8032FF1DC03E014F8013B91
:1002B80001F8013B8A42F9D8CFE753F8404C41F89E
:1002C800404C53F83C4C41F83C4C53F8384C41F8FE
:1002D800384C53F8344C41F8344C53F8304C41F80E
:1002E800304C53F82C4C41F82C4C53F8284C41F81E
:1002F800284C53F8244C41F8244C53F8204C41F82E
:10030800204C53F81C4C41F81C4C53F8184C41F83D
:10031800184C53F8144C41F8144C53F8104C41F84D
:10032800104C53F80C4C41F80C4C53F8084C41F85D
:10033800084C53F8044C41F8044C561A1D460C4618
:10034800403340313F2EB8DC2B460FE053F8101CE9
:1003580044F8101C53F80C1C44F80C1C53F8081CE7
:1003680044F8081C53F8041C44F8041C161B2146C6
:100378001D46103410330F2EE8DC2B4602E02468AB
:1003880041F8044B551A1C46032D03F10403F6DC0F
:1003980090E700BF032AC9B270B408D82AB103464F
:1003A800121803F8011B9342FBD170BC70478218E6
:1003B800044601E004F8011B14F0030FFAD14FF0D2
:1003C800013303FB01F31FE044F8403C44F83C3C94
:1003D80044F8383C44F8343C44F8303C44F82C3C6D
:1003E80044F8283C44F8243C44F8203C44F81C3C9D
:1003F80044F8183C44F8143C44F8103C44F80C3CCD
:1004080044F8083C44F8043C161B254640343F2E6B
:10041800DADC2C4607E044F8103C44F80C3C44F87D
:10042800083C44F8043C161B254610340F2EF2DC19
:1004380001E045F8043B541B032CFADC01E005F805
:10044800011B9542FBD3B0E710F0030F38B5044603
:1004580012D10368A3F1013222EA030313F0803FAB
:100468000AD1031D184653F8042BA2F1013525EAD9
:10047800020212F0803FF5D003782BB1431C1846D6
:1004880013F8012B002AFAD100F076F9204638BD7E
:10049800C9B2F0B4002950D010F0030F10D003787F
:1004A800002B79D0994246D0431C05E013F8012B64
:1004B800002A3FD091423ED013F0030F1846F5D1E1
:1004C800036841EA01270646A3F1013247EA0747D4
:1004D80022EA030212F0803F1DD187EA0303A3F149
:1004E800013222EA030313F0803F14D1043002E002
:1004F80012F0803F0FD1064650F8043BA3F10135B6
:1005080087EA030225EA0303A2F1013413F0803FCE
:1005180024EA0202ECD033783046002B3CD09942D2
:1005280009D0731C01E0914205D0184613F8012B3D
:10053800002AF8D11046F0BC704710F0030F0CD019
:100548000378002BF7D0431C03E013F8012B002A93
:10055800F1D013F0030F1846F7D102680346A2F151
:10056800013121EA020212F0803F0AD10430034629
:1005780050F8042BA2F1013121EA020212F0803F67
:10058800F5D01A781846002AD5D00133184613F842
:10059800012B002AFAD1CEE71846CCE780EA0102FF
:1005A80012F0030F3AD110F0030220F0030021F0FB
:1005B800030150F804CB08BF51F8043B0DD082F07A
:1005C80003024FEAC2026FF07F4323FA02F251F8A6
:1005D800043B4CEA020C43EA020300BFACF10132CF
:1005E8009C4501BF22EA0C0212F0803F50F804CB70
:1005F80051F8043BF2D04FEA0C604FEA1C2C01285A
:1006080028BFB0EB036F08BF1B0AF4D003F0FF0349
:100618004FEA1060A0EB0300704700BF10F0030F13
:100628000AD010F8012B11F8013B012A28BF9A4281
:10063800F4D0A2EB030070474DF8045D4DF8044D6B
:100648004FF0010242EA022242EA024201F0030CA0
:1006580021F0030150F8044B51F8045BBCF1020F80
:1006680026D04BD824F07F4CBCEB152FA4EB02030B
:1006780023EA04030DD113EAC21308BF51F8045B3F
:100688000AD18CEA040CBCEB056F0CD150F8044B72
:10069800E8E74FEA15255CE033F07F4352D10D7847
:1006A8004FEA146C55E04FEA146C05F0FF0550E072
:1006B8004FEA044CA4EB02034FEA1C4C23EA040360
:1006C800BCEB154F17D113EAC21308BF51F8045BEE
:1006D80007D18CEA040CBCEB054F08D150F8044B49
:1006E800E6E71B042ED10D884FEA144C31E04FEA9F
:1006F80005454FEA144C4FEA15452AE004F0FF0C73
:10070800BCEB156FA4EB020323EA04030DD113EA33
:10071800C21308BF51F8045B0AD18CEA040CBCEB85
:10072800052F0AD150F8044BE8E74FEA156510E0A9
:1007380014F0FF0F06D051F8045B4FEA142C25F093
:100748007F4506E04FF000005DF8044B5DF8045B60
:1007580070470CF0FF0205F0FF00012828BF904207
:1007680004BF4FEA1C2C2D0AF3D0A2EB00005DF861
:10077800044B5DF8045B704780EA0102844612F07E
:10078800030F4FD111F0030F32D14DF8044D11F082
:10079800040F51F8043B0BD0A3F101329A4312F035
:1007A800803F04BF4CF8043B51F8043B16D100BF0E
:1007B80051F8044BA3F101329A4312F0803FA4F19F
:1007C80001320BD14CF8043BA24312F0803F04BF26
:1007D80051F8043B4CF8044BEAD023460CF8013B93
:1007E80013F0FF0F4FEA3323F8D15DF8044B70473D
:1007F80011F0010F06D011F8012B0CF8012B002A7B
:1008080008BF704711F0020FBFD031F8022B12F069
:10081800FF0F16BF2CF8022B8CF8002012F47F4F24
:10082800B3D1704711F8012B0CF8012B002AF9D12C
:10083800704700BF20F0030110F00300C0F1000072
:1008480051F8043B00F1040C4FEACC0C6FF00002A5
:100858001CBF22FA0CF213434FF0010C4CEA0C2C8B
:100868004CEA0C4CA3EB0C0222EA030212EACC126B
:1008780004BF51F8043B0430F4D013F0FF0F1FBF3E
:10088800013013F47F4F013013F47F0F18BF01308C
:10089800704700BFF0B4002A46D041EA000313F0C5
:1008A80003032CD1032A07460E4643D904680D6872
:1008B800AC423FD1043A37D0A4F1013525EA04040B
:1008C80014F0803F18BF18462CD1041D0D1D0EE0F2
:1008D80054F8043B55F8041BA3F101308B4220EA7D
:1008E800030027D1043A1FD010F0803F1ED1032AFD
:1008F80027462E46ECD820462946002A1DD00478E3
:10090800013A0D78AC420CD172B18CB1002302E0EF
:1009180093420BD064B1013310F8014FCD5CAC4267
:10092800F6D0601BF0BC70471046FBE70020F9E7E3
:100938002046F7E738463146E1E724782D78F0E796
:1009480041EA000313F0030F0B4670B414BF0024F0
:100958000124032A94BF002404F001040546D4B9F5
:10096800BAB10E782B46013A03F8016B56B1AC1CAC
:100978007AB111F8015F2346013A04F8015C0134A9
:10098800002DF5D12AB19A18002103F8011B9342D2
:10099800FBD170BC7047194653F8044BA4F10136DB
:1009A80026EA040616F0803FDAD1043A45F8044BEB
:1009B800032A1946EFD8D3E701232DE9F0071D468E
:1009C80000264FF0FF37AC1900EB070C8C420DD214
:1009D8001CF805C010F80480E0452ED201252646F3
:1009E800E31BAC198C4200EB070CF1D34FF0010963
:1009F80000264D464FF0FF3C1360AC1900EB0C0885
:100A0800A1420ED918F8058010F804A0C2451AD9D9
:100A180001252646CCEB0409AC19A14200EB0C08D1
:100A2800F0D80CF101000137B8423CBF994638466E
:100A3800C2F80090BDE8F00770470BD00123374695
:100A48001D46F618BFE709D04FF00109B4464D46D8
:100A58004E44D2E79D4205D00135B4E74D4505D057
:100A68000135CAE72B4626460125ACE7A9462646A6
:100A78000125C2E72DE9F04FADF5826D81B014462E
:100A8800074610460DF580628B460C3219461D4606
:100A9800FFF792FF03AE04A901F57E72331F0090A1
:100AA80043F8045F9342FBD14DB1681E0023E25C1A
:100AB800C11A013303AEAB4246F82210F7D1DDF874
:100AC8000C142046009A6118FFF78AFB002877D19A
:100AD8000099814605F1FF380646C1F101020192ED
:100AE8005A46AB4609EB0B0501F1FF3AB81800214D
:100AF800AA1A00F0E5F900284FD1002D00F0C080B7
:100B08007B1903A913F8013C51F82330002B4CD171
:100B1800009B9E4228BF334698450FD903EB090135
:100B2800E05C7A18795C884205D038E012F8011F39
:100B3800E05C884233D101339845F7D8009A964251
:100B480080F0A48007EB090214F80A10534612F843
:100B58000A20914204BF0AEB0901791807D095E0F1
:100B680014F802C011F8010D844503D113465A1E2A
:100B7800B342F5D101369E4200F28D80DDF80C6457
:100B88002A46B144C6EB0B0609EB0B05B818002141
:100B9800AA1A00F095F90028AFD0002071E0019A58
:100BA8000026914499442A46EEE7002EFAD0DDF853
:100BB8000C2493423CBFC2EB0B0306469944F2E770
:100BC800009E4FF000080099AB1BB34238BF334674
:100BD800C1F101026E1E019201F1FF3A5A4689469F
:100BE800AB460133CDF80C3408EB0B05B8180021DF
:100BF800AA1A00F065F90028CFD1002D40D07B1942
:100C080003A913F8013C51F82330002B30D1B1452A
:100C180013D208EB090314F80910FA18FB5C99427F
:100C280018BF4B4627D14B4604E012F8011FE05C81
:100C3800884220D10133B342F7D3BAF1FF3F53467C
:100C48002CD007EB080C14F80A101CF80A20914263
:100C58000CD10AEB0802BA1804E0E05C12F8011D96
:100C6800884203D1013BF8D260460AE0DDF80C3433
:100C780098442A46B8E701992A4688449844B3E735
:100C8800284605B00DF5806DBDE8F08F009B013654
:100C98009E427FF673AF07EB0900F2E707EB080CFB
:100CA8006046EEE72DE9F04F8346037885B00C46A1
:100CB800002B00F0F9800A78A2B106460131012024
:100CC80002E011F8012B8AB1934214BF002000F012
:100CD800010016F8013F0D46002BF2D12B782BB1FD
:100CE8004FF0000B584605B0BDE8F08F0028F9D149
:100CF8000BF101002178FFF7CBFB2D1BA5F10102B9
:100D0800534243EB0203002808BF43F001030746A0
:100D180083B90BEB0508404594BFC0EB08084FF0BA
:100D280001081F2D08D9414622462B46FFF7A2FE8F
:100D38008346D7E78346D5E7294603AA2046FFF727
:100D48003BFE03996118814620464A46FFF748FA58
:100D580000284FD109F1FF33C9F10102064601927B
:100D680082464246C84699460AEB050BB818002148
:100D7800C2EB0B0200F0A4F80028B1D1BBF1000FC0
:100D8800B0D046452CBF334643469D420FD903EBAE
:100D98000A01E05C7A18795C884205D075E012F89F
:100DA800011FE05C884270D101339D42F7D1B04504
:100DB8007DD907EB0A0214F809104B4612F80920EE
:100DC800914202BF09EB0A01AC46791806D06EE0E1
:100DD800A55C11F8010D854203D113465A1EB34292
:100DE800F6D1654601369E4267D8039E5A46B244FC
:100DF800AE1BB9E7C9F10101C9EB0503424600265C
:100E080009F1FF3A88464B4538BF4B4601330393F7
:100E180006EB050BB8180021C2EB0B0200F050F8E6
:100E280000287FF45DAFBBF1000F3FF45BAF4D4589
:100E380012D906EB090314F80910FA18FB5C994259
:100E480008BF4B4605D026E012F8011FE05C884237
:100E580022D101339D42F7D1BAF1FF3F534628D042
:100E680007EB060C14F80A101CF80A20914217D157
:100E78000AEB0602BA1804E0E05C12F8011D884289
:100E88000ED1013BF8D2E3462CE7019A00269244A2
:100E98005A469A4468E74B4646445A46F618B7E716
:100EA800039B5A46F618B3E70D46012016E743465A
:100EB80098E707EB060CE34614E707EB0A0B11E784
:100EC80010F0030F034670B4C9B211D0002A22D023
:100ED80003788B421DD0013A013005E0DAB110F8F1
:100EE800014B013A8C4218D010F0030F0346F5D19C
:100EF800032A14D87AB1187888420ED0541E5D1C83
:100F080003E015F8016B8E4203D0013C2846F8D265
:100F1800002070BC70471046FBE71846F9E741EA25
:100F2800012646EA0646184653F8044B86EA0404A6
:100F3800A4F1013525EA040414F0803F03D1043AF2
:100F48001846032AEFD80346D4E700BF0000000084
:100F5800C1F30A5C0246ACF57E7C2DE9F84FACF192
:100F68000704132C0B4606460F468946804627DCA5
:100F7800002C52DB4FF6FF7CC0F20F0C4CFA04FA3F
:100F88000AEA0105054317D037A3D3E9002300F087
:100F980075F80022002300F0B3FC002856D0002F7B
:100FA80005DD4FF4801353FA04F407EB040929EA2A
:100FB8000A0900264B46324610461946BDE8F88F06
:100FC800332C07DDB4F5806FF6D100F057F80246F0
:100FD8000B46F1E74FF0FF3BACF11B0C2BFA0CFB77
:100FE8001BEA000FE8D020A3D3E9002300F046F85D
:100FF8000022002300F084FC40B3002F0ADD142CEB
:1010080006D00126C4F13404A64016EB080601D325
:1010180007F1010926EA0B0619E013A3D3E9002317
:1010280000F02CF80022002300F06AFC78B1002FB1
:1010380013DB46EA07054FF000094D45C3F6F07982
:101048000CBF2E46002608BFA94600E0B9464B460D
:10105800324610461946BDE8F88F00264FF0004981
:10106800F5E700BFAFF300809C7500883CE4377E4D
:1010780081F0004102E000BF83F0004330B54FEA41
:1010880041044FEA430594EA050F08BF90EA020FAE
:101098001FBF54EA000C55EA020C7FEA645C7FEA41
:1010A800655C00F0E2804FEA5454D4EB5555B8BF64
:1010B8006D420CDD2C4480EA020281EA030382EAD5
:1010C800000083EA010180EA020281EA0303362D67
:1010D80088BF30BD11F0004F4FEA01314FF4801C3A
:1010E8004CEA113102D0404261EB410113F0004F4C
:1010F8004FEA03334CEA133302D0524263EB430303
:1011080094EA050F00F0A780A4F10104D5F1200EA0
:101118000DDB02FA0EFC22FA05F2801841F10001FB
:1011280003FA0EF2801843FA05F359410EE0A5F1CF
:1011380020050EF1200E012A03FA0EFC28BF4CF000
:10114800020C43FA05F3C01851EBE37101F00045B6
:1011580007D54FF0000EDCF1000C7EEB00006EEBC3
:101168000101B1F5801F1BD3B1F5001F0CD349084D
:101178005FEA30004FEA3C0C04F101044FEA4452A4
:1011880012F5800F80F09A80BCF1004F08BF5FEA2B
:10119800500C50F1000041EB045141EA050130BD0B
:1011A8005FEA4C0C404141EB010111F4801FA4F1AE
:1011B8000104E9D191F0000F04BF01460020B1FA03
:1011C80081F308BF2033A3F10B03B3F120020CDA3B
:1011D8000C3208DD02F1140CC2F10C0201FA0CF019
:1011E80021FA02F10CE002F11402D8BFC2F1200C7E
:1011F80001FA02F120FA0CFCDCBF41EA0C01904034
:10120800E41AA2BF01EB0451294330BD6FEA04047C
:101218001F3C1CDA0C340EDC04F11404C4F1200267
:1012280020FA04F001FA02F340EA030021FA04F379
:1012380045EA030130BDC4F10C04C4F1200220FAD0
:1012480002F001FA04F340EA0300294630BD21FA0E
:1012580004F0294630BD94F0000F83F4801306BFD4
:1012680081F480110134013D4EE77FEA645C18BFC8
:101278007FEA655C29D094EA050F08BF90EA020F5F
:1012880005D054EA000C04BF1946104630BD91EA57
:10129800030F1EBF0021002030BD5FEA545C05D15A
:1012A8004000494128BF41F0004130BD14F5800499
:1012B8003CBF01F5801130BD01F0004545F0FE410D
:1012C80041F470014FF0000030BD7FEA645C1ABF42
:1012D800194610467FEA655C1CBF0B46024650EA79
:1012E800013406BF52EA033591EA030F41F40021A5
:1012F80030BD00BF90F0000F04BF0021704730B52B
:101308004FF4806404F132044FF000054FF00001FF
:1013180050E700BF90F0000F04BF0021704730B5C0
:101328004FF4806404F1320410F0004548BF404295
:101338004FF000013EE700BF42004FEAE2014FEAEA
:1013480031014FEA02701FBF12F07F4393F07F4FC5
:1013580081F06051704792F0000F14BF93F07F4FF7
:10136800704730B54FF4607401F0004521F000413A
:1013780020E700BF50EA010208BF704730B54FF0C0
:1013880000050AE050EA010208BF704730B511F0C5
:10139800004502D5404261EB41014FF4806404F1FD
:1013A80032045FEA915C3FF4DCAE4FF003025FEA7F
:1013B800DC0C18BF03325FEADC0C18BF033202EB07
:1013C800DC02C2F1200300FA03FC20FA02F001FA61
:1013D80003FE40EA0E0021FA02F11444C1E600BF00
:1013E80070B54FF0FF0C4CF4E06C1CEA11541DBFB3
:1013F8001CEA135594EA0C0F95EA0C0F00F0DEF87E
:101408002C4481EA030621EA4C5123EA4C5350EA62
:10141800013518BF52EA033541F4801143F48013B3
:1014280038D0A0FB02CE4FF00005E1FB02E506F044
:101438000042E0FB03E54FF00006E1FB03569CF099
:10144800000F18BF4EF0010EA4F1FF04B6F5007F9F
:1014580064F5407404D25FEA4E0E6D4146EB060611
:1014680042EAC62141EA55514FEAC52040EA5E509A
:101478004FEACE2EB4F1FD0C88BFBCF5E06F1ED844
:10148800BEF1004F08BF5FEA500E50F1000041EB7B
:10149800045170BD06F0004646EA010140EA020028
:1014A80081EA0301B4EB5C04C2BFD4EB0C0541EA4A
:1014B800045170BD41F480114FF0000E013C00F35F
:1014C800AB8014F1360FDEBF002001F0004170BD83
:1014D800C4F10004203C35DA0C341BDC04F114049C
:1014E800C4F1200500FA05F320FA04F001FA05F228
:1014F80040EA020001F0004221F0004110EBD370F5
:1015080021FA04F642EB06015EEA430E08BF20EA20
:10151800D37070BDC4F10C04C4F1200500FA04F3C3
:1015280020FA05F001FA04F240EA020001F0004155
:1015380010EBD37041F100015EEA430E08BF20EAC8
:10154800D37070BDC4F1200500FA05F24EEA020E10
:1015580020FA04F301FA05F243EA020321FA04F03F
:1015680001F0004121FA04F220EA020000EBD370F6
:101578005EEA430E08BF20EAD37070BD94F0000FF6
:101588000FD101F00046400041EB010111F4801F2A
:1015980008BF013CF7D041EA060195F0000F18BFDB
:1015A800704703F00046520043EB030313F4801F17
:1015B80008BF013DF7D043EA0603704794EA0C0FD1
:1015C8000CEA135518BF95EA0C0F0CD050EA4106E7
:1015D80018BF52EA4306D1D181EA030101F0004164
:1015E8004FF0000070BD50EA410606BF104619468C
:1015F80052EA430619D094EA0C0F02D150EA013698
:1016080013D195EA0C0F05D152EA03361CBF1046D8
:1016180019460AD181EA030101F0004141F0FE4177
:1016280041F470014FF0000070BD41F0FE4141F4FB
:10163800780170BD70B54FF0FF0C4CF4E06C1CEAFB
:1016480011541DBF1CEA135594EA0C0F95EA0C0FB0
:1016580000F0A7F8A4EB050481EA030E52EA03356B
:101668004FEA013100F088804FEA03334FF080558C
:1016780045EA131343EA12634FEA022245EA1115B9
:1016880045EA10654FEA00260EF000419D4208BF6A
:10169800964244F1FD0404F5407402D25B084FEA17
:1016A8003202B61A65EB03055B084FEA32024FF4C3
:1016B80080104FF4002CB6EB020E75EB030E22BF20
:1016C800B61A754640EA0C005B084FEA3202B6EBE0
:1016D800020E75EB030E22BFB61A754640EA5C008F
:1016E8005B084FEA3202B6EB020E75EB030E22BF1F
:1016F800B61A754640EA9C005B084FEA3202B6EB20
:10170800020E75EB030E22BFB61A754640EADC00DE
:1017180055EA060E18D04FEA051545EA16754FEA40
:1017280006164FEAC30343EA52734FEAC2025FEA5E
:101738001C1CC0D111F4801F0BD141EA00014FF0ED
:1017480000004FF0004CB6E711F4801F04BF0143BE
:101758000020B4F1FD0C88BFBCF5E06F3FF6AFAEDA
:10176800B5EB030C04BFB6EB020C5FEA500C50F16A
:10177800000041EB045170BD0EF0004E4EEA1131ED
:1017880014EB5C04C2BFD4EB0C0541EA045170BDF4
:1017980041F480114FF0000E013C90E645EA060E38
:1017A8008DE60CEA135594EA0C0F08BF95EA0C0F66
:1017B8003FF43BAF94EA0C0F0AD150EA01347FF4AE
:1017C80034AF95EA0C0F7FF425AF104619462CE785
:1017D80095EA0C0F06D152EA03353FF4FDAE1046E8
:1017E800194622E750EA410618BF52EA43067FF439
:1017F800C5AE50EA41047FF40DAF52EA43057FF4C9
:10180800EBAE12E74FF0FF3C06E000BF4FF0010CD3
:1018180002E000BF4FF0010C4DF804CD4FEA410C37
:101828007FEA6C5C4FEA430C18BF7FEA6C5C1BD004
:1018380001B050EA410C0CBF52EA430C91EA030F85
:1018480002BF90EA020F0020704710F1000F91EAE2
:10185800030F58BF994208BF90422CBFD8176FEAB0
:10186800E37040F0010070474FEA410C7FEA6C5C7E
:1018780002D150EA013C07D14FEA430C7FEA6C5C85
:10188800D6D152EA033CD3D05DF8040B704700BFB1
:101898008446104662468C461946634600E000BFFF
:1018A80001B5FFF7B7FF002848BF10F1000F01BDD1
:1018B8004DF808EDFFF7F4FF0CBF012000205DF89C
:1018C80008FB00BF4DF808EDFFF7EAFF34BF012021
:1018D80000205DF808FB00BF4DF808EDFFF7E0FFBA
:1018E80094BF012000205DF808FB00BF4DF808ED0B
:1018F800FFF7CEFF94BF012000205DF808FB00BF72
:101908004DF808EDFFF7C4FF34BF012000205DF853
:1019180008FB00BF4FEA4102B2F1E04324BFB3F530
:10192800001CDCF1FE5C0DD901F0004C4FEAC0024E
:101938004CEA5070B2F1004F40EB830008BF20F032
:101948000100704711F0804F21D113F13872BCBFEC
:1019580001F00040704741F480114FEA5252C2F141
:101968001802C2F1200C10FA0CF320FA02F018BF8A
:1019780040F001004FEAC1234FEAD32303FA0CFCDD
:1019880040EA0C0023FA02F34FEA4303CCE77FEA6C
:10199800625307D150EA01331EBF4FF0FE4040F4B6
:1019A8004000704701F0004040F0FE4040F4000065
:1019B800704700BF80F0004002E000BF81F00041A6
:1019C80042001FBF5FEA410392EA030F7FEA226CDD
:1019D8007FEA236C6AD04FEA1262D2EB1363C1BF6D
:1019E800D218414048404140B8BF5B42192B88BFDC
:1019F800704710F0004F40F4000020F07F4018BFFF
:101A0800404211F0004F41F4000121F07F4118BF1E
:101A1800494292EA030F3FD0A2F1010241FA03FCC6
:101A280010EB0C00C3F1200301FA03F100F00043AE
:101A380002D5494260EB4000B0F5000F13D3B0F176
:101A4800807F06D340084FEA310102F10102FE2AE5
:101A580051D2B1F1004F40EBC25008BF20F0010055
:101A680040EA03007047490040EB000010F4000F03
:101A7800A2F10102EDD1B0FA80FCACF1080CB2EB96
:101A88000C0200FA0CF0AABF00EBC25052421843F5
:101A9800BCBFD0401843704792F0000F81F400019A
:101AA80006BF80F400000132013BB5E74FEA41036D
:101AB8007FEA226C18BF7FEA236C21D092EA030FD9
:101AC80004D092F0000F08BF0846704790EA010F53
:101AD8001CBF0020704712F07F4F04D1400028BF80
:101AE80040F00040704712F100723CBF00F5000062
:101AF800704700F0004343F0FE4040F40000704798
:101B08007FEA226216BF08467FEA23630146420243
:101B180006BF5FEA412390EA010F40F48000704756
:101B28004FF0000304E000BF10F0004348BF4042FC
:101B38005FEA000C08BF704743F0964301464FF038
:101B480000001CE050EA010208BF70474FF0000394
:101B58000AE000BF50EA010208BF704711F00043D5
:101B680002D5404261EB41015FEA010C02BF8446A5
:101B78000146002043F0B64308BFA3F18053A3F504
:101B88000003BCFA8CF2083AA3EBC25310DB01FA4B
:101B980002FC634400FA02FCC2F12002BCF1004FCF
:101BA80020FA02F243EB020008BF20F00100704760
:101BB80002F1200201FA02FCC2F1200250EA4C00B4
:101BC80021FA02F243EB020008BF20EADC707047FA
:101BD8004FF0FF0C1CEAD0521EBF1CEAD15392EA08
:101BE8000C0F93EA0C0F6FD01A4480EA010C4002E4
:101BF80018BF5FEA41211ED04FF0006343EA50103E
:101C080043EA5111A0FB01310CF00040B1F5000F7F
:101C18003EBF490041EAD3715B0040EA010062F12E
:101C28007F02FD2A1DD8B3F1004F40EBC25008BF18
:101C380020F00100704790F0000F0CF0004C08BF36
:101C480049024CEA502040EA51207F3AC2BFD2F103
:101C5800FF0340EAC250704740F400004FF0000311
:101C6800013A5DDC12F1190FDCBF00F0004070474B
:101C7800C2F10002410021FA02F1C2F1200200FA89
:101C880002FC5FEA310040F1000053EA4C0308BF50
:101C980020EADC70704792F0000F00F0004C02BFA1
:101CA800400010F4000F013AF9D040EA0C0093F01C
:101CB800000F01F0004C02BF490011F4000F013B76
:101CC800F9D041EA0C018FE70CEAD15392EA0C0FE4
:101CD80018BF93EA0C0F0AD030F0004C18BF31F04F
:101CE800004CD8D180EA010000F00040704790F025
:101CF800000F17BF90F0004F084691F0000F91F0C9
:101D0800004F14D092EA0C0F01D142020FD193EA8E
:101D18000C0F03D14B0218BF084608D180EA010016
:101D280000F0004040F0FE4040F40000704740F0F2
:101D3800FE4040F4400070474FF0FF0C1CEAD052C0
:101D48001EBF1CEAD15392EA0C0F93EA0C0F69D01C
:101D5800A2EB030280EA010C49024FEA402037D087
:101D68004FF0805343EA111143EA10130CF000407E
:101D78008B4238BF5B0042F17D024FF4000C8B426E
:101D880024BF5B1A40EA0C00B3EB510F24BFA3EB4E
:101D9800510340EA5C00B3EB910F24BFA3EB91031E
:101DA80040EA9C00B3EBD10F24BFA3EBD10340EA78
:101DB800DC001B0118BF5FEA1C1CE0D1FD2A3FF6BE
:101DC80050AF8B4240EBC25008BF20F00100704773
:101DD8000CF0004C4CEA50207F32C2BFD2F1FF0316
:101DE80040EAC250704740F400004FF00003013A47
:101DF80037E792F0000F00F0004C02BF400010F4EB
:101E0800000F013AF9D040EA0C0093F0000F01F0FE
:101E1800004C02BF490011F4000F013BF9D041EA20
:101E28000C0195E70CEAD15392EA0C0F08D1420253
:101E38007FF47DAF93EA0C0F7FF470AF084676E726
:101E480093EA0C0F04D14B023FF44CAF08466EE7FF
:101E580030F0004C18BF31F0004CCAD130F00042CD
:101E68007FF45CAF31F000437FF43CAF5FE700BF25
:101E78004FF0FF3C06E000BF4FF0010C02E000BF4E
:101E88004FF0010C4DF804CD4FEA40024FEA4103F0
:101E98007FEA226C18BF7FEA236C11D001B052EAA6
:101EA800530C18BF90EA010F58BFB2EB030088BF6C
:101EB800C81738BF6FEAE17018BF40F001007047DB
:101EC8007FEA226C02D15FEA402C05D17FEA236CBD
:101ED800E4D15FEA412CE1D05DF8040B704700BF04
:101EE800844608466146FFE70FB5FFF7C9FF00289B
:101EF80048BF10F1000F0FBD4DF808EDFFF7F4FFD4
:101F08000CBF012000205DF808FB00BF4DF808ED6C
:101F1800FFF7EAFF34BF012000205DF808FB00BF8F
:101F28004DF808EDFFF7E0FF94BF012000205DF8B1
:101F380008FB00BF4DF808EDFFF7D2FF94BF012062
:101F480000205DF808FB00BF4DF808EDFFF7C8FF5B
:101F580034BF012000205DF808FB00BF42000ED20C
:101F6800B2F1FE4F0BD34FF09E03B3EB126209D4CC
:101F78004FEA002343F0004323FA02F070474FF082
:101F88000000704712F1610F01D1420202D14FF0F7
:101F9800FF3070474FF00000704700BF00F026F890
:101FA8000C4880F30888002103E00B4B5B58435032
:101FB80004310A480A4B42189A42F6D3094A02E009
:101FC800002342F8043B084B9A42F9D318F014FC5A
:101FD8007047000000C0002024A303080000002070
:101FE8006413002064130020C06400207047FEE7DB
:101FF80010B586B0002301244FF46022114801A9CE
:1020080001938DF80930039204938DF808408DF8F8
:10201800144027F0B7FC0B48214627F0D9FC0948A3
:1020280027F0E0FC074827F0E2FC0028FAD1054831
:1020380027F0E1FC034827F0E3FC0028FAD106B0BA
:1020480010BD00BF00240140014610B50D48012213
:10205800032327F0E3FC0B48012127F0D5FC7F2060
:1020680028F012FB0748022127F022FD0028F6D0AD
:102078000448022127F022FD0248BDE8104027F05D
:1020880014BD00BF002401400C4A0C2303FB0123AC
:1020980010B59C880CB9588010BD5B8803F11304F7
:1020A800844204DA142B07D9133B834204DC0C2343
:1020B80003FB012102238B8010BD00BFF02D0020FF
:1020C8000A4B10B500241C7021464FF4E0720848F2
:1020D800FEF760F9074B43F604501C70064B1C7062
:1020E8000FF01AFE054B187010BD00BF64150020D4
:1020F800301700207B190020F8180020FA1800205B
:10210800074B1978013101F01F011970054B1A7836
:102118008A4203D1013202F01F021A70704700BFD1
:10212800F81800207B19002010B50E4A0E2303FB77
:1021380000200D4A014614780C4A03FB042300F1E1
:102148000C0251F8044B914243F8044BF9D10A8828
:1021580000211A800E22FEF71DF9BDE81040FFF796
:10216800CFBF00BF68150020F818002030170020E6
:10217800084B1A5C002352FA03F111F0010FD8B290
:1021880002D00130C0B270470133042BF3D10120D3
:10219800704700BF361A002000F07F0000F5745029
:1021A8002DE9F84309300C46154698460FF0B4FD62
:1021B80000284FD043F63C37002638460FF0ACFDD8
:1021C800C0B25FFA86F988B120280FD04FEA5909C2
:1021D8004BF2B77048440FF09FFDC0B208B1022817
:1021E80004D10123B340227813432370113743F6F7
:1021F800C43301369F42E0D14BF25E600FF08CFD94
:10220800C0B280B120280ED02B784BF24D6043F03D
:1022180001032B700FF080FDC0B220B1202802D03E
:10222800012388F800304BF28F600FF075FDC0B2C3
:1022380080B120280ED02B784BF24D6043F002037A
:102248002B700FF069FDC0B220B1202802D0012305
:1022580088F80030BDE8F883034610465A1E10B5CA
:10226800032A1DD8DFE802F00F0F0209124A52783C
:1022780002F00202D2B2A2B111E00F4A527812F073
:1022880001020ED00BE00D4A927802F04002D2B261
:102298003AB10B4A127802F003029A4200D140B1D7
:1022A80000220848105C984203D00132052AF8D170
:1022B8000021084610BD00BFC45E0020EC39002094
:1022C8008B3D002028170020F8B5064643F63C351C
:1022D800002428460FF020FDC0B2E7B268B12028DC
:1022E8000BD07F084BF2B77038180FF015FD012896
:1022F80003D1A04033781843307001341135082CCD
:10230800E7D1F8BD03780E2202FB0313084AD3185D
:102318009978002351FA03F010F00100DAB202D0E4
:10232800501CC0B270470133082BF3D1704700BF6F
:10233800301700202DE9F04101248C40284A294912
:102348000346E4B2107891F800C019E0264F0E2633
:1023580006FB0076F178A9B996F80680B8F1000F67
:1023680010D196F80580B8F1000F0BD196F80480CB
:10237800B8F1000F06D1F67926B9013000F01F0038
:10238800054626E0FBB1012B05D0022B06D10E2114
:1023980001FB007739790C4218D014E0042B04D1E2
:1023A8000E2101FB0077B9790CE0032B04D10E2133
:1023B80001FB0077797905E0052B07D10E2101FB98
:1023C8000077F97911B11570BDE8F081013000F09E
:1023D8001F006045BAD11570FF20BDE8F08100BF2D
:1023E8007B190020F8180020301700202DE9F04351
:1023F800444D454B2A780E2101FB0232917A85B073
:102408000446984639B101390523594301F56E51FF
:10241800443189B201E043F6C431204604220FF06A
:102428008CFC2B780E2505FB038393F80B80364E26
:10243800344FB8F1000F25D131232371073363716D
:102448003B7801A86B430422F15E06F009FB3B7858
:1024580002A805FB03630222997A06F001FB3B7888
:102468000DF10A0005FB03650322697A06F0F8FA04
:10247800A01D01A90922FEF763FA4FF00F0984F89D
:10248800108012E0B8F1010F0FD132232371053308
:1024980063713B784FF0080905FB036393F901303A
:1024A800E3713B785D43735BA371002320461A46B2
:1024B80012E010F8011BA1F13005EDB2092D04D886
:1024C800EB183029DBB203D004E037395B1800E0A1
:1024D8000A33DBB20132D2B24A45EAD10F21B3FB4B
:1024E800F1F10801411A5B1AC3F10F03DBB2092BA2
:1024F800A35401D8303300E03733A35405B0BDE806
:10250800F08300BF2E17002030170020024B1A78E6
:1025180042F001021A7070479D1C002008B50C4B50
:102528000C4A1B780E2101FB0323D97A21B101291A
:102538000CBF0921002100E0102140221346064863
:1025480006F0B2F8054B1A7842F002021A7008BD7C
:102558002E17002030170020FB1800209D1C00209B
:10256800034B1A7802F0F8026FF3C3021A7070472F
:102578009D1C0020024B1A7842F004021A70704722
:102588009D1C0020024B1A7842F008021A7070470E
:102598009D1C002038B5114B1C7814F0010502D1A0
:1025A800FFF7B4FF05E004F00405EDB21DB9FFF72D
:1025B800E1FF284638BD04F00805EDB215B9FFF76C
:1025C800E1FFF6E704F00204E4B21CB9FFF7A6FF46
:1025D800204638BDFFF7C4FF012038BD9D1C0020F0
:1025E800014B1878704700BF6415002030B51E4BAA
:1025F80085B01B780446002B34D11C4D2B78034141
:1026080013F0010F2ED01A4B1A4A1B780E2101FB2A
:102618000323DA78024112F0010F1CD11B79034120
:1026280013F0010317D110F0010001F1F1014FEA95
:10263800540206D001320091019302926D20FE39B6
:1026480005E001320091019002923C200121032211
:102658000B460FF0DFFB012313FA04F42B7823EA6F
:1026680004042C7005B030BDFA180020F1180020C1
:102678007B19002030170020037830B513F0010FC4
:10268800144A4FF00E0419D104FB01210133012231
:1026980012FA03F3CD7825EA0303CB7004780D7999
:1026A800A41812FA04F425EA04040C7103789B18A0
:1026B8009A408B7823EA02028A7030BD04FB01211C
:1026C800013B012212FA03F38A7822EA03038B7092
:1026D80030BD00BF3017002010B500230278590024
:1026E80052FA01F404F00304022C05D1013414FA5F
:1026F80001F122EA010202700133042BEED110BD70
:102708002DE9F04F85B00192BDF838201C46734B77
:102718000092DA78054612F020028B4640F0D88005
:102728008DF80E208DF80F208DF80D20DCB99B78E0
:1027380003F04003DBB21BB101238DF80F3020E01A
:10274800674B1B7803F04003DBB21BB101238DF804
:102758000E3016E00DF10F010DF10E020DF10D0313
:10276800FFF71AFD0DE0012C0BD19B7803F0400315
:10277800DBB223B90DF10F00FFF7A6FD01E08DF8DC
:102788000F409DF80F3023B99DF80E00002800F087
:10279800A28044B905F07F01490001F574510DF19B
:1027A8000A00663109E0012C0AD1E90101F51E4150
:1027B800E8310DF10A0001EB4B0102220FF0BDFADE
:1027C800BDF90A3013B9002C00F08480009B33B99E
:1027D800444B454F93F80080FFF792FC08E0434BC9
:1027E800434F93F8008008F1010202F01F021A70AB
:1027F8000DF10F00FFF770FF002C44D1BDF80A302F
:1028080069B240F6B83212EA210238BF4FF47A7240
:10281800D2180E2303FB08F3ADF80A20FA529DF8EC
:102828000F90224649460120FE18FFF715FD49463C
:10283800F07022460220FFF70FFD86F802903071F3
:102848009DF80E90224649460420FFF705FD4946AB
:10285800B071824622460320FFF7FEFC05F07F0593
:1028680070713572BAF1000F00D128B1214B1B7875
:1028780013B99DF80D3000E00023F37186F809B014
:10288800019AB2721CE0012C1AD10E2303FB08F343
:10289800BDF80A202046FA529DF80F600022314602
:1028A800FD18FFF7D9FC3146E87000220220FFF737
:1028B800D3FC00232871AE70AB716B71EB71AB72F6
:1028C8000E2303FB0877FC72009B0120BB8102E00A
:1028D800002000E0204605B0BDE8F08FEC3900206C
:1028E800C45E0020F818002030170020631500206F
:1028F80068150020821C002073B5154B04461B7810
:102908000E46D3B11348214622F02DFD0546A0B945
:10291800012E04F1010606D12046FFF729FC009597
:102928000246812005E02046FFF722FC009502467A
:10293800982031462B46FFF7E3FE2146054822F052
:10294800FCFC0548214602B0BDE8704022F000BDFD
:10295800F9180020A21B0020991900202DE9F7433F
:102968007B4B04461B7843B17A4B1B7803F0240356
:10297800042B02D1002900F0E880774B774F1B78B1
:10298800002B00F0C7807648214622F0ECFC002896
:1029980040F0C08007F5C470214622F0E4FC804670
:1029A800002840F0B7803B1993F880302D2B01D0D8
:1029B800532B3AD16B4E357845B30FF011FD04F126
:1029C8000108054650B12046FFF7D2FB337802468E
:1029D8001E33009393204146002307E02046FFF76B
:1029E800C7FB00950246414693202B46FFF788FE19
:1029F8000FF0F6FC014628B1337803201E3300930C
:102A0800002101E0009003200A4680E02046FFF7FD
:102A1800AFFB611C02462B4693200095FFF770FE22
:102A28000095032029462A4671E0542B09D12046F7
:102A3800FFF79EFBCDF800800246611C94204346B8
:102A480066E0462B474D20D12E78BEB10FF0C8FC6A
:102A580004F10109064648B12046FFF789FB2B78A7
:102A680002461E3300939A20494622E02046FFF78B
:102A78007FFB0096024649469A2025E02046FFF74C
:102A880077FB009602469A2039E02E78002E2CD04B
:102A98000FF0A6FC04F11C09064660B12046FFF7BA
:102AA80067FB2B7802461E3369F07F000093C0B2A3
:102AB800611C434609E02046FFF75AFB024669F0CD
:102AC8007F000096C0B2611C3346FFF719FE0FF075
:102AD80087FC21B2024628B12B7803201E330093CD
:102AE800002214E00090032011E02046FFF740FB8D
:102AF800024604F11C0060F07F000096C0B2611C21
:102B08003346FFF7FDFD0096032021463246012398
:102B1800FFF7F6FD124821463F1922F00EFC97F800
:102B280080302D2B0AD0532B08D0542B06D0462B9F
:102B380004D00D48214622F016FC30B10B4821463E
:102B480003B0BDE8F04322F003BC03B0BDE8F08356
:102B580066150020901B0020F9180020302C00205A
:102B6800A21B0020FA1B0020B82D00209A1B002071
:102B7800002302780E2101FB0232044901338A182E
:102B88000021062B9170F4D1704700BF3017002048
:102B9800064B00201870064B1A78064B1B789A4291
:102BA80002D00146FFF7C6BBFF207047641500201E
:102BB800F81800207B1900200121814038B5114BFD
:102BC800C9431A78104BC9B202F0030203F5E07446
:102BD800012A04D1DD7801EA0505DD7005E0022A45
:102BE80003D11D7901EA05051D710E33A342EFD10A
:102BF800FFF7FCFC43F604500FF08EF8034B1870F7
:102C080038BD00BF8B3D002030170020FA18002087
:102C18002DE9F743A34D8DF807002B78A24C1BB183
:102C28002378C2B29A4204D043F604500FF074F8E5
:102C380028709DF8073023709C4C2278072A00F2F0
:102C48002D81DFE812F008002400360054005D00F2
:102C580072008D00BA00964A3C211170954A1946B7
:102C6800107800F00300FFF765FB934BFF281870FE
:102C780000F0368121F06EF8904B002093F8742014
:102C880042F0010283F874208D4B187064E0884B81
:102C98001B78002B00F0248121F024FA012840F051
:102CA8004D812378142201332370864B01381A7022
:102CB80047E17F4B1B78002B00F01281814E307862
:102CC80008B901234AE021F00DFA022804D021F0C6
:102CD80009FA032840F0328121F03CF823780422D5
:102CE800013323701D233370774B1A7026E1704B24
:102CF8003C221A707548FFF779FB2378013323705B
:102D08006B4B1B78002B00F0EB806E4B1D78002D71
:102D180040F014811020FFF73DFC002800F01181DD
:102D280023782846013323700BE1614B1B78002B75
:102D380000F0D68005F022FD002800F00281614BEA
:102D48007D221A705E4B002018705C4B93F874203B
:102D580042F0010283F87420237801332370F0E0F5
:102D6800534B1B78002B00F0BB8021F0BBF90128E6
:102D7800544E03D021F0B6F903280FD19DF807204F
:102D8800012111FA02F2524B197821EA02021A7053
:102D980064233370237801332370CFE03078002820
:102DA80040F0CC80484A032323701378013BDBB200
:102DB8001370002B00F09480C3E0404A414E92F813
:102DC8006A201AB13278002A40F0B88000223270A6
:102DD800013212FA03F3DFF8E0803E4F98F8001052
:102DE8004FF00E0909FB0172DB4392F803E0DBB2F6
:102DF80003EA0E0E907882F803E092F804E003EA02
:102E08000E0E0340937082F804E00DF10700FFF7FF
:102E180033FC98F8003009FB0372D278DFF89490FD
:102E28002AB999F8002002F00302012A0AD00E22DA
:102E380002FB03721279B2B999F8002002F003027A
:102E4800022A10D10E2202FB0377BA785AB9224F10
:102E58003A789A4207D11848FFF78AFE3B7801333F
:102E680003F01F033B7099F800009DF8071000F06D
:102E78000300FFF75FFA144B0422FF281A7088F842
:102E88000000164B42D0987800F04000C0B20028ED
:102E98003CD1032323701A33337052E00020207092
:102EA8004FE000BFFA1800206715002064150020C5
:102EB800F21800208B3D00202E170020103D002026
:102EC8006515002062150020F0180020FB1800206E
:102ED800F1180020301700207B190020EC39002061
:102EE800FFF73EFB0023237020F034FF2B78013BD3
:102EF800DBB22B702BB1144B9B7803F04003DBB291
:102F0800F3B19DF80700FFF757FE19E09B780E4ACA
:102F180003F04003DBB22BB1136843F400031360E2
:102F2800FFF7CEF8FFF71CFB20F014FF00232370F7
:102F380043F604500EF0F0FE287001E0002000E097
:102F4800FF20BDE8FE8300BFEC390020044B1A784F
:102F58000AB1013A1A701B780BB9FFF72DBE7047FA
:102F6800FA180020044A054B10781B7803EA501021
:102F780000F00100704700BFEC390020681B0020FA
:102F8800044B054A1B781078C3F3400303EA10107A
:102F9800704700BF681B0020EC390020034B044A2F
:102FA8001B78D078C3F3800318407047681B002053
:102FB800EC390020044B054A1B78D078C3F3C003D2
:102FC80003EA5000704700BF681B0020EC3900205E
:102FD800044B054A1B78D078C3F3001303EA90002A
:102FE800704700BF681B0020EC390020044B18789C
:102FF800044BDB785B005BB2DB1103EAD01070474F
:10300800681B0020EC39002008B50E2104481DF08B
:10301800D7F8044B5B7803EA000000F0010008BD14
:1030280084190020681B002070B500241BE030467E
:10303800E9B21DF003F980B14FF4366363433422DB
:1030480002FB05330A4AD3181B7A13F0010F04D088
:10305800084B1878C0F3001070BD0135382DE6D143
:103068000134022C02D0E6B20025E0E7002070BD52
:10307800643E0020681B002008B51CF0FBF9034BD8
:103088001B7800EA931000F0010008BD681B0020BF
:10309800044B054A1B78D078C3F3401303EAD000E9
:1030A800704700BF681B0020EC3900202DE9F74F5E
:1030B800FFF758FF8246FFF763FF8346FFF76EFF6F
:1030C8000190FFF777FF8146FFF782FF0446FFF77D
:1030D800ABFF0546FFF7DCFF8046FFF7CDFF07464D
:1030E800FFF784FF0646FFF78FFF019B45EA0404BC
:1030F8009B0043EA4B0343EA0A0343EAC90343EA52
:10310800481343EA871343EAC61343EA0023E0B2AD
:1031180043EA0010BDE8FE8F044B987800F00F00DA
:10312800A0F10203584240EB03007047D619002073
:10313800044B987800F00F00A0F10102504240EBD8
:1031480002007047D6190020044B987800F00F0051
:10315800A0F10301484240EB01007047D619002056
:10316800054B987800F00F00A0F1060CDCF1000088
:1031780040EB0C00704700BFD6190020514AF0B54B
:1031880013781446012B29D003D3022B40F09880E2
:103198005EE04D484D4B047819786FF3C304047012
:1031A80001F0F80158786FF3C301197000F080013D
:1031B800C9B2002900F08480012111709C78062290
:1031C80004F00F04544302464148005D60F30602D0
:1031D8005A701A7861F302021A70F0BD3B494D78B3
:1031E8000B4625F07F00002838D00A7802F0080244
:1031F800D2B222B9344A117841F0080111709A7894
:1032080002F00F02012A04D12F4A117841F001017E
:10321800117015F07F0F53D119789E7801F00700CF
:10322800062206F00F0602FB0606294F5D78BE5DF2
:10323800013066F3060500F007005D7090FBF2F5BB
:1032480002FB150262F30201197002232370F0BD1C
:103258001E494D780B4625F07F0028B98B7860F31E
:1032680003038B701070F0BD174A11786FF3C30118
:103278001170997801F00F01012903D111786FF3CA
:103288000001117015F07F0F1AD119789E7801F09E
:103298000700062206F00F0602FB06060C4F5D78B3
:1032A800BE5D013066F3060500F007005D7090FB17
:1032B800F2F502FB150262F3020119700123237073
:1032C800F0BD00BF251A002098190020D61900204B
:1032D800F0A6020810B51F4A1F4B92F9031009B156
:1032E800002231E008B1032119701978032930D878
:1032F800DFE801F00209192C1178002929D01548B6
:1033080081700121197092F90200124920B1134B02
:103318001A786FF3861217E0487808B9032213E089
:1033280088700221197092F902100A4889B90B4A6B
:10333800147861F386141470026861F30F22D1B215
:1033480061F31742026001221A7010BD002111605A
:10335800197010BDFC1B002093190020F03B0020C1
:1033680070B543F6EF23044643F6F020012A08BF60
:1033780018460D460EF0D0FC2678C0B20640164C12
:103388000CD001201DF03AF943F6EE200EF0C4FCF3
:10339800236860F307036FF30F2314E02B781842B8
:1033A80012D030461DF02AF90C4B43F6EE201A884D
:1033B80066F34D321A800EF0AFFC2368C0B260F39A
:1033C800070360F30F23236094F9003013B1024B15
:1033D8000F22DA7070BD00BFFC1B0020901B00207C
:1033E80008B543F6FB200EF097FC014B187008BD9A
:1033F80094190020014B1870704700BF721B002001
:103408002DE9F0474FEAD2084BF25F79C14402F048
:1034180007030446012748460D469F4016460EF00E
:103428007BFCFFB2C1B215B921EA070100E03943BC
:1034380008F5D048484608F14E080EF063FC4046AF
:103448000EF06AFCC1B214B921EA070100E0394361
:1034580040460EF057FC254305D106483146BDE8E5
:10346800F04721F075BF03483146BDE8F04721F029
:1034780064BF00BFD9190020024B1A5C6FF3030226
:103488001A5470477F1A002070B50C46C10001F528
:10349800D2411B483F3108220EF04FFC0025184846
:1034A8002946EEB221F05FFF08B9237823BB154BFC
:1034B8002278EB5C1A421FD13046FFF7DDFFF60891
:1034C8004BF25F7030180EF027FC05F00703C0B20E
:1034D800184110F0010F0FD10B48294621F043FF86
:1034E80050B12946084821F033FF074B06F5D04074
:1034F8004E30995D0EF006FC0135402DCFD170BDE0
:10350800741B0020361A0020D919002038B546F659
:10351800960540242046FFF7AFFFA5F5D043094A9A
:10352800563BD15C11F0100F06D06FF30411D15443
:10353800284600210EF0E6FB0134E4B20135E92CFF
:10354800E8D138BD7F1A00203F287FB5054607D847
:1035580000F5E440C1300EF0DFFBC3B22BB925E122
:10356800964A1478002C00F02681954E725D02F080
:103578000F014C1C04F00F0464F303023F2D725535
:1035880033D8002C00F0178101339C4240F01081A1
:103598008C4B5A1992F88020522A725D03D161F33C
:1035A8000302725504E16FF30302EC081B1972550C
:1035B80093F8902105F0070352FA03F313F0010F73
:1035C80040F0F8802946804821F0B7FE7E4B04F58C
:1035D800D040195D4E3001240EF094FB2D190223C2
:1035E8000093019402951820DAE0002C00F0E380A3
:1035F800724B1B7801339C4240F0DA80735D05F50D
:10360800D0406FF303035630012173550EF07AFB57
:10361800735D43F010037355A5F14003DBB2032B30
:1036280007D8042200920133023201920293192032
:1036380031E0A5F14803DBB2032B0CD80422009239
:1036480001330332019202931A200121043A0B46F6
:103658000EF0E0FBAEE0502D07D1042300930124C7
:103668000333019302941B209AE0572D07D10423BA
:1036780000930124033301930294212090E0A5F1E3
:103688005B03DBB2012B09D804220092013302321A
:103698000192029322200121033AD8E75D2D06D139
:1036A800042300930193043B0293284662E05E2DB5
:1036B80007D10423009301330193053B02935E2055
:1036C80058E0A5F15F03DBB26F2B09D80422009202
:1036D800013392180192029333200121053AB6E78B
:1036E80005F13103DBB2032B07D804220092013322
:1036F8000332019202935F20A7E705F12903DBB2A9
:10370800012B07D80422009201330332019202935D
:1037180060209AE7DA2D07D1042300930124043BA3
:103728000194029361203BE0D92D07D10423009333
:10373800023B0193023B029362201BE0DD2D08D17E
:10374800042300930322043B019202936320012186
:103758007DE7DB2D06D104230093043B01930293FC
:10376800642007E0DC2D08D104230093043B019377
:10377800029370200121032269E7DE2D07D104237B
:1037880000930124023301930294682008E0E22D9B
:1037980010D10423009301240233019302946A2078
:1037A8002146032223460EF035FB04E01C4602E0C6
:1037B800002400E00124204604B070BD0000002071
:1037C8007F1A0020302C0020D9190020024B185CE9
:1037D800C0F30010704700BF7F1A0020F8B5082218
:1037E8000E4600210746FCF7D5FD46F63F15002496
:1037F8003378234113F0010F08D0294606480822E0
:103808000EF09BFA3846044921F065FD013408356D
:10381800042CEDD1F8BD00BF7E1B0020024846F6FF
:103828004E0108220EF089BAD919002070B5044655
:1038380000F56A5044300EF06FFA0B4D06462B78AF
:1038480013F0010F02D1CC2022F0B2FB2B8843F0F9
:1038580001032B80054B1E55054B13F8242042F01D
:10386800010203F8242070BD901B0020BA19002023
:10387800A9190020024B185C084100F001007047AC
:10388800361A002070B505460024094BE0B2E61848
:10389800E35C4BB12946FFF7EDFF28B100233370F5
:1038A8000448214621F054FD0134402CEDD170BD6F
:1038B800B21B0020C619002038B50546002428464A
:1038C800E1B2FFF7D7FF10B1044BE35C23B9013431
:1038D800042CF4D1002038BD012038BDBA190020CD
:1038E80038B505460EF07CFDA0B100242846E1B2AB
:1038F800FFF7C0FF40B1084B13F8243013F0010F55
:1039080002D0064BE35C23B10134042CEED1002035
:1039180038BD012038BD00BFA9190020BA19002000
:10392800F8B5114800214022FCF734FD46F63F1552
:10393800002401270D4829460822A7400EF0FDF96A
:10394800FFB200260948314621F00DFD20B1064B93
:10395800F25C47EA0202F2540136402EF2D10134F9
:103968000835042CE5D1F8BD361A00207E1B00204E
:103978002DE9FF4100263446B0461A4B1B782341F7
:1039880013F00102184B23D0184F1D5D17F824308F
:10399800A84538BFA84613F0010F1AD0CDB965F372
:1039A800000307F8243023B20122F71902935B20A1
:1039B80029462B46009201950EF02CFA7B78B878B0
:1039C800F9781843621C2B460095FEF799FE00E033
:1039D8001A5501340436042CCFD1054B83F80080E6
:1039E800BDE8FF8194190020BA190020A919002008
:1039F8009219002010B50C4B1B78A3B10B4B1B7808
:103A08008BB100240A48214621F0ADFC40B1094899
:103A1800214621F0A8FC18B920460121FEF79EFF97
:103A28000134402CEED110BDF91800206615002095
:103A38009A1B00202A2300202DE9F043324C334AF8
:103A4800238800266FF386136FF3C4032380304B5B
:103A5800304F85B016701E709146984617F8013B96
:103A68005BB32278D20052B243EAA2122388402ED6
:103A780062F3C40343F0400323801ED00025304680
:103A8800E9B2FFF7F7FEA8B117F8013C13F0010FF0
:103A980006D00122AA4099F800100A4389F80020AC
:103AA80013F0020F06D00123AB4098F8002013430F
:103AB80088F800300135042DE1D10136F6B2412EE7
:103AC800CCD1237803F04005EDB2D5B903F0240337
:103AD800042B0BD1FFF78EFFFF23009340202946CC
:103AE80001222B46019502950EF094F923880022B5
:103AF8006FF345136FF382036FF3C4032380064B00
:103B08001A7005B0BDE8F083901B00208C3B0020A4
:103B1800A93B0020E4190020731B002010B50024E5
:103B28000548214621F01FFC08B9044BE054013434
:103B3800402CF5D110BD00BF6A1B0020E4190020FD
:103B480010B5127804469DF80810DAB1D3B111B156
:103B58000D4921F0B5FBACB1082246F64E010B48E1
:103B68000EF0EBF82146094821F0B5FB0749082279
:103B780046F64E000EF0DBF805480449BDE8104053
:103B880021F0BFBB10BD00BFC82D00207C1900204C
:103B9800D919002030B5064B04781D7824EA0504AD
:103BA8000C7001781B7823EA0103137030BD00BF45
:103BB8009419002038B50A4D002415F8013F2D2B23
:103BC80009D0532B07D0542B05D0462B03D00548DA
:103BD800214621F0BDFB0134402CEED138BD00BF99
:103BE800AF2C00209A1B002010B50F4821F060FB75
:103BF80000240E48214621F0B6FB80B10C4BE31897
:103C080093F88030482B06D003D82D2B03D0462BB1
:103C180000E0542B03D10448214621F08EFB0134E7
:103C2800402CE6D110BD00BF261A00209A1B0020A8
:103C3800302C0020094A0A4B117831B1997801F0EB
:103C48000F01814201D0002111709A7860F30302BC
:103C58009A705A7842F080025A707047251A0020EC
:103C6800D61900202DE9F0431F4685B07C4BDDF8BE
:103C78003090154604461A7888460023794911F889
:103C8800231011F0010F05D001219940C1F10F0156
:103C980001EA02020133042BF0D1734B1A70002C95
:103CA80000F0878014F0010F0CD00121FF230026BB
:103CB800009352200B460A46019602960EF0AAF887
:103CC8006A4B1E7014F0020F0DD0FF2301210093E0
:103CD800FF3B019302930A460B4653200EF09AF8D5
:103CE800624B01221A7014F0040F0DD0FF2301213A
:103CF8000093FF3B019302930A460B4654200EF0B3
:103D080089F85A4B02221A7014F0080F0DD0FF23BD
:103D180001210093FF3B019302930A460B4655206D
:103D28000EF078F8514B03221A7014F0100F0DD0D2
:103D3800FF2301210093FF3B019302930A460B46A0
:103D480056200EF067F8494B04221A7014F0200F21
:103D58000DD0FF2301210093FF3B019302930A46F4
:103D68000B4657200EF056F8404B05221A7014F0F7
:103D7800400F0DD0FF2301210093FF3B01930293D5
:103D88000A460B4658200EF045F8384B06221A70A2
:103D980014F0800F0DD0FF2301210093FF3B019306
:103DA80002930A460B4659200EF034F82F4B07228F
:103DB8001A70B8F1000F1CD02C4B09221A7000247D
:103DC8003846214621F0CFFA60B1FF230093FF3B2C
:103DD8000193631C1BB2012102935A200A460B4629
:103DE8000EF018F821463846013421F0B1FA402C7B
:103DF800E6D1CDB100244846214621F0B4FA80B17D
:103E0800012D0ED104230093631C1BB208260293D4
:103E180074202B462946032201960DF0FBFF134B15
:103E28001E700134702CE6D10F481149114AFFF772
:103E3800B1FE114B00221A70013200920632019233
:103E4800083202920A490B4A074809F071FD0B4BE8
:103E58003C2251201A7005B0BDE8F0430EF0ACBB0F
:103E680094190020A9190020081D0020856300204E
:103E7800F11D0020E41D0020CD1C0020B9190020F0
:103E880037B5FFF713F904460E4821F03FFAD0F191
:103E9800010538BF00250C480E211CF091F910B11E
:103EA80014F4807F03D124B95DB1224602E00122D7
:103EB80000E00022044B204600932946014BFFF7FF
:103EC800D1FE3EBD771A002084190020054B03EB74
:103ED800D00393F8903100F0070053FA00F000F097
:103EE80001007047302C002010B50F4B04461B789A
:103EF80013F0010315D0FFF7DFFC28B90B4B1B1992
:103F080093F88030462B0DD10EF06AFA18B9204686
:103F1800FFF7DCFF30B10648214621F00EFA0120F8
:103F280010BD184610BD00BF901B0020302C00208B
:103F3800771A0020024B1878003818BF0120704704
:103F4800B919002010B5034C04EB8303587099701D
:103F5800DA7010BDA919002010B500240948002105
:103F680000190E220E34FCF715FAB4F5E07FF5D1EE
:103F7800054A00231370054A002199520233AA2BDF
:103F8800F9D110BD6815002063150020661E0020B9
:103F9800044B187800F02400A0F10403584240EBC9
:103FA80003007047901B00207FB5474B04461B78E1
:103FB8000E46AA2B78D04548214621F0D4F905466B
:103FC800002871D12046FFF78FFF00286DD14048A7
:103FD800214621F0C8F950B93E48214621F0C3F9DD
:103FE800054620B92046FFF7AFFA00285DD13A4BC5
:103FF8001B7823B9394B1B7813F0010F09D1384BC3
:10400800DB7803F02003DBB21BB9364B032283F8BD
:104018004020012E05D82E48214621F0A4F940B1B0
:1040280042E0022E07D12B48214621F09CF910B11D
:104038003AE0274800E02748214621F07EF92A483F
:10404800214621F085F9022E15D1012529460322A2
:104058002B4600964A206619019502960DF0DAFE65
:104068002046FEF785F800230246314618200093C3
:10407800FEF746FB19E0012E09D102230093631CC9
:1040880002930196122031460322334609E07EB995
:104098000121022300936318029301911120032246
:1040A8000B460DF0B7FE03E00025284604B070BDAE
:1040B8002046FEF75DF802460120002321180093F0
:1040C8000125FEF71DFBF0E7721B0020D91900201F
:1040D80099190020F21B002094190020611E00206D
:1040E800EC390020E4190020A21B00202DE9FF472D
:1040F80004460D467548214621F035F981460028C9
:1041080040F0DF802146714821F017F970482146B8
:1041180021F01EF96F4E0DBB01274FF00208E3197D
:1041280002934246032039463B46CDF8008001976A
:104138000DF070FE327862B10EF052F9024630B1DD
:10414800337840461E33009321462A4604E0009007
:1041580000E00092404621463B4628E0012D2BD145
:104168005D4B04F5E440C1301F5D0DF0D5FD07F04F
:104178000F07874209DA631C022202930E202946A0
:104188002B46009201950DF045FE327892B10EF063
:1041980027F9024638B14F4B0D201B7821461E33B4
:1041A8000093002202E000900D2021460123FEF733
:1041B800A7FA5EE00092F7E7022D0BD101230193E5
:1041C800E3180293142049462A464B4600950DF001
:1041D80021FE4EE0032D4CD101272A464FF002085C
:1041E80004EB070A4D2039463B46CDF8008001977D
:1041F800CDF808A00DF00EFE35783DB30EF0F0F8BE
:10420800024630B1337840461E33009321464A4671
:1042180002E00090214640463B46FEF771FA0EF058
:10422800DFF8671C054648B12046FDF7A1FF337843
:1042380002461E3300931A2039462CE02046FDF72B
:1042480097FF0095024639461A202DE021462A4656
:104258003B4640460095FEF753FA2046FDF788FF97
:10426800514602462B461A200095FEF749FA384671
:1042780028E03578EDB10EF0B3F804F11C060546D8
:1042880058B12046FDF774FF124B02461B783046A2
:104298001E330093611C002307E02046FDF768FFEA
:1042A800009502463046611C2B46FEF729FA01208C
:1042B80008E02046FDF75CFF0095024604F11C006B
:1042C800F1E7002004B0BDE8F08700BF9A1B00208A
:1042D800A21B0020FA1B00207F1A0020064B1B1887
:1042E80093F84001492804D0452814BF0320022030
:1042F80070470120704700BF302C00202DE9F041A5
:10430800244F00243C702448214621F02CF8E5B2C3
:10431800224B002837D01E5D3B789E4200D303B95C
:104328003E70002E30D131461C484022FCF732F84E
:104338001B4B1C4803EBD50393F8888104F0070353
:1043480048FA03F8214608F0010821F00CF868B98A
:10435800B8F1000F02D02846022101E02846314674
:10436800FFF7C4FE28460EF027F90DE0B8F1000F5C
:104378000AD12846FFF7B2FF0B4BDB7803F0200386
:10438800DBB20BB9094B18550134402CBBD1BDE841
:10439800F08100BFFA1B0020C6190020B21B0020C4
:1043A800302C00209A1B0020EC390020E419002052
:1043B8002DE9F04F914B8BB01B7813F0010F06D00D
:1043C8008F4B1A786FF386121A7001F07CBA8D49F8
:1043D8008D4A0B7810788D4D984218BF8C49137010
:1043E80018BF0B706B7803F00803DBB24BB143F6D0
:1043F800CF200DF091FC864B18702B886FF3CB23E0
:104408002B80844B1B78AA2B08D18349AA3B0B70BD
:104418002B8843F080032B8000F0BEBE6A787B4B6C
:1044280002F01002D2B27D4CA2B11A886FF30C329E
:104438001A807B4B1B7823B97A4B1B7813F0010F3A
:1044480008D1E37803F02003DBB21BB9764B0322D3
:1044580083F840202368754F6FF3186323603A7818
:1044680002F00202D2B232B96B494A781AB16B4AE9
:1044780043F080731360E67816F0010648D05D209B
:10448800FFF7A4F900285AD16B78DFF8808103F090
:104498000203DBB22BBB5D30FFF756F8064600BBC4
:1044A800B8F80030012143F40073A8F80030042361
:1044B80003220093019302900B460D200DF0AAFCF5
:1044C80045200EF079F83146012233460D2000963A
:1044D800FEF716F909203146324601230096FEF709
:1044E8000FF96B7803F00203DBB243B34C4B1B7834
:1044F80023B94C4B1B7813F0010F20D1E37803F05C
:104508002003DBB2DBB9484B032283F8402016E0D6
:104518006B7803F00203DBB26BB1314632460123FC
:104528000A200096FEF7ECF88D203146012233462A
:104538000096FEF7E5F82B886FF349232B80236854
:10454800354A6FF35963236093787BB1D37823B9E5
:104558003B7813F00C0F05D108E03B7803F00C030F
:10456800042B03D0236843F000732360E17801F043
:104578000201C9B200295BD05E20FFF727F90028A5
:1045880065D16B78214F03F00403DBB2EBB95E30E1
:10459800FEF7DAFF0646C0B93B88012143F4806381
:1045A8003B800423009301330322019302900B46BE
:1045B80017200DF02FFC45200DF0FEFF0D20314691
:1045C800012233460096FEF79BF86B7803F004034C
:1045D800DBB2002B3BD0124B1B7823B9114B1B7855
:1045E80013F0010F33D1E37803F02003DBB273BB80
:1045F8000D4B032283F8402029E000BF091D00204D
:10460800F03B00207C1B00207D1B0020901B00201D
:10461800FB1B0020721B002064130020EC390020D3
:1046280094190020611E0020E41900202E2C00207F
:104638006B7803F00403DBB22BB18D2001220B460B
:104648000091FEF75DF82B886FF38A232B8023688F
:104658004FF05F0B6FF3DF732360002696E0069838
:10466800F9B21BF0EBFD002875D04FF436637343A5
:10467800342202FB0733A749A8F15E0ACB1803F1DD
:1046880008021B7A5FFA8AFA13F001034DD02368F7
:10469800404643F0004323600592FFF797F8059AD8
:1046A800002864D1937813F0040F20D14046FEF718
:1046B8004BFF059A8146D0B99378012143F0040352
:1046C800937004230093DB180322019332200B46D6
:1046D800CDF808A00DF09EFB4A200DF06DFF0C20D0
:1046E800514601224B46CDF80090FEF709F84FF4E9
:1046F80036637343342202FB0733864AD3189B7A06
:1047080013F0040F33D0844B1B7823B9834B1B78E9
:1047180013F0010F2BD1E37803F02003DBB233BB96
:104728007F4B032283F8402021E0927812F0040F97
:1047380005D08C20514601220093FDF7E1FF4FF48C
:1047480036637343342202FB07337249CB189A7AD3
:104758006FF382020AE04FF436637343342202FB9C
:1047680007336C4AD3189A7A60F382029A72013737
:1047780008F10108382F5FFA88F87FF470AF013626
:104788000BF1380B022E5FFA8BFB04D0F3B20693C1
:10479800D846002763E72368624923F080636FF3F4
:1047A8009E7323600B79002B00F0B9835E4ADFF813
:1047B8007CB106924FF0CF0800261BF8011F374640
:1047C8000136002952D0236808F1710A43F080634A
:1047D8005FFA8AFA23605046FEF7F8FF00285CD19A
:1047E80029237B43DFF8489119F8032012F0100FB2
:1047F80023D150460593FEF7A7FE059B8246E0B9F4
:1048080019F80320012142F0100209F803200423BB
:1048180000930233019333B2032202930F200B4615
:104828000DF0F8FA45200DF0C7FE0D205146012283
:104838005346CDF800A0FDF763FF29237B4319F801
:10484800033013F0100F28D0334B1B7823B9334BA8
:104858001B7813F0010F20D1E37803F02003DBB2BB
:10486800DBB92F4B032283F8402016E029237B4332
:10487800DFF8BC9019F8033013F0100F05D08D2025
:1048880001220B460091FDF73BFF29237B4319F8D2
:1048980003206FF3041209F80320069B13F8011F85
:1048A8000693002946D02368404643F0804323609E
:1048B800FEF78CFF002854D14FF0290909FB07F9AE
:1048C800DFF86CA01AF8093013F0200F49D14046E0
:1048D800FEF73AFE0746002843D11AF809300121AD
:1048E80043F020030AF809300423009303330193AB
:1048F80033B2032202934B200B460DF08BFA502063
:104908000DF05AFE1920394601223B460097FDF763
:10491800F7FE26E0643E002094190020611E002066
:10492800E419002064130020B33A0020D83A00208C
:10493800E23A002029237B43DFF8A89219F80330D4
:1049480013F0200F05D0992001220B460091FDF7A6
:10495800D7FE29235F4319F807306FF3451309F889
:10496800073008F10108042E5FFA88F87FF425AFB4
:10497800934B1978002945D02368E22043F08063DF
:104988002360FEF723FF00284BD18E4B1A789846F8
:1049980012F0400F1FD1E230FEF7D6FD0746D0B91E
:1049A80098F80030032243F0400388F8003000965E
:1049B8000623033E314601936920334602960DF0E3
:1049C80029FA45200DF0F8FD0D20394632463B46C0
:1049D8000097FDF795FE98F8003013F0400F20D0AF
:1049E800794B1B7823B9794B1B7813F0010F18D139
:1049F800E37803F02003DBB29BB9754B032283F8FD
:104A080040200EE06F4E337813F0400F05D08D2014
:104A180001220B460091FDF773FE33786FF386137E
:104A280033706C4B197800292DD02368502043F03F
:104A380080432360FEF7CAFE002833D1614E3378E5
:104A480013F0200F2ED15030FEF77EFD074648BBED
:104A58003378032243F020033370042301260093A4
:104A68000333314601931020334602960DF0D2F9F4
:104A780050200DF0A1FD1920394632463B460097DB
:104A8800FDF73EFE0EE04F4E337813F0200F05D0B1
:104A9800992001220B460091FDF732FE33786FF31F
:104AA800451333704C4B1978002946D02368DE2013
:104AB80043F080632360FEF789FE00284CD1474B02
:104AC8001A78984612F0400F20D1DE30FEF73CFDF0
:104AD8000746D8B998F80030012643F0400388F813
:104AE80000300423009302333146032201936720E8
:104AF800334602960DF08EF945200DF05DFD0D2030
:104B0800394632463B460097FDF7FAFD98F80030E3
:104B180013F0400F20D02C4B1B7823B92B4B1B785C
:104B280013F0010F18D1E37803F02003DBB29BB92F
:104B3800274B032283F840200EE0284E337813F0E9
:104B4800400F05D08D2001220B460091FDF7D8FDBE
:104B580033786FF386133370214B1978002943D0CB
:104B68002368572043F080432360FEF72FFE002878
:104B780049D11A4E337813F0200F44D15730FEF73D
:104B8800E3FC074600283ED13378032243F0200394
:104B980033700423012600930333314601931F2009
:104BA800334602960DF036F950200DF005FD192018
:104BB800394632463B460097FDF7A2FD23E000BF89
:104BC800A83A0020863A002094190020611E00208F
:104BD800E4190020F03900203B3A0020523A002026
:104BE800403A0020E23A0020834E337813F0200F39
:104BF80005D0992001220B460091FDF781FD3378FD
:104C08006FF3451333704FF000084FF05B094FF016
:104C1800D70A4646794B08F10108F15C784F00291C
:104C280049D02368484643F080632360FEF7CEFDF1
:104C3800002852D124237343FA5C12F0200F22D1AA
:104C480048460593FEF780FC059B8346D8B9FA5C75
:104C5800012142F02002FA54042300930233019305
:104C68000FFA88F30322029320200B460DF0D2F8A6
:104C780045200DF0A1FC0D20594601225B46CDF8D8
:104C880000B0FDF73DFD24237343FB5C13F0200FB8
:104C980023D05C4B1B7823B95B4B1B7813F0010FB7
:104CA8001BD1E37803F02003DBB2B3B9574B0322DF
:104CB80083F8402011E024237343FB5C13F0200F9A
:104CC80005D08D2001220B460091FDF719FD242304
:104CD8007343FA5C6FF34512FA544D4BF15C0029AB
:104CE80033D02368504643F080432360FEF76EFDBF
:104CF80000283ED1242303FB06735A7812F0200FB4
:104D080037D150460593FEF71FFC059B834680BBB1
:104D18005A78012142F020025A7004230093033389
:104D280001930FFA88F3032202934C200B460DF0EF
:104D380071F850200DF040FC1920594601225B46BD
:104D4800CDF800B0FDF7DCFC13E0242303FB067369
:104D58005B7813F0200F05D0992001220B460091B3
:104D6800FDF7CEFC242303FB06735A786FF3451234
:104D78005A70284B2422F35C002B4FD07243BB5C43
:104D8800C3F3801BBBF1000F1DD123490978D1B1B2
:104D980043F04003BB5404230093DB180121019323
:104DA8000FFA88F3032202932F200B460DF032F8F6
:104DB80047200DF001FC0920414601225B46CDF851
:104DC80000B0FDF79DFC24237343FB5C13F0400FF8
:104DD80035D00C4B1B7823B90B4B1B7813F0010F04
:104DE8002DD1E37803F02003DBB243BB074B03224A
:104DF80083F8402023E000BF523A0020B13A002057
:104E0800F339002094190020611E0020E4190020C5
:104E1800A93A0020423A0020483A00207243BA5C7E
:104E280012F0400F05D08920414601220093FDF77A
:104E380067FC24237343FA5C6FF38612FA54013635
:104E48000AF1010A09F10109022E5FFA8AFA5FFAEA
:104E580089F97FF4DFAEDFF854A24827023E1AF83A
:104E6800013FB04601362BB9894BF31813F8011CE2
:104E7800002937D02368384643F080432360FEF783
:104E8800A5FC002847D14FF0370909FB08F9DFF8DE
:104E980020B21BF8093013F0200F3CD13846FEF73A
:104EA80053FB8046002836D11BF80930012143F016
:104EB80020030BF80930042300930333019333B222
:104EC8000322029313200B460CF0A4FF50200DF090
:104ED80073FB1920414601224346CDF80080FDF7B7
:104EE8000FFC18E0372303FB08F3DFF8C49119F827
:104EF800033013F0200F05D0992001220B460091B2
:104F0800FDF7FEFB372303FB08F819F808306FF3A9
:104F1800451309F808300137042EFFB29FD1A6784F
:104F280006F00806F6B2002E40F03681594906917F
:104F38005FFA86F8B8F1000F0CBF4022702247F6DE
:104F48009B530992079349F69E69002447464FF4FC
:104F5800E07A0AFB06FA4F495FFA84F8514408914F
:104F68000846214620F0FFF948B94A480AF1700A74
:104F78005044214620F0F7F9002800F0FA80454A0D
:104F88004FF4E07A0AFB062A0AF1E00A5046214665
:104F980020F0E9F9002840F0EC805046214620F046
:104FA800CCF9DFF810A10FB9484600E007980CF0DB
:104FB800B3FE8AF800009AF80000DFF8F8B000287D
:104FC80000F0D7800138C0B28BF800000BF07AFAF5
:104FD800002840F0CE809BF8000000F56A507C3035
:104FE8000CF09AFE2C4BC0B218701FB92B4B19F855
:104FF80003A003E006990B1993F850A100EA0A0AE6
:10500800BAF1000F00F0B5800898214620F0ABF9FE
:10501800DFF894B000B31F4A4FF4E07000FB06209D
:105028002146703020F09FF9B0B91D49012F0B7847
:105038004AEA030A8BF800A058D13823B8FBF3F2E8
:1050480003FB12834FF436614A43DBB2342101FB80
:105058000323144AD31843E00E4B4FF4E07000FBCF
:1050680006302146703020F07EF938B10898214684
:1050780020F079F910B90A490B7804E0084A137846
:105088001AEA030F18D023EA0A0A8BF800A02DE0C9
:10509800793A0020A8280020A21D0020528EFF1F68
:1050A80094190020643E0020081D0020813A002049
:1050B8001C3C0020761A00204AEA030A012F8BF8CC
:1050C80000A013D13823B8FBF3F203FB12834FF48B
:1050D80036614A43DBB2342101FB03238E49CB18E6
:1050E80093F8302042F0200283F830208B488C4916
:1050F8008C4AFEF74FFD8A4B1B781BB1FDF7D6FF94
:10510800002836D18648884913F0ACF868B10DF00C
:1051180067F970BB844808F07FFC50BB01238248C4
:1051280082497F4A0093FEF70BFD00230093804AD3
:10513800013301931378794802937949794A7B4B73
:1051480008F0F6FB012F14D13823B8FBF3F203FB68
:1051580012884FF436635A435FFA88F8342303FB06
:1051680008236D49CB1893F8312042F0010283F8E7
:1051780031200134079A0999E3B205328B4209F1CB
:1051880001090792FFF4E3AE069A013602F5E072D0
:10519800022E06927FF4CCAE664E73786FF3C71377
:1051A80073702B7803F08002D2B2002A00F0E680F8
:1051B80061490C78002C40F0E18003F02403042BB3
:1051C8000BD1FEF717FCFF23009340202146012254
:1051D8002346019402940CF01DFE2B8800246FF3E3
:1051E800C7136FF3820364F3451364F3410364F355
:1051F8000003524A64F3492364F38A2314702B8012
:105208004F4B1A7842F0C0021A705A7864F3C302FE
:105218005A70FEF7CFFC4B4820F04AF84A4820F075
:1052280047F84A4820F044F8412249482146FBF70C
:10523800B1F8484B1A7802F0DF0264F304121A70CE
:1052480093F8292002F0DF0264F3041283F829207E
:1052580093F8522002F0DF0264F3041283F852201C
:1052680093F87B2002F0DF0264F3041283F87B20BA
:10527800394B1A7802F0DF0264F386121A70374B42
:105288001A7864F345121A7093F8372064F34512BC
:1052980083F8372093F86E2064F3451283F86E2064
:1052A80093F8A52064F3451283F8A5202C4B1A78AF
:1052B80002F0DF0264F386121A702A4B5A7864F3FC
:1052C80045125A701A7802F0BF0264F345121A7038
:1052D80093F8252064F3451283F8252093F82420B9
:1052E80002F0BF0264F3451283F8242011E04FF462
:1052F80036626243342101FB03221B4901335218F1
:105308009178382B6FF382019170F0D10134022C1F
:105318002CD00023EBE700BF643E0020081D0020CE
:10532800F11D0020E41D0020A1190020CD1C002043
:10533800A21D0020D619002064130020731B002032
:10534800F03B0020F21B002099190020C61900200C
:10535800E4190020E23A0020863A00201C3C002094
:10536800523A0020F33900206C3E00200422734892
:105378000021FBF70FF8724B00221A70714C23784A
:10538800002B4DD12978704A01F00201C9B201B34E
:105398006E49487863F3820048706D4811884778F1
:1053A80063F34D3163F3C30741F080014770118007
:1053B800CA2020F0FDFDC62020F0FAFD20F046FEB0
:1053C800644A13780BB90DF083F9FEF79FF8FEF7DE
:1053D800C3FD614A2B8811786FF341036FF3000115
:1053E8006FF3000311705D48002140222B80FAF70B
:1053F800D1FF5B481FF05CFF5A481FF059FF5A481D
:105408001FF056FF59481FF057FF04224B48002150
:10541800FAF7C0FF4A4A00231370554A13706AE02E
:105428002F7807F00203DBB293B917F001070FD109
:105438004B481FF03DFF2378F8B23B4113F0010FB2
:1054480003D0FEF7F3F90CF0C1FF0137042FF2D1B6
:105458002B783D4F13F0010F25D0FEF711FD3B8847
:1054680043F002033B80FEF783FA354B93F8008044
:10547800B8F1000F14D1CA2020F09AFDCD2020F0F9
:1054880097FD3B883B4868F300033B80324B1A7812
:1054980042F001021A701FF00BFFFEF737F802E026
:1054A8000120FEF7C7FB2B7803F00202D2B212B339
:1054B8002F4A12782AB113F0010F02D10220FEF709
:1054C800B9FBFEF71BFF2C4926481FF00FFF2549A3
:1054D80025481FF0F5FEFEF787FB224927481FF0F5
:1054E800EFFE274925481FF0F6FEFEF717FB1F4879
:1054F8001C491FF006FF204922481FF0E1FE15490C
:105508000B780BB9FEF798FA737803F08003DBB2D7
:10551800002B3FD1FEF73CFD30B143F6EC200CF0F8
:10552800FBFB08B1062033E0FEF704FD08B10520B7
:105538002EE00DF0B7F938B3032029E0BA1900209E
:105548009219002094190020901B0020073C00208D
:10555800F03B00206413002098190020B21B0020A3
:10556800593100206A1B0020C6190020AA1B002000
:10557800FA1B0020771A0020D91900209A1B002056
:10558800261A0020BE19002001F066F810B1042088
:10559800FEF750FB6C4B1B781BB173786FF3C71386
:1055A80073706A4A137813B1694B1B78CBB12B78A7
:1055B800684E03F04403402B13D10021BF330093FE
:1055C8003F200B460222019102910CF023FC338804
:1055D80043F6CE2043F0040333800CF09DFB5E4B72
:1055E80018705A495D4E0B789BB1594B197881B99F
:1055F8002A78584B02F04002D2B252B11A8861F3AD
:1056080082021A80337823B943F6CE200CF084FB4B
:1056180030702A78DFF83C8102F00400C0B2504BA9
:1056280000287FD002F02000C0B24B4F90B11A780A
:10563800002042F0C0021A70FDF74CFE3B78002BA8
:1056480076D1B8F8002063F3820263F34512A8F814
:1056580000206DE0D20052B219789211D2B241F016
:10566800C00112F0010F197003D0C9B260F3C7115D
:10567800197012F0020F03D01A786FF386121A709D
:105688001B78374A03F04003DBB273B9537843F011
:1056980008035370237843B12B8843F400532B80BD
:1056A800304B5A7842F004025A700120FDF712FE7E
:1056B80043F6CD200CF030FBC0B20128307002D187
:1056C800264B02221A703C78002C31D1FEF792F951
:1056D800FF2301220093402021462346019402948F
:1056E8000CF098FB2B8843F6CD2043F020032B8049
:1056F8000CF012FB184B1C4A1870154B14701A78D2
:105708000AB1013A1A70197891B9104A13787BB125
:10571800FF230093412002220B46019102910CF0D5
:1057280079FB05E01A7842F0C0021A70FDF7D2FD45
:105738000DF068F80D481FF0E9FD0D4BD0B91A7847
:1057480060F3820219E000BFAA5800207C1B0020E9
:10575800FB1B0020901B0020731B0020E319002076
:10576800F03B0020073C0020641300202E1A002084
:10577800981900201A7842F004021A706A7853487F
:1057880012F001011A780CBF61F3410242F00202E3
:105798001A704F491FF0B5FD4E494C481FF09BFD4C
:1057A8004A484D491FF097FD3378012B40F08B8014
:1057B8002B8800246FF349236FF38A232B80474BF0
:1057C80041221C7021464648FAF7E4FD45481FF07F
:1057D8006FFDFEF7EFF93F481FF06AFD3E481FF0E6
:1057E80067FD414B1A7802F0DF0264F304121A7065
:1057F80093F8292002F0DF0264F3041283F82920C9
:1058080093F8522002F0DF0264F3041283F8522066
:1058180093F87B2002F0DF0264F3041283F87B2004
:10582800324B1A7802F0DF0264F386121A70304B9A
:105838001A7864F345121A7093F8372064F3451206
:1058480083F8372093F86E2064F3451283F86E20AE
:1058580093F8A52064F3451283F8A520254B1A7800
:1058680002F0DF0264F386121A70234B5A7864F34D
:1058780045125A701A7802F0BF0264F345121A7082
:1058880093F8252064F3451283F8252093F8242003
:1058980002F0BF0264F3451283F8242011E04FF4AC
:1058A80036626243342101FB032214490133521842
:1058B8009178382B6FF382019170F0D10134022C6A
:1058C80001D00023EBE70BB0BDE8F08FDE350020F8
:1058D8009A1B002099190020F21B0020E3190020D0
:1058E800E4190020C6190020E23A0020863A002078
:1058F8001C3C0020523A0020F33900206C3E002066
:105908002DE9FF4104460D460CF0A6FFA04B1A19DD
:1059180092F880709F4A98461278AA2A0AD1A7F16D
:105928004F03DAB20B2A00F2AD819B4A5BB29A4070
:1059380040F1A881994B0C2202FB04335A7A0833B0
:10594800AA42C0F09F81FF2A00F09C81FF229A7032
:10595800934808EBD403214693F888511FF003FDC0
:105968000646002840F08E8104F007031D41502FA1
:1059780005F0010500F0268114D8462F00F0F280CA
:1059880009D8412F00F09E80452F00F01B812D2F54
:1059980040F0768134E0482F00F0C5804F2F40F06A
:1059A8006F810EE0542F67D006D8522F00F08A80FE
:1059B800532F40F065811CE0A7F15903012B00F239
:1059C8005F81784821461FF0CEFC0646002840F04B
:1059D80059815A2F01D1744802E0592F04D17348D4
:1059E80021461FF0AAFC54E121466F481FF0A5FC90
:1059F800F5E76F4821461FF0B6FC002800F0428109
:105A08006C4821461FF0AFFC8046002840F03A81E0
:105A1800214668481FF091FC674821461FF098FC12
:105A28000227012655B1A419142041463A46434697
:105A38000097019602940CF0EDF92AE129463A46BE
:105A4800334604F101080A2000970196CDF8088032
:105A58000CF0E0F92046FCF78BFB414602462B464A
:105A680013200095FCF74CFE384629462A46334653
:105A78000095FCF745FE0CE14E4821461FF073FCEB
:105A88000746002840F005810126022231463346A8
:105A9800A5193E200092019602950CF0BBF920460C
:105AA800FCF766FB294602463B4614200097FCF7A4
:105AB80027FE21463F481FF040FC21463E481FF084
:105AC80047FCE6E03A4821461FF04DFC0646002810
:105AD80000F0DF80374821461FF045FC064628B90C
:105AE8002046FDF731FD002840F0D380002D40F01E
:105AF8008E802046FEF7F8F9002840F0C580204641
:105B0800FEF7ECFB2D4BDB7803F02003DBB20BB97F
:105B18002B4B1855412F00F08880522F40F0B08051
:105B28002046012183E0234821461FF01CFC28B9A8
:105B38002046FDF709FD002840F0A480002D66D11D
:105B48002046FEF7D1F9002840F09E801B4BDB78F9
:105B580003F02003DBB2002B67D1194B032283F833
:105B6800402062E0134821461FF0FDFB064628B995
:105B78002046FDF7E9FC002840F08B802046FEF720
:105B8800B3F900287ED1002D41D1204603214EE0F3
:105B9800302C0020721B002000003080F02D0020E7
:105BA800D919002088290020A828002018290020B9
:105BB8006A1B00209A1B0020A21B0020EC39002041
:105BC800E4190020354821461FF0CDFB0646002881
:105BD8005FD02046FDF784FE20B1214630481FF0F3
:105BE800ACFB4FE0502F28D12E4B1B782BBB204607
:105BF800FDF762FE08BB2C4821461FF0B4FB0646A1
:105C080020B92046FDF7A0FC002842D115B1204656
:105C180002210CE02046FEF761FB244BDB7803F001
:105C28002003DBB20BB9224B185520460021FEF7A2
:105C38005DFA061E18BF01262BE02046FDF73CFE44
:105C48000546F8B91B4821461FF08DFB0646D8B912
:105C58002046FDF779FC0746D8B9164821461FF0BB
:105C68006CFB154A135D8BB910494E7806F0200677
:105C7800F6B26EB908EB040393F80031135508E047
:105C8800012606E0002604E02E4602E03E4600E03B
:105C98001E46304604B0BDE8F08100BF6A1B0020F4
:105CA800771A0020FA1B00209A1B0020EC390020EC
:105CB800E4190020C6190020B21B0020032210B5E9
:105CC80005490648FAF73CFE054806490222BDE8A0
:105CD8001040FAF735BE00BF03260020040200205A
:105CE800090200200126002070B5834B1B7813F0B1
:105CF800010F0AD00CF07CFB38B100207F4902F07C
:105D080089FE7F4B7F48197847E07F4D2B78002B21
:105D180048D00CF073FB002844D07C4B1B7863B947
:105D28007B4B5B7813F0010F07D00CF059FB20B9BF
:105D3800FEF72EF908B10320BEE0764C207870B14A
:105D48000020754902F066FE21780122734802F0AE
:105D580087FE00201021621C07F0D2FA02E0704989
:105D680002F058FE6F4C684807F0F0FA2378002BD1
:105D780000F018810CF03CFB002800F013816A4900
:105D88006A481022FAF7DCFD68485B21FAF780FBC5
:105D9800002800F00781217801308322BDE8704097
:105DA80002F05EBE624C237803F00503012B5DD13F
:105DB8000020604902F02EFE202110225E48FAF7EA
:105DC800E9FA601D5D490322FAF764FD40BBE01C57
:105DD8005B490222FAF75EFD30B95A48FAF72AFD04
:105DE8005849024654480BE0E01C57490222FAF78A
:105DF80051FD40B95548FAF71DFD544902464E4831
:105E0800FAF79EFD0EE0E01C51490222FAF742FD26
:105E180030B95048FAF70EFD4E4902464648EFE7BA
:105E2800FFF74CFF6278303AD3B2092B00F2BA8000
:105E38003F4B9B78303BDBB2092B00F2B3800A2141
:105E480001FB0231C9B2002900F0AC80374BFF22B8
:105E58000C291A7740F2A68010295A7740F2A280BE
:105E680013299A7740F29E80DA7770BD3A4C2378EE
:105E780003F00203DBB213B1002038498EE0234E51
:105E88003378EBB9224B5B7813F0010F18D00CF084
:105E9800A7FAA8B932481FF039FA60B12268314B25
:105EA80002EA03033BB919F0E5FA20B9E37803F0F5
:105EB8004003DBB223B10020BDE8704009F0D6BD35
:105EC800337863B90CF08CFA48B1274B1B7803F090
:105ED8000603042B03D02B780BB90120ECE7FEF75F
:105EE80029F810B10020214958E0214B1D78002DD8
:105EF80042D0204952E000BF901B0020F13C03082B
:105F0800921900200002002094190020A01D0020F2
:105F1800611E0020EA1C002004120308050200206C
:105F2800C2110308FA1B0020E3110308F401002042
:105F3800FE2500200B170308040200202CA00308EC
:105F480030A003086E17030833A003084D17030891
:105F580036A003082C170308EC3900206226030832
:105F68002E1A00203000000F9819002094240308EE
:105F780069130020251203080B4802F0FAFC0A48AE
:105F880002F0EEFC094802F0EBFC1DF061FEE3783C
:105F980003F02003DBB22BB105492846BDE8704069
:105FA80002F038BD70BD00BFF41D0020141D002094
:105FB8001D110308054B1B78D8019B015BB2DB114F
:105FC80040B243EAE070C0B2704700BF901B0020A7
:105FD80070B50E4686B041000122054601F5E9710B
:105FE80005A80BF0AAFE0021012E8DF815104FF020
:105FF800FF0205F1010305D10092019102930920E6
:10600800FB3A04E00092019102931E2004220B4601
:106018000BF000FF05A83D49FAF7C0FA50B105A8F2
:106028003B49FAF7BBFA28B105A83A49FAF7B6FA94
:10603800002867D105A83749FAF7B0FA364B044665
:10604800F8B95A78214642F010025A70FF2302220A
:1060580000930190FE3B02903D200BF0DBFE4D20AB
:106068000CF0AAFA691C0122234612200094FCF7BE
:1060780047FB12202146224601230094FCF740FBEF
:1060880003E05A786FF304125A700024E0B25521E5
:1060980016F066FA38B12846214616F002FC10B10F
:1060A800204616F0EDFB0134082CEFD13EBB1B480F
:1060B8001B491C4AFDF76EFD19481B4912F0D2F81E
:1060C80068B10CF08DF950B9174807F0A5FC30B944
:1060D800012315481549124A0093FDF731FD144B69
:1060E8000F491D700023009305330193114B0D4A8E
:1060F8001B780A4802930D4B07F01AFC02E00E4B7E
:1061080000221A7005A806B070BD00BFBDA0030824
:1061180039A00308C9A20308F03B0020081D00208D
:10612800F11D0020E41D0020A1190020CD1C002035
:106138000B3C0020A21D0020B919002007B5410022
:10614800012201A801F5E9710BF0F7FD002301A870
:1061580004498DF80530FAF721FAD0F1010038BF6B
:1061680000200EBDBDA0030807B54100012201A80B
:1061780001F5E9710BF0E1FD002301A804498DF850
:106188000530FAF70BFAD0F1010038BF00200EBD38
:1061980086A2030870B5154B04461B1893F8805067
:1061A800B1B1134821461FF0DEF888B911482146DD
:1061B8001FF0C3F8A5F15903DBB2012B0CD94F2D01
:1061C8000AD0542D08D021460B481FF0B6F807E036
:1061D800084821461FF0BCF8074821461FF0B8F8C8
:1061E80004480649BDE870401FF06AB8302C00200A
:1061F800D91900202E1A0020CE190020AA1B002031
:10620800024B1878C0F38000704700BF981900202F
:10621800024B1A8860F308221A807047901B0020EE
:10622800034B5878C00140B2C011C0B2704700BFDC
:10623800901B0020014B1878704700BF941900206C
:1062480030B5457800230021C218917055FA03F142
:1062580011F0010F08D0064959188C7C017804EA1E
:106268000101A14208BF91700133042BEBD130BD6D
:10627800EA1C002046F6295104220BF05EBD0000FE
:1062880070B5104C0546112220460021FAF782F815
:10629800002004F8010C2A78103414F8011FC3B246
:1062A80091420BD152B10849013301F8013B112247
:1062B80046F67973BDE8704002F0F8BA0130042858
:1062C800EBD170BDEB1C0020EA1C00201FB520B1EB
:1062D800134B1A8842F480521A80124B00245A78C1
:1062E800214642F010025A70FF23022200933D20FB
:1062F800FE3B019402940BF08DFD4D200CF05CF9EF
:1063080020210122234612200094FCF7F9F91220DB
:106318002146224601230094FCF7F2F91FBD00BF75
:10632800901B0020F03B00202DE9F3412D4C072263
:10633800E37849F6346702FB0030C0B200F51E402E
:1063480055300BF0E9FC257964795FFA80F800266E
:1063580048FA06F313F0010F3AD03946042201A88F
:106368000BF0EBFC9DF804009DF805309DF8061035
:106378009DF8072000282BD0002929D0002B27D0F2
:10638800002A25D0934204D19C4221D185421FD3B3
:106398000FE09A4210D99C421AD3944218D89C42D2
:1063A80001D994421AD39C4201D1854216D2944213
:1063B8000ED18D420CD811E09C4201D185420DD2FC
:1063C800944201D18D4209D99C4207D8944205D301
:1063D80001360437082EBBD1002000E00120BDE8BB
:1063E800FC8100BF1856002010B5044649F68D60A0
:1063F80000EBD4000BF090FC04F00704C0B220417D
:1064080000F0010010BD70B5C30849F68D655D192F
:10641800044628460E460BF07FFC04F00704C0B281
:10642800012126B9A14040EA0101C9B202E0A14018
:1064380020EA01012846BDE870400BF063BC00006B
:10644800F0B57D4B8DB0DD78042200EBC505EDB2CB
:10645800E90001F50A4104A8BC310BF06EFC774B4A
:10646800774E1A78002304A9C95C312905D130393F
:10647800994041EA0202D2B205E0302903D12F390E
:10648800994022EA01020133042BECD132706C48A6
:106498006C496D4AFDF77EFB6A4B1B7813B96A4B52
:1064A8001B78F3B16748694911F0DCFE68B10BF05D
:1064B80097FF50B9654807F0AFFA30B90123634830
:1064C8006349604A0093FDF73BFB002300930233C6
:1064D8000193FD3302935A485A495B4A5C4B07F0D3
:1064E80027FA05EB0511002401F50C41347004A8C6
:1064F8007C3108220BF021FC2646E0B2542116F02C
:106508002FF8002838D004AB1B5D312B03D120466F
:1065180016F0BCF838B104AB1B5D302B2CD12046EB
:1065280016F0B4F840B34EB9FF2300933420314637
:1065380004223346019602960BF06CFC04AE305DE3
:106548002146303816F0B0F8335D0126312B4FF074
:10655800030306D10093A3191BB2019602933520B9
:1065680005E00093631C1BB20196029336200021BC
:1065780004220B460BF04EFC0134082CBDD1A901B6
:1065880001F5104104A8343120220BF0D6FB083C59
:1065980004AD274615F8013BE6B20134302B03D190
:1065A8003046FFF721FF38B115F8013C312B2CD1CB
:1065B8003046FFF719FF40B34FB9FF23009334204B
:1065C800394604223B46019702970BF023FC15F845
:1065D800011C30463039C9B2FFF715FF15F8013CE8
:1065E8000021302B4FF0FF0305D1009323B2019116
:1065F8000293372004E0009323B2019102933820DC
:1066080004220B460BF006FC0127202CC2D1114DA9
:106618006B7803F00403DBB263B1203C2046FFF73C
:10662800E3FE38B90134E4B2202CF7D16B7860F37B
:1066380082036B700DB0F0BD18560020941900202D
:10664800081D0020F11D0020E41D0020A1190020D4
:10665800CD1C0020F03B0020014B1878704700BF8C
:10666800691300202DE9F04F4E4B00221A704E4A54
:1066780085B01678002E40F091804C4B4FF4B468EA
:10668800DA78997808FB02F24FF03C0808FB0128F9
:106698005A78474F90441FFA88F8BA466CE03AF89F
:1066A80015303C24DAB2544304EB13244C44A4B20E
:1066B800042CEEB207D842F25A73984503D904F570
:1066C8001C546034A4B2444511D949F654600BF007
:1066D80023FBC8EB0403834209DC364B1A787B1989
:1066E80093F83830934302D02E4901230B702F4A78
:1066F800D378B34232D142F26073B4FBF3F203FBB6
:1067080012439BB2434523D12B4B9B7813F0090FBF
:1067180044D12A4B5B7803F08003DBB2002B3DD1D8
:10672800274B5B7803F00203DBB2002B36D1254BF5
:106738001A781BEA020F11D10199009841EA020266
:106748001A70FFF7F1FD48B90098FFF779FE05E0E8
:106758001C4B02991A7801EA02021A70013509F5F0
:10676800B469072D1FFA89F999D1039E07370136B5
:10677800042E0AF10E0A11D04FF0010B0BFA06FB9A
:106788005FFA8BF301936FEA0B03F2B2DBB24FF0BF
:106798000009009202934D46039680E705B0BDE8D4
:1067A800F08F00BF69130020011C0020185600203C
:1067B800021C002094190020EC390020FF3B002027
:1067C800D6330020001C002073B50C4601EBC00135
:1067D800C9B2C90001F50A410546042201A8BC3125
:1067E8000BF0ABFA104B002003EBC402121B52193A
:1067F80082F8380001AA125C312A0AD101218140AD
:1068080003EBC402121B521992F83860314382F824
:10681800381001300428EDD101A9312230231EF0AF
:10682800AAFDC0B27CBD00BF021C002000B501EB70
:10683800C001C9B2890189B001F510413431202263
:1068480068460BF07AFA20206946312230231EF080
:1068580092FDC0B209B000BD07B501EBC001C9B2D5
:1068680001EB011101F50C417C31082268460BF05F
:1068780064FA08206946312230231EF07CFDC0B23C
:106888000EBD00002DE9F843002634462BE02146D2
:106898002846FFF799FF214681462846FFF7C6FF9D
:1068A800214640EA09092846FFF7D6FF5FFA89F929
:1068B80049EA000010F0FF0F05D040463946022291
:1068C8000BF03BFA03E04FF0FF33A8F80030013536
:1068D800EDB20237072D08F10208D8D10134E4B22D
:1068E8000E3E042C07D0054BC6F50A47C6EB030835
:1068F8004C370025CBE7BDE8F88300BF021C002019
:1069080010B523F055FA4FF4803023F071FA23F0D4
:1069180089FB0128044628D1102023F06BF90220B6
:1069280023F05CF9002023F0A3FA002023F0B4FA46
:106938004FF4806023F0A6FA4FF4404023F0B6FAF3
:106948004FF480304FF4E01123F06EFA204623F024
:1069580077FA392023F052FB0028FAD0022023F0DE
:1069680075FA23F07DFA0828FBD17C20012123F059
:106978000FFB46F60120012123F00AFB0C480121F8
:1069880023F012FB0B48012123F00EFB0420012108
:1069980023F00AFB7E2023F031FB38B123F058FBAB
:1069A800054B04211A7861F344021A7010BD00BF28
:1069B80003400600200808188D58002010B50C4622
:1069C800014620B110220C48F9F7BAFF04E00A4842
:1069D80020211022F9F7DEFC34B1084821461022A4
:1069E800BDE81040F9F7ACBF044820211022BDE8EB
:1069F8001040F9F7CFBC00BFF401002004020020CA
:106A080010B5FF2B1446029A03D0421802F8013C35
:106A180008E06FF07F439A4204D0131443701312B6
:106A28008370C2701CF028F802E07F2023F02CFE4F
:106A38001CF00EF80028F8D1ACB10B4890F82010E3
:106A4800163001F00F011CF017F802E07F2023F048
:106A58001BFE1BF0FDFF0028F8D1044B93F86930AA
:106A680013F0010FE9D110BD900C0020A8570020A9
:106A780010B50A4B002203EB8003013B104608497E
:106A880051184C7813F8011F8C4205D10130C0B25F
:106A98000C320428F3D1FB3010BD00BF1AA702083E
:106AA800F02D002070B50D4C05460E464FF40072CF
:106AB80000212046F9F76EFC2A46314604F500709D
:106AC800F9F7C0FB642024F8035C1DF093FB002356
:106AD800A4F82D33024B64221A6070BD11590020AE
:106AE8000826002010B5054C002120464FF40072FE
:106AF800F9F750FC0023A4F82D3310BD11590020DC
:106B0800164B2DE9F0415D8907462846FBF708F842
:106B18001349FBF711F9134B134E1860D723B5FB34
:106B2800F3F5EDB2822229460446F01901F098FFE8
:106B38002846FAF7F9FF01462046FAF73FFF0B49C6
:106B4800FBF746F8FBF70AFA0337BE19C1B28122F0
:106B58003046BDE8F04101F083BF00BF2C31002072
:106B680000005743581C0020F40100200000204179
:106B780070B54B4D2868FAF7DFFB45A3D3E900232E
:106B8800FAF77AFAFAF7C6FEFAF7D6FB42A3D3E980
:106B98000023FAF725FC3EA3D3E90023FAF74AFDC0
:106BA800FAF7B8FEFAF7C8FBFAF7D2F9FAF7B2FE25
:106BB8003C4906462860FBF7B3F920B13046FBF79D
:106BC800CDF9C4B25EE030463649FBF7BDF950B1A5
:106BD80030463549FBF7A4F928B13046FBF7BEF932
:106BE800C0B2441C4EE030462F49FBF7ADF950B116
:106BF80030462E49FBF794F928B13046FBF7AEF939
:106C0800C0B2841C3EE030462849FBF79DF950B1DC
:106C180030462749FBF784F928B13046FBF79EF93F
:106C2800C0B2C41C2EE030462149FBF78DF950B1A3
:106C380030462049FBF774F928B13046FBF78EF946
:106C4800C0B2041D1EE030461A49FBF77DF950B169
:106C580030461949FBF764F928B13046FBF77EF94D
:106C6800C0B2441D0EE030461349FBF76DF948B138
:106C780030461249FBF754F920B13046FBF76EF95C
:106C8800C0B2841D0A202146BDE870400BF03AB816
:106C9800736891ED7CFF7F400000000080842E41E6
:106CA8005C1C0020000010410000F0410000484238
:106CB80000008E420000B8420000E0420000F242AC
:106CC8002DE9F04FA1B01BF06DFE09201DF02EFC40
:106CD8001DF014FA4FF461401DF064FC09201DF00A
:106CE800E1FC0022A1484FF4804122F0E8FFA048CF
:106CF800002123F0B1FB9F4904224B78DFF898E28A
:106D08006FF300034B709C4B9C4C1A705A709A702E
:106D1800DA709B4B033A1A709A4B00201F328EF898
:106D2800000020705A7105900546069006467F209F
:106D380023F0AAFC23780E2B01F2B681DFE813F0CA
:106D48000F004F009500E0007902DE03300485044F
:106D5800EA06DC07EF075808B108D00882098A4E0E
:106D68008A48317801F00F01013149014118FFF7D4
:106D780025FE337813F00F0308D1854A92F80123D2
:106D8800012A41F09181834A138024E0012B03D129
:106D98007F4B93F819330BE0022B04D17C4B93F80B
:106DA8000D33032B05E0032B06D1794B93F80D33F4
:106DB800012B41F079810EE0774901220A7077486A
:106DC8004FF4007122F07BFF754BC8221A603378AC
:106DD8006FF30303BFE333785A1C01F05FB8704BBD
:106DE8001A6822B96D484FF4007122F068FFDFF885
:106DF80098816C4898F8001001F00F0101314901A1
:106E08004118FFF7DBFD36B198F800305A1C62F3E1
:106E1800030388F800305F4B00221A8098F80010AE
:106E280001F00F02022A03D11A7842F010020AE098
:106E3800042A03D11A7842F0040204E0052A05D195
:106E48001A7842F040021A7001F02EB9062A04D1CD
:106E58004D4B6FF3030119707EE301F00F0101221E
:106E680012FA01F1198001F01FB9474E4E483178E6
:106E780001F00F01013149014118FFF79FFD96F814
:106E8800008008F00F08B8F1070F27DC18F0010F91
:106E9800464B02D00020588002E04FF0FF31598065
:106EA8004FEA6809062209F1010902FB09394FF086
:106EB800FF32A9F802204046FFF7DAFDFF2806D086
:106EC8003B4B03EB40005823437401F0EDB800231B
:106ED800A9F8023008F1010801F08AB8002110224F
:106EE8001BA8F9F757FA17A800211022F9F752FA48
:106EF80023780133237033786FF3030301F07BB8F1
:106F0800DFF884A09AF8008018F00F0840F03F815D
:106F1800284E337803F04003DBB2F3B926486FF00C
:106F28007F43817A0122009301F00F01FF23FFF7CD
:106F380067FD224B93F8692012F0400F08D093F8B0
:106F48006C3013F0040F03D0337843F040033370F0
:106F58007378142262F3C7037370737813F0F80F11
:106F680030D0174800F12001A7E300BF0018014006
:106F7800002C014046310020302C0020621C0020EB
:106F880067130020E23A0020611C00203AA702089B
:106F9800F02D0020F03B002038260020000C014096
:106FA80008260020DAA70208BAA80208AA3B00208F
:106FB800F4010020D7390020900C0020A8570020A9
:106FC800DAA90208BC4B1B7803F04003DBB2002BA4
:106FD80000F0D980DFF80483DFF8049398F80030D4
:106FE80013F00C0B30D1B54E6FF07F4396F82B1091
:106FF80006F12100009301F00F0101220523FFF79C
:10700800FFFC96F84C104FF4860A06F1420001F096
:107018000F010122FF23CDF800A0FFF7F1FC96F83D
:107028004110FF2306F1370001F00F015A46CDF851
:1070380000A0FFF7E5FC042389F8003098F8003039
:1070480043F0080301F02EB803F00803DBB2002B6D
:1070580039D099F800A0BAF1000F03D0984800F190
:10706800400138E0954E6FF07F4B717D06F10B00C3
:1070780001F00F010122FF23CDF800B0FFF7C0FC9B
:1070880096F82B1006F1210001F00F0101220723C9
:10709800CDF800B0FFF7B4FC96F836104FF486032D
:1070A800009306F12C00FF2301F00F015246FFF771
:1070B800A7FC98F800306AF3C303DBB243F004037B
:1070C80088F800305AE099F800C0BCF1000F08D0E9
:1070D8007B4800F16001FFF771FC99F8002030321D
:1070E80008E2764E6FF07F40717DFF23009001F03B
:1070F8000F0106F10B000122CDF80CC0FFF780FC50
:107108009AF80030DFF8C4B103F0100A5FFA8AFA7F
:10711800DDF80CC0BAF1000F0CD098F800206CF321
:10712800820288F800205A1C62F303038BF80030AF
:1071380000F0BABF96F82B106FF07F42009206F16C
:10714800210001F00F0101220C23FFF759FC96F8EA
:1071580036104FF4860300935246FF2306F12C00A5
:1071680001F00F01FFF74CFC9BF8003083F0100290
:10717800C2F3001262F304138BF80030042389F879
:10718800003000F091BF4E4800F1800195E2B8F15F
:10719800010F3CD14A4800F1A001FFF70FFC002E77
:1071A80000F082879AF80030444E5A1C62F30303B9
:1071B8008AF8003096F82B106FF07F4906F121000D
:1071C80042460F2301F00F01CDF80090FFF718FC9D
:1071D80096F82B1006F1210042460E2301F00F010C
:1071E800CDF80090FFF70CFC96F82B1006F1210063
:1071F800424601F00F010F23CDF80090FFF700FC85
:1072080030488021424622F05AFD00F04DBF2C48FC
:1072180000F1C001FFF7D2FB002E00F045872A4B92
:1072280096221A609AF800306FF303038AF8003048
:1072380092E1264E317811F00F0A16D1244800F158
:107248002001FFF7BBFB204B1B68002B40F02C876D
:107258001BA8F9F7EFFA4022134601461BA801F0D4
:1072680023FA3378012200F019BEBAF1010F39D19F
:1072780012486FF07F4390F82010002200931630D8
:1072880001F00F01FF23FFF7BBFB01F077FA00289D
:1072980000F00A873378022262F3030333700D4B40
:1072A8001A7842F080021A700B4B5A7842F00202A8
:1072B8005A7000F0F9BE00BFD7390020900C0020AA
:1072C800DAA902080010014008260020611C0020ED
:1072D800BAAA0208DC390020863D00202C5F002075
:1072E800B360002001F00F0101F10E0303F00F035A
:1072F800012B44D89B4849014118FFF75FFB9A4886
:107308006FF07F4390F8201000221630009301F0B0
:107318000F01FF23FFF774FB1CF038FD337803F0EF
:107328000F03022B13D118F071F8002800F0BC8667
:107338008E4B1A7842F040026FF304121A705A7892
:107348006FF345125A703378032200F0A7BD18F086
:1073580047F878B118F0E6F817F09EFF844B002044
:107368001A7858816FF3C7121A703378042262F3BF
:10737800030333707F4B1A786FF3000263E5BAF1A9
:10738800040F4DD1DFF8DC914901DFF81082494440
:107398004846FFF713FB98F80010774B01F00402FA
:1073A800D2B27AB941F004016F4883F800A088F896
:1073B800001090F836104FF4860300932C3001F03B
:1073C8000F01EEE293F800A0BAF1000F40F06C86CE
:1073D80065486FF07F45417D01220B3001F00F01B8
:1073E800FF230095FFF70CFB64480122817AFF23F5
:1073F80001F00F010095FFF703FB98F80030052214
:107408006AF3820388F800303378484662F303034E
:10741800337009F1A001FFF7D1FA554600F044BED8
:10742800DFF84481FF2398F8201000226FF07F498D
:1074380008F1160001F00F01CDF80090FFF7E0FA0F
:107448002BB2072B18D1337808F121006FF303030F
:107458003370237801220133237098F82B100E2300
:1074680001F00F01CDF80090FFF7CAFA44488021D7
:10747800002222F024FC0025424E96F86B3013F0CF
:10748800040F00F0118698F857106FF07F43002220
:1074980000933D48FF2301F00F01FFF7B1FA96F87A
:1074A8006B303A4A03F00F03012B137003D1002D00
:1074B80008BF01250CE0022B04D12BB2012B08BF19
:1074C800032505E0032B03D12BB2032B08BF0725A7
:1074D800ABB213F0010F02D02D4A3121517713F0CE
:1074E800020F02D02A4A3221917713F0040F00F0DC
:1074F800DB853322264BDA7700F0D6BD1948254EB6
:1075080000F1C001FFF75AFA96F80090DFF85C80A6
:1075180019F00F090CD117F0D9FD98F8003069F36C
:10752800000388F8003033785A1C62F30303337081
:1075380017F05EFE98F8003013F0010F00F0B485E4
:1075480000221548802122F0BAFB0A4B00225A700B
:10755800337862F30303337023780133237000F028
:10756800A3BD00BFBAAA0208900C0020863D0020E7
:10757800DC390020FE3C0020B36000200100002020
:1075880000100140A8570020DD0C0020D63900204B
:10759800F4010020611C0020001801402C5F00202D
:1075A8008648874E00F1E001FFF708FA17A8F9F7B7
:1075B80041F917A902468348F9F7C2F90021824820
:1075C800B18090F8C5106FF07F4300220093BB3064
:1075D800FF2301F00F01FFF713FA7C4A92F86B10B2
:1075E80092F86C30327843EA012312F0010FB3802D
:1075F80010D0A3F1EB0292B20A2A04D9A3F5E673DC
:107608009BB2282B02D8F3880133F38033786FF3C9
:10761800000333707378002B40F04685684AD2889F
:107628007AB16B4A1FA8117863F3030111702278AD
:107638008DF87F300132227028228DF87C2022F0CC
:107648005DFB0022F28000F02FBD624EDFF8ACA196
:10765800337803F004085FFA88F8B8F1000F15D101
:1076680011A841461522F8F795FE5B4BCAF8008031
:107678001B684546CDF847303368474643F0040356
:107688003360564BA3F8368300F00EBD03F0800339
:10769800DBB2002B67D1DAF80010002940F004852E
:1076A8004F48FFF78BF94F484FF4805122F0FDFA0D
:1076B800012806D04A4800F1A001FFF77FF900F041
:1076C800F3BC4649B1F83623002A43D0093146486D
:1076D800013AF9F735F9444B03F1100113F8012B7E
:1076E8000D2A01D00A2A02D1202203F8012C8B424C
:1076F800F4D13E4B4FF03C0808FB073808F11E0850
:107708004046F9F797F8414602463948F9F7C2F872
:10771800D8B9022F03D1336843F0100304E0032FD4
:1077280003D1336843F040033360327853005BB2CF
:1077380003EAC263DB173268DBB263F3C712326055
:107748001BB1FFF7CFF900F0AFBC0137FFB2042F30
:1077580008BF0227254B3C2606FB07363046F9F7BB
:1077680069F8314626E0DAF80080B8F1000F40F0F9
:107778009B84737803F02002D2B2002A40D11D4BBB
:1077880011A81A889B781C498DF84630ADF844201A
:10779800F8F75AFE114B5B7A302B07D1FFF7A2F9A5
:1077A800336843F40053336000F07EBC11A8F9F746
:1077B80041F811A9FFF776F900F076BCBAAA0208D9
:1077C800FE3C002008020020900C0020A857002052
:1077D800611C00200C2600203BA00308085900204B
:1077E800BAAB020800080140040200200C00002087
:1077F8001159002040A0030844A0030808260020CF
:1078080003F04003DBB2002B40F08980B14800F15F
:107818006001FFF7D3F8B048F9F70CF88046AE4995
:10782800AE484246F9F736F8002873D1AC4B4344CA
:107838005B7A302B6ED1FFF755F93368DFF8D092B9
:1078480043F48043336099F82B106FF07F43009323
:1078580009F12100082301F00F010122FFF7D0F8F8
:107868006423CAF800307F2022F00EFFDAF80030D7
:10787800002BF8D1984699F88E10D633994E89F88E
:1078880086304B3B6FF07F4A89F88730964801F085
:107898000F0142467433CDF800A0FFF7B1F896F80F
:1078A800B91106F5D670033001F00F014246FF23E7
:1078B800CDF800A0FFF7A4F896F8C41106F5DD701E
:1078C80001F00F014246FF23CDF800A0FFF798F81A
:1078D80096F8CF1106F5E270013001F00F0142462B
:1078E800FF23CDF800A0FFF78BF896F8DA1106F51C
:1078F800E87001F00F014246FF23CDF800A0FFF722
:107908007FF899F899107948CDF800A001F00F0197
:10791800424646E07648F8F78DFF75494AE796F8FB
:1079280002B0DFF8EC910BF0020B5FFA8BFBBBF1B6
:10793800000F3AD199F82010FF236FF07F4809F122
:10794800160001F00F015A46CDF80080FFF758F8ED
:10795800684B93F86B3003F00803DBB2002B00F0A0
:10796800A38399F82B10012209F1210001F00F01DE
:107978000323CDF80080FFF743F83368554843F4F4
:10798800003300F180013360FFF718F855485A4674
:1079980090F8E51100F5EC70CDF80080033001F0A7
:1079A8000F01FF23FFF72CF87EE3CAF8008099F84F
:1079B80020106FF07F4300934246FF2309F1160021
:1079C80001F00F01FFF71CF82AB241F211139A4295
:1079D8001DD1434B5B7A302B13D1FFF783F8336803
:1079E800454668F3514368F38E3368F34D3333608B
:1079F800414B1A7868F303021A7023780133237015
:107A080052E33E48F8F716FF3C49FFF74BF8394E6A
:107A180096F86B3013F0040F00F0468325B9384808
:107A280020211022F8F7B6FC7F2022F02DFE99F8CD
:107A380057106FF07F43002200933248FF2301F074
:107A48000F01FEF7DDFF96F86B202F4B02F00F02B7
:107A58000D2A1A7005D125B92C4A412191754FF488
:107A680080551A78062A08D12AB2B2F5805F04D167
:107A7800264A3621D1754FF488551A78082A08D134
:107A88002AB2B2F5885F04D1204A3821117641F232
:107A980010151B780B2B09D12AB241F210139A4208
:107AA80004D11A4B2A225A7641F211150D486FF06B
:107AB8007F4390F8F0110022009300F5F370FF2344
:107AC80001F00F01FEF79CFF96F86B3013F0010FE1
:107AD800AAD0E9E2BAAB02081A0100201159002025
:107AE8000859002001000020140D00201F0D00205F
:107AF800FC000020A8570020611C0020380100204D
:107B080004020020DD0C0020D6390020F4010020FA
:107B1800900C0020A34B1A7842B300221A700F2051
:107B2800FAF792FA06460A20FAF78EFA9E4B9F4910
:107B380058814A7812F0010F18D06436301A5882EA
:107B48009B4B1A78642A01D19B321A701B78984E85
:107B5800FF2B0BD00A21B3FBF1F1964B1931198099
:107B6800954822F079FC337801333370DFF864826A
:107B780098F8003013F00F0612D18E4B19228B485B
:107B88001A804378192143F0010343708A4822F090
:107B980063FC8A4800F12001FEF710FF04967CE29E
:107BA800012E68D1804B5A8AA2F1690189B2112944
:107BB80008D8049911F0010F04D141F00101C9B2AC
:107BC80004910592049A12F0020F0DD15B897C4A48
:107BD8001380A3F5C263023B9BB2D72B04D8049849
:107BE80040F00203DBB204931B20FEF789FF0599DE
:107BF800744B0AB2632A05DD642192FBF1F230323C
:107C08001A7401E0092A0CDD059A11B2642291FB6D
:107C1800F2F002FB10120A2012B292FBF0F230329C
:107C28005A74059802B2642092FBF0F100FB11210E
:107C38000A2209B291FBF2F002FB101230329A7458
:107C48005B4B1B78FF2B08D158495B484B786FF387
:107C580000034B70002122F0FFFB049A032A40F036
:107C680023825248002143786FF30003437052483F
:107C780022F0F2FB11E2022E03D1534BC8221A6004
:107C88000BE2032E16D1504B1B68002B40F00C82E0
:107C98004A4800F14001FEF791FE1B20FEF730FF35
:107CA800414B5B89A3F51E630F3B9BB2542B00F23B
:107CB800FB81F2E1042E0CD13B4B98890FF084FE36
:107CC800002840F0F1813D4800F16001FEF776FEA2
:107CD800E3E1052E07D1344B98890FF075FE032890
:107CE80040F0E281D9E1062E40F0D78122786FF387
:107CF800030301322270D5E1344800F12001FEF778
:107D08005DFE334B1B78002B00F0CE8123780133C6
:107D18002370304B1A786FF30302FFF794B82D4E97
:107D2800DFF8A480337813F00F021AD12A4800F143
:107D38002001FEF743FE2948F8F77CFD2749024653
:107D48002748F8F77FFA2548F8F774FD254BA3F87C
:107D5800160233785A1C62F3030333701CF0CCFC10
:107D680091E0012A16D1D8F80030002B40F09C8110
:107D78001CF0EEFC012840F097811B48F8F75AFDEB
:107D8800194902461948F8F785FD002840F08C810A
:107D980011486FE0D8F80020002A40F085810B21B7
:107DA8007BE000BF6A1300202C3100204631002000
:107DB800701C00208C0C0020002C01407AAC0208BA
:107DC800641C0020F401002008260020FAAC0208F8
:107DD800601C0020611C00203AAD020874010020DC
:107DE800C4370020AC5C002092010020AD5C00206C
:107DF800874E337813F00F080CD186484146FEF7BA
:107E0800DDFD33785A1C62F303033370824BA3F809
:107E1800028049E1B8F1010F18D18048042121F00E
:107E280044FF002800F040817A4800F12001FEF765
:107E3800C5FD33784FF0FF315A1C62F303033370EA
:107E4800774B64221A60744B59802DE1B8F1020F08
:107E5800DFF8CC811BD1D8F80030002B40F024810A
:107E68006E48042121F021FF002840F01D816A4B53
:107E78005880684800F14001FEF7A0FD33785A1C8D
:107E880062F3030333706423C8F800300CE1D8F8B8
:107E98000020002A40F008810C21217062F30303BE
:107EA800A9E0604910234FF40052CB700D3B8B7052
:107EB8000A805D4821F0AAFE0A2200215B48F8F7F3
:107EC80069FA802021F006FE237801332370504B95
:107ED8001A786FF303021A70514BC8221A60E3E054
:107EE8005348DFF848A100F12001FEF767FD9AF832
:107EF8000030002B00F0D8804E48DAF80020444EBD
:107F08000260BAF8042082809AF8062082713178DB
:107F180011F00F0159D1DFF80881D8F800100029B5
:107F280040F0C2809AF80410A2F5A6524FF0640BF4
:107F3800103A0BFB01229AF805004FF00A0909FBD9
:107F480000200393F9F7ECFD3B49F9F7F5FE0246EB
:107F58009AF80200039BA0F5A65010380BFB030B00
:107F68009AF80100354B09FB00B018600392F9F745
:107F7800D7FD039A01461046F9F722FD304B1860E9
:107F8800F9F7DAF91EA3D3E9002382468B46F9F7FD
:107F9800ADFC002800F08880504659461AA3D3E962
:107FA8000023F9F799FC00287ED0FEF7E1FD33782D
:107FB80048465A1C62F303033370C823C8F80030DC
:107FC80009F0AAFEC0B207906EE001296CD10D300D
:107FD8000799832200F044FD114BD3F80080B8F1D3
:107FE800000F61D1404621F075FD237801332370DD
:107FF800337868F30303337056E000BFAFF30080B3
:10800800736891ED7CFF7F400AD7A3703D008040E4
:10801800611C00209AAD0208AA3B0020000C014018
:10802800082600204231002000100140781C002062
:10803800FAAD02080402002000007A44741C0020F3
:108048005C1C00208448854E00F12001FEF7B6FC38
:10805800F37913F0010F27D0DFF8488298F80090E1
:1080680019F00F0920D17E4B0A2259781878103957
:1080780002FB0011B1701979D878103902FB001190
:108088007170D9799B79103902FB0312327019F09B
:108098007DFCF37969F30003F37198F800305A1CFA
:1080A80062F3030388F80030DFF8FC9199F8006068
:1080B80016F001063EF43BAE6A4B01221A701BF023
:1080C800DBFA2378092B01D00D2B28D10120664932
:1080D80012F048FD654B664A5B7803F01F03D35CDA
:1080E800644A522B137002D1634B01221A70634BFE
:1080F800634A03F1200153F8040B8B4242F8040B46
:10810800F9D1002109A812F06BFD09A80D211CF076
:108118008FFA5C4B1A78013202F003021A7099F850
:10812800006006F00206F6B2002E00F08B800FF019
:10813800F9FE14F043FA06980322431C93FBF2F26B
:1081480002EB42029B1ADBB20693002B79D1DFF8CF
:10815800488198F84960C246002E4DD0022E03D1BE
:1081680098F80130312B49D023780E2B13D146488B
:1081780046490522F8F78EFB8246002840D1B21FF7
:1081880037484349F8F7DCFB344B5646DA7942F076
:108198000102DA7135E00D2B03D13E483A49072236
:1081A80027E0032B22D13C4B002713F8012F2C2A60
:1081B80003D00137FFB2B742F7D11BA832493A467C
:1081C800F8F7BEFB7B1C07E00AEB03025278303A53
:1081D800D2B2092A03D80133DBB2B342F4D30AEB93
:1081E8000701FA4317A80231D21802E0264911A85C
:1081F800721EF8F7A5FB03E0069E02E0012600E0E8
:1082080000261E4B204A03F1100153F8040B8B4241
:1082180042F8040BF9D1214B214A03F1100153F81C
:10822800040B8B4242F8040BF9D1402388F8113033
:108238001C3B88F82230023B88F84B301BF080FF4B
:1082480000E0002699F8003003F0F5036FF300030F
:1082580089F80030FEF76BBD3AAE020818560020C8
:10826800661C00206A130020495C0020485C00203E
:1082780044E40208763A0020601C0020F401002043
:10828800B93A0020F2390020B758002047A0030867
:10829800BC580020781C0020B6580020040200209A
:1082A800C8580020611C002090580020AFF30080BF
:1082B80010B5044640181146F8F75EFA2046F8F75C
:1082C800B9FAC0B210BD42540131C8B270470000BB
:1082D80010B50D4B0D4A1B780C460E2101FB0323EC
:1082E800997A39B101390523594301F56E51443161
:1082F80089B201E043F6C4310019042209F01DFDDA
:10830800201DC0B210BD00BFCD5E00203017002078
:1083180010B5054B0C46197800190131042200F0FC
:108328009FFB201DC0B210BDCD5E002000F5364079
:1083380008B54B3009F0F0FC10F0FF0F14BF002017
:10834800012008BD10B50A4600210446FFF7B0FF1A
:1083580001462046FFF7DCFF114A01462046FFF799
:10836800A7FF232201462046FFF7ADFF014620461E
:10837800FFF7AEFF5B2201462046FFF7A4FF23224A
:1083880001462046FFF79FFF01462046FFF7A0FF62
:108398007C2201462046BDE81040FFF794BF00BF8D
:1083A8004DA0030810B55D220446FFF78CFF0D228F
:1083B80001462046FFF787FF0023235410BD38B538
:1083C8001D460C4640182C1911461A4600F048FB69
:1083D800E0B238BD2DE9F04118490446FFF7B2FF75
:1083E800174F0E263B78174D73430146EA5A20462D
:1083F8000423FFF7E4FF202201462046FFF763FF2E
:108408003B78014606FB035320469A7A0223FFF77E
:10841800D6FF202201462046FFF755FF3B7801464C
:1084280006FB035520466A7A0323FFF7C8FF014677
:108438002046BDE8F041FFF7B5BF00BF50A00308D4
:10844800CD5E0020301700202DE9F047264E0E2281
:108458003378264F534337F90380FA1824494FF4E9
:108468007A73044698FBF3F8157AFFF76BFF4E22F0
:1084780001462046FFF727FF1E4B1C2202FB05354D
:108488005FFA88F8B8F1030F01460CBF05F1120234
:1084980005F108022046FFF70BFFA146804600259C
:1084A80019E019F8013BA32B07D133780E2202FB00
:1084B8000373204629465A7A08E0242B09D13378D9
:1084C8000E2202FB03739A7A204629460223FFF7FD
:1084D80076FF0135EDB24545E3D120462946BDE892
:1084E800F047FFF75FBF00BFCD5E002030170020C8
:1084F8005AA0030864E40208074B187800F0040047
:10850800C0B240B11A686FF382021A60034B0022AE
:108518001A70034B18787047EC3900209C1C002017
:10852800841C0020054B00211970054B05481A686A
:1085380061F382021A601222F7F72CBF9C1C0020FC
:10854800EC390020841C002038B5084C08492278F2
:108558000546F7F777FE23780021E954054B1A689A
:1085680061F382021A60207838BD00BF9C1C00208D
:10857800841C0020EC390020064A07491378112B87
:10858800C85401D801331370044A136843F0040334
:10859800136070479C1C0020841C0020EC390020CC
:1085A800054B1B7813F0010F05D1044B181810F870
:1085B800010CFFF7E1BF70479D1C00207AAE02084E
:1085C8002DE9F041334C002314F8101094F82A20B8
:1085D80001F00F0161F3030284F82A2004EB400044
:1085E80084F8293084F828304378DFF8B88063F3BA
:1085F8000712638C4FF4D277E38498F800302A2668
:108608007B4306FB0133244D2448E95A84F82A2089
:1086180021F020FF98F8003094F82A207B4302F0DC
:108628000F0206FB0233EB1859881C48013989B23E
:1086380021F014FF01210A46184821F0DBFE012130
:10864800164821F0C8FE98F8003094F82A207B4399
:10865800120906FB02331248E95A21F0FBFE98F88A
:10866800002094F82A3057431B0906FB0376AD19FE
:1086780069880B48013989B221F0EEFE01210A46CA
:10868800074821F0B7FE06480121BDE8F04121F076
:10869800A2BE00BF9E1C002086AE02080008004053
:1086A80000340140CA1C002030B5164C94F82B50F9
:1086B800A38445F00105002384F82B50628484F8D4
:1086C800211084F8203019E0C55CA5F13002D2B23F
:1086D800092A08D9A5F14102D2B2052A9ABFA5F103
:1086E8003702D2B22A46084D013305EB420292F80E
:1086F800495392F84823257062700234DAB28A42EC
:10870800E2D330BD9E1C002086AE0208124B10B585
:108718009A8C0024DA8483F8294083F8284022467A
:1087280001210E4821F066FE64210C4821F092FEDA
:1087380032210A4821F092FE01212246084821F000
:1087480059FE6421064821F085FE05483221BDE81E
:10875800104021F081BE00BF9E1C00200008004090
:108768000034014010B500212C220348F7F712FE0F
:10877800BDE81040FFF7CABF9E1C002070B5214C11
:108788002378042B39D8DFE803F0030D152A3000CD
:108798001D4B012093F82B3013F0010F30D02070BF
:1087A800013870BD184B93F82000FFF709FF02232A
:1087B800237022E0144DEE8CFEB9FFF7A7FF95F861
:1087C800203095F821200133DBB29A4285F8203019
:1087D80001D8042300E003232370304670BD0A4B00
:1087E800D88C50B90123237070BD074BDD8C35B987
:1087F800FFF7B8FF2570012070BD002070BD002074
:1088080070BD00BFCB1C00209E1C0020044B002222
:108818005A701A709A7842F001029A70704700BF35
:10882800F41D0020202102480A46F7F7B3BD00BF17
:10883800F401002038B5044608460D46F7F7FAFF5C
:1088480098B10319202B094BC8BFC4F120001C198B
:10885800002308E014F8012BE02A14BFEA5C202268
:1088680004F8012C01338342F4DB38BDF401002005
:108878000D4B46F6E9421B689B6893420FD043F6BE
:10888800FC2293420BD0122B09D0B3F5E97F08D014
:1088980046F68D501B1A584240EB030070470120E2
:1088A80070470120704700BF041D0020F0B51F4627
:1088B80087B006460C46084600211546F7F76AFDBC
:1088C800244B07B19F80B3F9041005A801EB86017A
:1088D800042209F032FA002605AB9B5D013BDBB2AE
:1088E800B92B34D81D2B4FEA031208D8D31803F537
:1088F80028416846FE31112209F01FFA0BE016499B
:10890800D3185B186A4603F11007186859680833CA
:10891800BB4203C2F9D12046F7F78CFFC7B26846BD
:10892800F7F788FF3818A84203D8E0196946F7F71F
:1089380023FF6846F7F77EFF7B1C1B18AB4203D268
:10894800E0190649F7F780FD0136042EC4D107B0B7
:10895800F0BD00BFF41D0020887B030872A0030847
:1089680010B500216C220446F7F714FD0123A3700B
:1089780010BD002343700370837843F001038370B4
:10898800704700002DE9F0419378804613F0010FFD
:108998000D4614463AD06FF3000393701BF0A8FB02
:1089A8006378002B32D123780BB90A336370A3782C
:1089B800174F6FF30003A3701BF09AFB217807EBA6
:1089C80008066118073130462A46F7F7B9FF3046DE
:1089D800F7F730FFC6B2AE420DD80AD20023237093
:1089E80006EB08000A33637038182021AA1BF7F732
:1089F800D1FCAE420AD12278A3181B7A1BB10132EE
:108A08002270BDE8F08123700A236370BDE8F0810D
:108A1800F4010020054B1A780AB100221A701B785D
:108A280046F68A4202FB0311FFF704BFE71C002049
:108A3800F8B505460C460818002109F063F9013C11
:108A4800E4B26719384609F067F9C6B2202E03D890
:108A58003846002109F056F90CB1202EEFD9F8BD9F
:108A680002F00F03032B22F07F0230B5D2B20CD9EB
:108A78004FF47A7491FBF4F42025E4B2057002B146
:108A880014B13034047000220130B1F57A7F05DB6F
:108A98004FF47A7491FBF4F504FB1511022B0BD9F2
:108AA800642491FBF4F42025E4B2057002B114B1FA
:108AB8003034047000220130632904DD642491FB02
:108AC800F4F504FB1511012B0AD90A2391FBF3F3E2
:108AD8002024DBB2047002B10BB1303303700130D3
:108AE800092904DD0A2391FBF3F203FB121130314B
:108AF800017030BD13B5104B01461B689A899C7BE9
:108B080012F0100214BF0220012034B10B4C9B7CE0
:108B18002478634303FB001109B23AB10DF1060052
:108B2800022209F00AF9BDF8060002E0084609F039
:108B3800F3F800B21CBD00BF041D0020931D0020E7
:108B480010B50F4B1B689A899C7B12F0100214BF5A
:108B58000221012134B10B4C9B7C2478634303FB35
:108B6800010000B22AB108490222BDE8104009F00C
:108B7800DEB8054B1968BDE8104009F0C3B800BF5E
:108B8800041D0020931D0020AC1D00203038C0B209
:108B9800092894BFFF20002070470000024B1A7874
:108BA8006FF300021A707047E31D002070B5FFF7DD
:108BB800F5FF884B1A781E2A01D91E221A70864C96
:108BC8002678254606F0F006202E72D109F008FC1A
:108BD80000286ED1814B1B7833B92378C3F3031275
:108BE800013262F307135EE07D4B1B7803F08003CC
:108BF800DBB2002B59D07B48F7F71CFEC5B27A4C84
:108C0800BDB1204679493246F7F79AFE0A2D0BD8AE
:108C18002A4620467349F7F793FE60193146C5F195
:108C28000A02F7F7B7FB04E020466E490A22F7F775
:108C380087FE6F4B1B7813F0010F01D0472300E02C
:108C48002023E372684C042204F10C00A521F7F7F5
:108C5800A1FB684B1A7852B1FF23012A237306D966
:108C6800022A637303D0032AA37318BFE373624C09
:108C7800257815F0600502D194F8A33013B95F4840
:108C88005F4902E05D4804F1A3010622F7F758FEA8
:108C98005C4B1B78452B40F08D81002D40F08A817C
:108CA800237843F08003237070BD4F4856493246FD
:108CB80075E12C7804F0F004102C3FD109F090FBFA
:108CC80000283BD1202251494748F7F739FE46484A
:108CD8004E492246F7F734FE4D4B1B7813F0010F2F
:108CE80006D04C48F7F7A6FD4A4902464A4805E02F
:108CF8004A48F7F79FFD494902464748F7F720FEDB
:108D0800364B1B781BB946484649102247E1444870
:108D180045491022F7F714FE314B1B7803F0800306
:108D2800DBB22BB13B48F7F785FD02463F484FE0E1
:108D38003A48F7F77FFD02463C4842E02B7803F0BB
:108D4800F003302B7ED109F04BFB00287AD1264C5A
:108D5800202237492046F7F7F3FDA521052204F123
:108D68000B00F7F717FB334B1B78042B02D9FF23B3
:108D7800E37300E002D1FF23A37301E0032B02D1C8
:108D8800FF23637301E0022B02D1FF23237300E06A
:108D98000BB1FF23E372284B5B7813F0600F05D00B
:108DA8003F23E37223736373A373E373234B1B782B
:108DB80003F02003DBB233B11848F7F73BFD024656
:108DC8001F481649EBE01348F7F734FD02461C48E4
:108DD8001049E4E0EF1D0020E31D002038260020A4
:108DE8000C26002010260020F401002074410308FE
:108DF800C45E002006270020412600200E02002025
:108E08008F170308CC1C002032410308777703082A
:108E1800863D0020C178030801020020E27803089B
:108E280004020020447D03089877030811020020FB
:108E3800341803082F2C00204C310020EC39002076
:108E48000F0200202B7813F0F0030CD120225A498E
:108E58005A48F7F775FD5A4B584819888322BDE8D8
:108E68007040FFF7FDBD602B1ED109F0B9FAD8B9E3
:108E7800544920225148F7F763FD5348F7F7DAFCC5
:108E8800514902465148F7F75BFD5148F7F7D2FCC4
:108E98004F4902464F48F7F753FD4F48F7F7CAFCCA
:108EA8004D4902464D487AE02B7803F0F003102B29
:108EB80006D109F095FA18B14048494920226EE0D8
:108EC8002B7803F0F002402A02D0502A6BD10AE036
:108ED800444920223948F7F733FD0FF0A1FD044635
:108EE8000FF0BCFD09E0404920223448F7F728FD7F
:108EF8000CF074F904460CF095F9FF2806D13B48AC
:108F0800F7F798FC39490246394817E0FD2806D199
:108F18003848F7F78FFC3749024635480EE00228F3
:108F280006D13548F7F786FC33490246304805E054
:108F38003248F7F77FFC314902462D48F7F700FD24
:108F4800202107222E48F7F725FAFE2C06D12748BC
:108F5800F7F770FC25490246294820E0012C06D184
:108F68002848F7F767FC27490246254817E0022CEE
:108F780006D12548F7F75EFC2349024620480EE053
:108F8800042C06D12148F7F755FC204902461C4815
:108F980005E01F48F7F74EFC1D4902461848BDE892
:108FA8007040F7F7CDBC1B4A6FF3071313701A4BC9
:108FB80000221A6070BD00BFD1170308F401002019
:108FC800E21C0020B0170308B0100308F8010020C5
:108FD800BA10030808020020B51003080F02002089
:108FE80013180308B9770308DA7703080379030825
:108FF800FD010020247903087F780308C17803085D
:109008000D020020FB7703081C7803083D7803084D
:109018005E780308E31D0020041D0020204B70B576
:10902800F022204D1A702B7813F0010F0BD01E4C34
:10903800207810F0010006D11C49FFF7EBFC2378DB
:1090480043F0010323701A4E3378532B0ED1164C7C
:10905800237813F0010F07D000201649FFF7DAFC38
:1090680023786FF300032370FFF798FD3378232BE1
:1090780014D10D4B1B7813F0010F0FD1FFF78EFDA4
:109088002B780D4A43F006032B701378013BDBB2B3
:1090980013700A4A52F82320094B1A6070BD00BFAA
:1090A800EF1D0020E31D0020091D0020486D030866
:1090B800CC1C0020276D0308C31D0020D01D0020F4
:1090C800041D00202DE9F0415C4BF0225C4D1A7024
:1090D8002A7802F01003DBB2002B2DD1594963F333
:1090E80047120B601C462A70574A9A5C2D2A01D0F9
:1090F8000134E4B20133082BF6D1544E3A213046FC
:10910800F7F7C6F938B1801BC0B2013030182146D4
:109118000222FFF7A5FC4E4B1B78452B40F08B80B5
:1091280000242046013413F0A1FA082CF9D12B7839
:1091380043F010032B7038E0464C237813F0010FEE
:1091480017D1404E4448FFF70BFC404F3168384672
:1091580001310222FFF784FC2D23BB70307846F6DC
:1091680015733E496522FFF7A1FB237843F00103FD
:10917800237003200D21384AFFF704FC2D78304E68
:1091880015F0E00541D110203549FFF743FC304B7D
:109198001B78442B0DD12B4A136801332A4903F05D
:1091A8000703C95C2D29F8D01360BDE8F041FFF72B
:1091B800F5BC532B0DD132784E3B63F34712327016
:1091C800204A28491268062000FB02125380BDE895
:1091D800F081232B2FD11B4B1D60337803F0EF0355
:1091E80065F347133370FFF7D9FC23781E4A43F021
:1091F800060323701378013BDBB213701B4A52F845
:1092080023201B4B1A60BDE8F081104C102019492F
:10921800FFF700FC04F110002821F7F739F950B1E5
:10922800001B3178C0B20130201849098022BDE8FE
:10923800F041FFF715BCBDE8F08100BFEF1D00202D
:10924800091D0020AC1D00208D3B0020F4010020EA
:10925800CC1C0020E31D0020F41D0020FB1D002075
:10926800C46C0308AA3B0020C31D0020D01D0020A9
:10927800041D0020E56C0308454B2DE9F041F02260
:10928800444E1A703378444D43F0010333702B6811
:10929800424C9B7C022B06D1414B1B7803F04003C8
:1092A800DBB23BB10FE0012B0DD13E4B1B7813F025
:1092B800010F08D109F00CFA236800206FF3555309
:1092C8002360394944E0A378344F03F02003DBB22C
:1092D800C3B909F0FDF9F87800F02000C0B288B9E8
:1092E8002968324B897C1A7861F301021A703B684D
:1092F8002D4943F400133B60FFF78CFB2C4B802275
:1093080083F843200DF010FF804678B12B689B7CD2
:10931800012B08D1234B5B7803F01003DBB213B1A8
:109328000020244914E00020234911E00DF02CFF0F
:10933800074610B1404621490AE00DF06DFF10B113
:1093480038461F4904E01A4B93F8433013B91D49B6
:10935800FFF760FB1C4B1B78232B16D1FFF71EFC75
:10936800337843F00603337009F0B2F923686FF3DA
:10937800555323600CF092FD144A1378013BDBB27D
:109388001370134A52F823302B60BDE8F08100BFF8
:10939800EF1D0020E31D0020041D0020EC390020F3
:1093A8000C260020863D0020696D03088B3D0020B7
:1093B8008D210020AB6D03088A6D0308ED6D03084D
:1093C800CC6D03080E6E0308CC1C0020C31D0020C2
:1093D800D01D00202DE9F341704B714DF0221A7019
:1093E8002B68704C9B7C1BB9637843F0020302E046
:1093F800637843F001036C4E6370337843F00103E4
:109408003370238823F4FF739B059B0DB3F5007F0E
:1094180007D0664B1B787BB1624B5B7813F0010F6A
:109428000AD0237800206FF3861361492370FFF771
:10943800F1FAF8F745FE84E023785A4F03F0400329
:10944800DBB2FBB9BB78EBB95A4B93F8008018F044
:10945800010817D1F8F734FE3B7843F040033B701E
:109468002B68B3F91030022B3B780CBF43F0800314
:1094780068F3C71300213B70082001220B460091B6
:10948800F9F73EF9A378474A032B28D003D8012BD4
:109498000BD00DD806E0052B2DD0117825D3FF2B46
:1094A80032D12BE00020424949E00020424946E001
:1094B8004248F7F7BFF9DFF83C81C7B23F4908F1E6
:1094C80010003A46F7F73CFA0F2F3AD807F1100088
:1094D80040442021C7F11002F6F75CFF31E0384B19
:1094E800187800282DD1374929E06FF386111170BB
:1094F8000020354923E00020344920E06FF386112D
:109508001170002032491AE0053BDBB26FF3861177
:10951800022B117002D100202E4910E0012B02D13C
:1095280000202D490BE0032B02D100202B4906E037
:10953800052B02D100202A4901E02A490020FFF723
:1095480069FA237803F04003DBB20BB9F8F7B8FDEA
:10955800254B1B78232B1ED1FFF720FB337822786D
:10956800617843F00603337001F0FE01002302F036
:10957800BF0263F3C71263F34101A37022706170E5
:10958800F8F79EFD194A1378013BDBB21370184AAD
:1095980052F823302B60BDE8FC8100BFEF1D00208E
:1095A800041D0020C45E0020E31D0020E6350020D5
:1095B800696D0308CA5E0020AC690308D35E002009
:1095C800C85E0020CD690308716E0308516A03085C
:1095D800B46A0308EE6903080F6A0308306A0308CF
:1095E800726A0308936A0308CC1C0020C31D00207C
:1095F800D01D0020F40100207B4B2DE9F341F0221F
:109608007A4E1A7033787A4D43F0010333702B6821
:10961800784C9B7C022B11D1774B1B7803F04003CD
:10962800DBB293B1754B1B7803F02003DBB2BBB1FF
:10963800A37803F04003DBB23BB111E0012B0FD15B
:109648006F4B1B7813F0010F0AD1F8F739FD236827
:10965800002023F480036FF3D753236069498FE018
:10966800A778DFF8908107F04003DFB2002F34D1EC
:10967800F8F726FD2968644B897C1A78384661F327
:1096880001021A70D8F800305E4943F4800367F38A
:10969800D753C8F80030FFF7BDF92B68198A21B9EC
:1096A8000091082001220B4615E00BB2022B0CD1C9
:1096B80001223B46082039460097F9F721F8534B19
:1096C8001A7842F008021A7007E0012B05D10097BA
:1096D8000E2039463A46F9F713F80DF025FD0746EE
:1096E80078B12B689B7C012B08D1454B5B7803F044
:1096F8001003DBB213B10020454941E00020454981
:109708003EE0414B3946187800F00300F8F712FEA6
:10971800FF280FD13D4B1B7803F01803182B31D0CD
:10972800A07800F08000C0B210B138463A4927E06E
:109738003A4925E00DF028FD8046E0B1334B187812
:1097480000F008085FFA88F8B8F1000F0AD1F8F7B6
:1097580047FFC0B2022801D840460AE0062811D8BF
:10976800404604E000F01000C0B210B138462C4961
:1097780006E02C4904E00DF04FFD18B12A49404697
:10978800FFF748F9294B1B78232B29D1FFF706FA55
:10979800337843F006033370F8F792FC236823F418
:1097A80080036FF3D7532360184B1A786FF3C30203
:1097B8001A701F4A1378013BDBB213701D4A52F826
:1097C80023302B60104B1B7803F00303022B02D1CC
:1097D8000DF080FC20B102B0BDE8F0410CF05EBB9A
:1097E80002B0BDE8F08100BFEF1D0020E31D00209E
:1097F800041D0020EC3900200C2600204126002002
:10980800863D0020696D03088B3D00201C1F002049
:10981800AB6D03088A6D0308716E0308926E030826
:10982800506E03082F6E0308CC6D0308CC1C002073
:10983800C31D0020D01D002010B5FFF7AFF90A485E
:109848002523C377094B0A4A1B6824219B7C1C30BB
:1098580001FB03235B781A3903F00F035943832272
:10986800BDE81040FFF7FCB8F4010020041D0020FB
:10987800F33900202DE9F047514D524F2B78F02253
:1098880043F001032B70504BDFF878911A703B6856
:109898009C6847F67313E21A544244EB02042421ED
:1098A80061434A4A565C5318C6F300065FFA86F8C5
:1098B8009246B8F1000F23D140464549FFF7AAF870
:1098C80099F80030232B79D1FFF768F92B78414AB2
:1098D80043F006032B701378013BDBB213703E4A4A
:1098E80052F823303B603D4B1E703D4B1E703D4B84
:1098F8001E703D4BC3F800803C4B1E70BDE8F087DE
:1099080099F80020232A21D19A786FF300029A70DF
:109918000EF0B4FBFFF742F92B782E4A43F006030A
:109928002B701378013BDBB213702B4A52F82330AB
:109938002A4A3B6000231370294A1370294A13707E
:10994800294A1360294A1370BDE8F087532A13D1B6
:109958009A7812F001010FD172206043244D42F031
:1099680001022E5C61F300062E549A701E4B0122F0
:109978001A60204617F038FA242303FB04A39B78C7
:1099880013F0010F02D000201A4913E0164B1B6890
:1099980073B9382102221848FFF762F8204616F0FA
:1099A800A3FC014615480222BDE8F047FFF758B866
:1099B80013490020BDE8F047FFF72CB8BDE8F08751
:1099C800E31D0020041D0020EF1D0020F3390020B6
:1099D800FF250308C31D0020D01D0020E91C00201E
:1099E800121D0020931D0020AC1D00209E1D00208C
:1099F80024550020A2700308120200200D02002046
:109A080081700308CC1C00202DE9F0412D4E2E4F0B
:109A1800307800F5E640713008F07EF93B78C4B242
:109A280013F0010F26D0294D2B78552B0AD1EC2C99
:109A380001D0013CE4B23078214600F5E6407130AF
:109A480008F060F92B78442B0DD1A4F11403DBB294
:109A5800D72B01D90134E4B23078214600F5E6402D
:109A6800713008F04FF92B78532B03D1FFF796F894
:109A78000EF004FB164B1B7803F08003DBB253B1E6
:109A88003B7813F0010F06D0124820210422BDE8CC
:109A9800F041F6F77FBC14F0800F0F4805D12B2357
:109AA8000A2103746143113006E02D230374373B08
:109AB8005C43113004F520610322BDE8F041FEF754
:109AC800CFBF00BF931D0020E31D0020CC1C002049
:109AD800EC39002004020020F40100201FB5204BBF
:109AE80020491A781AB1087840F0010008700978FE
:109AF8001C4C11F0010F31D01B490978532901D0B2
:109B08000AB103E082B901221A700DE023290BD1B2
:109B1800002018701549FEF77DFFFFF73FF82378FE
:109B280043F00603237019E01B78012B16D120217E
:109B38000A460F48F6F72EFC0E4B68461B681022A3
:109B4800996808F0FAF8002409491DF8040001EBA7
:109B5800440101341BF022FC102CF5D11FBD00BFBD
:109B6800931D0020E31D0020CC1C0020BA730308BD
:109B7800F4010020041D0020034B1B78532B01D156
:109B8800FFF70CB8704700BFCC1C0020084BFF281B
:109B98001A68936807D1917B41B10649927C09788C
:109BA80001FB023302E0927C02FB00331846704747
:109BB800041D0020931D00204328F8B504460D46D7
:109BC800174608D1114B0A261A7891FBF6F66FF35F
:109BD800C3021A7000E00E462046FEF7D7FF90B188
:109BE8000A4B303C1A780A2602F00801C9B200294B
:109BF80018BF002506FB05466FF3C30236B21A707C
:109C0800BE42A8BF3E4630B2F8BD00BFE31D0020EB
:109C1800614B2DE9F3411A689846157C977C5F4C97
:109C28002DB15F4821780222FEF71AFF00E0257067
:109C3800FF01237807F51E47E83707EB4307594E1E
:109C48000BB90DB10FE015B901A8394601E001A81B
:109C5800B91E022208F071F89DF80430F3759DF8DA
:109C68000530337605E006F117003F210222F6F7AA
:109C780091FB5B23B375023373764B4B1B7813F060
:109C8800010F5DD0494B1B78A3F13002D2B2092AEB
:109C980031D822780AB9002D3CD1454A1178964628
:109CA8009942444A01D00021117043481178A3F128
:109CB800300490F800C004EB840404EB010802A807
:109CC80001318444C9B23D48641810F80880005D29
:109CD8000CF8048C117008B1032901D90021117006
:109CE8008EF800300DB9384600E0B81E01A90222EE
:109CF80008F01DF817E0232B04D12F4B1A7892B9DE
:109D0800013205E02A2B05D12B4B1A785AB1013ABA
:109D18001A7008E0532B06D1294A533B1370264A80
:109D28001370FFF729FF274B1B7803F08003DBB282
:109D3800002B2FD0204B1B78F6182023F37529E031
:109D480045B31A4B1878A0F13003DBB2092B10D8B1
:109D58001B4A137803B92370013303F0010313700E
:109D6800D8F800302178B3F91020FFF725FF2070CC
:109D780005E0432803D1124B1B7803B92370114B1C
:109D88001B7803F08003DBB223B1054820210222AF
:109D9800F6F700FBBDE8FC81041D0020131D002020
:109DA80002020020F4010020E31D0020CC1C00204A
:109DB800E61C0020121D0020E41C0020F4B102085B
:109DC8009E1D0020EC390020F7B5384E384D337809
:109DD800384C6FF34103337019F07CFFFFF7CCFE6A
:109DE80002238DF807302B7883B1334AD17941F0BB
:109DF8000101D171314A207802EBC3035F6B93F8FC
:109E080039203978FFF7D8FE38700DE0337813F031
:109E1800010F06D02378303BDBB2062B9CBF264AC5
:109E2800D37003238DF80730337813F0010F12D065
:109E3800234B1B7803F08003DBB263B129781F4BF7
:109E4800204803EBC10393F838309DF80720C01869
:109E58002021F6F79FFA2378232B09D11A4A2B7869
:109E68001268927C013A934202DA114A0133137064
:109E780023782A2B04D12B7813B10D4A013B137098
:109E88002378532B0FD117F081FD0B4B002129703C
:109E9800DA7961F30002DA71FFF76EFE0B4B9A79FB
:109EA80042F004029A7100232370FEBDE31D0020D6
:109EB8009E1D0020CC1C002018560020F4B102087A
:109EC800EC390020F4010020041D0020101F0020A0
:109ED8002DE9F74F864E874C3378874D232B874FD4
:109EE80025D12368986843F6F123984217D1DFF803
:109EF8003482296898F8000000F56A50713007F03C
:109F080001FF98F80000013000F0010088F8000017
:109F180000F56A50713007F0FFFE286007E000B2D4
:109F2800FEF7E8FD28603B7843F008033B70337880
:109F3800532B40F06E81236849F695629B689342E3
:109F480002D12A686E4B15E04BF23662934202D179
:109F58002A686C4B0EE04BF2B352934202D12A6846
:109F6800694B07E049F6E662934204D12A68674BD9
:109F780002B101221A7023689A6843F6DD239A42D7
:109F88000AD1634B29681A7861F300021A7008F045
:109F980027FA08B108F042FA236843F6E0229B68E2
:109FA800934206D15A4B29681A7861F3C7121A707E
:109FB80019E043F6EA22934206D1554B29685A78AC
:109FC80061F300025A700EE043F6E72293420AD189
:109FD8002968504B19B11A6842F0005202E01A6819
:109FE80061F35D721A6023689A684BF2CC639A42F7
:109FF8000AD12968484B19B11A7842F0040202E0E4
:10A008001A7861F382021A7023689A684BF25973BE
:10A018009A4202D128781AF0C5FB236843F6DA225F
:10A028009B68934202D12A683C4B05E043F6DE2246
:10A03800934203D12A683A4B1A7008E049F69E62A7
:10A04800934204D12B6813B92B4B01221A60236861
:10A058009A684BF25A739A420BD1324A2B6812789B
:10A068003149032B8B5404D1304B5A7942F01002FA
:10A078005A71236849F6DE629B68934202D12968C7
:10A088002B4A05E049F6E162934203D12968294A3F
:10A09800117016E049F6E262934203D12968264A14
:10A0A800117015E049F6E462934203D12968234A06
:10A0B80011704DE049F6E562934202D12A68204BBF
:10A0C80013E043F60852934202D12A681D4B0CE074
:10A0D8004AF6EC02934202D12A681B4B05E04BF288
:10A0E8004A62934234D12A68184B1A703BE000BF89
:10A0F800CC1C0020041D0020AC1D0020E31D002006
:10A1080038260020D4390020CB330020CA1C002078
:10A11800611E0020EC390020C45E0020A6580020F3
:10A12800483A0020931D002028170020E025002031
:10A13800583E0020563E0020893D0020FD3C00206E
:10A14800901F002066150020011C0020821C0020A2
:10A1580049F69662934206D12A68A04B01201A70EC
:10A1680001460EF0C5FD2368986843F6F12398422E
:10A178000DD1DFF87482296898F8000000F56A505C
:10A18800713007F0BFFD002388F8003002E000B20C
:10A19800FEF7D6FC23689A6843F698139A4236D19C
:10A1A8002968DFF840B2DFF848A20BEBC1031B793E
:10A1B800DFF83482C3F34113012BDFF8389221DD35
:10A1C80098F8000000F566501C3007F09BFD98F8E1
:10A1D8000030DAF8001009EB030211710BEBC10231
:10A1E8001279C2F34112032A0CD17D4A1268906891
:10A1F8000830C01807F086FD98F80030DAF800201B
:10A208004B441A7298F800302A6809F80320FFF7BF
:10A21800B3FC3B78DFF8E08113F0010F00F0EE802B
:10A22800216843F698128B68934240F081806D4A0A
:10A238002B68914602EBC3010979C1F34111012949
:10A2480006DD694A1278032A02D9FEF7A7FCE1E085
:10A258003278442A36D15FFA83F82DE008F10108F4
:10A26800604B5FFA88F803EBC8031B79C3F341130B
:10A27800012B06DD5D4B1B7823BB5B4B1B78032B47
:10A2880020D8DFF864A19AF800300F2B08D808F01E
:10A29800A7F870B109EBC8031B7913F0100F08D1A8
:10A2A8009AF800300F2B07D909EBC8031B79DB0993
:10A2B80002D0C5F8008005E009EBC8031B7913F04C
:10A2C800080FCBD03378552B40F0A4802E782CE0A3
:10A2D800013EF6B209EBC6031B79C3F34113012B08
:10A2E80009DD424B1B78002B40F094803E4B1B78D5
:10A2F800042B00F28F80DFF8F08098F800300F2BE5
:10A3080008D808F06DF870B109EBC6031B7913F093
:10A31800100F08D198F800300F2B06D909EBC603A7
:10A328001B79DB0901D02E6074E0002ED0D171E0DA
:10A338004BF25A7293420AD005DCA3F536424A3AE8
:10A34800012A0ED803E04BF2B772934209D1337851
:10A358002F2B5FD9B1F91020303293425ADC303BB1
:10A3680030E043F6F122934207D11F4B1B7823B10B
:10A378003078B5F900103B222CE008F031F818B31A
:10A38800236843F6C4219A688A4203D047F28121A0
:10A398008A4204D13078B5F900102D221AE0A2F5CE
:10A3A8006A516139052903D943F6E9218A4201D165
:10A3B800012307E043F6E0218A4202D00A318A42AB
:10A3C80003D100232B6025E023683078B5F900100D
:10A3D800B3F91020FFF7F0FB28601BE0FE3B0020DC
:10A3E800041D002014040020931D0020820D00206D
:10A3F800AC1D0020302C0020E31D00202368B3F999
:10A408000800FEF777FB286098F8003043F008034F
:10A4180088F80030FFF7B0FB236843F6D22298682B
:10A4280090420BD12B6813B99C489D4901E09B4889
:10A438009C490222F6F784FA0226AEE14BF2B77283
:10A4480090420AD12B6813B99748984913E0012B19
:10A4580095480CBF964997490DE04BF25A729042C5
:10A4680018D12B68012B02D18F48934903E0022BA6
:10A4780005D18D4891491022F6F762FA8CE1032B39
:10A4880002D189488E49F6E7042B87480CBF8D49CD
:10A498008D49F0E74BF24A6290420AD12B6813B912
:10A4A80081488A49E7E7022B7F480CBF88498949D8
:10A4B800E1E74BF24B6290420AD12B6813B97A4814
:10A4C8008549D8E7012B40F0678177488349D2E76F
:10A4D80049F6E362904203D043F6EE2290420ED151
:10A4E80028680A21B0FBF1F201FB12017C4B3031E4
:10A4F800D97730322E2199775A7703264DE143F6E2
:10A50800F12290423ED1774B1B78E3B902222968A9
:10A518007548FEF7A5FA43F6F220FEF7EBFA022299
:10A5280001465E48FEF79CFA3B7813F0010F00F0F5
:10A5380084816E4B1B7803F08003DBB2002B00F0A4
:10A548007C81694819E0FEF7D5FA0222014666487F
:10A55800FEF786FA022251482968FEF781FA3B780D
:10A5680013F0010F00F06981604B1B7803F0800342
:10A57800DBB2002B00F06181484820210222F5F768
:10A5880009FF5AE143F69812904240F0F3802B6895
:10A59800574EDFF8508156F8331010224248F6F72C
:10A5A800CFF90DF1060298F800000DF1070110F03F
:10A5B80075FC4246334620B316784E49895D032917
:10A5C8001FD0296803EBC1010979C1F341110129A1
:10A5D80017D1032E15D948490B224848F6F7B0F988
:10A5E8004748711C0222FEF73BFA9DF807104548C0
:10A5F80001310222FEF734FA9DF806104248013173
:10A6080018E02E68157803EBC601097903EBC60636
:10A618003679C1F34111012906F00706C8BF05F0D4
:10A628000305012E0ADC394934480B22F6F788F96C
:10A638003348691C0222FEF713FAADE0022E0BD153
:10A6480033490B222D48F6F77BF932462C48691C12
:10A65800FEF706FA0E36A0E0032E0BD12D490B2289
:10A668002648F6F76DF92648691C0222FEF7F8F924
:10A678000D3692E0042E51D127490B221F48F6F7D8
:10A688005FF91F48691C0222FEF7EAF91D48691D97
:10A698000222FEF7E5F90C367FE000BF1202002027
:10A6A80058B202085AB20208040200209E5F03084A
:10A6B800E05F0308BF5F0308755E0308965E030842
:10A6C800B75E0308D85E0308545E030843600308B6
:10A6D8008560030864600308C7600308E86003082E
:10A6E800F4010020931D00200F020020EC39002007
:10A6F80014040020302C00202C7A0308F9010020D3
:10A70800FA010020FE01002001020020EA79030876
:10A7180045790308C979030887790308052E10D1FC
:10A7280047490B224748F6F70BF94748691C0222AC
:10A73800FEF796F94548691D0222FEF791F90B3696
:10A748002BE0062E28D142490B223E48F6F7F8F8AE
:10A758003D48691C0222FEF783F93C48691D022224
:10A76800FEF77EF93B4805F109010222FEF778F968
:10A778000A3612E0B3F91060092E04DD632ECCBF4F
:10A788000326022600E0012633482968801B46F08C
:10A798008002FEF765F900E010263B7813F0010F00
:10A7A8000BD02E4B1B7803F08003DBB22BB12A4869
:10A7B8002021801B3246F5F7EDFD294EB37803F0D2
:10A7C8000203DBB2002B38D0FEF752F8254D0346C2
:10A7D80028B92878F11D6522FEF768F808E0B279F3
:10A7E8002978B388F01D01FB023109B207F0A5FAF8
:10A7F800236847F281229B68934213D006DC43F614
:10A80800C42293420ED043F69E5209E047F2013229
:10A81800934207D049F69E62934203D047F2C12281
:10A8280093420AD105200B210D4AFEF7ABF829788F
:10A838000D4801310222FEF713F9BDE8FE8F00BF73
:10A8480066790308F9010020FA010020FE010020C2
:10A85800A87903080202002014020020EC39002025
:10A86800F41D0020931D0020F5010020F0B5114BC8
:10A878001F78114B303F1E680DE0D6F814C01CF845
:10A8880003C00133644501D112E00023DAB28242E9
:10A89800F3D301350D70094B0622094902FB073332
:10A8A8000D785B1993F86840002CEED10C70F932E2
:10A8B8001046F0BDCC1C0020041D0020F4B1020895
:10A8C800121D00202DE9F74F974C984E23689A687F
:10A8D80043F609539A4203D133780BB901333370E5
:10A8E8002368934F9968B3F910303A78B3F10108A7
:10A8F80048BF03F106084FEAE808337808F1010871
:10A9080012F0010F03FB08188A4D00F0AD808A4B46
:10A918001A789946432A4DD128780FFA88FA0AEB13
:10A92800D00007F0F9F92268844B916846F648028E
:10A938009142186001D12A783AB12A78012102F0AF
:10A94800070211FA02F250401860287819780AEBC9
:10A95800D00007F0D7F9236847F261329B68934229
:10A9680009D1744B1A78764B03EBD203734A1268F9
:10A9780083F8A0211EE046F62952934205D131788A
:10A98800002001310EF02EFD14E046F63F1A4FF07C
:10A99800000B23689B68534504D101200BEB000191
:10A9A8000EF020FD0AF1080A46F65F139A450BF1EE
:10A9B800010BEED199F80030232B10D122682B78A7
:10A9C800927C013A93420ADA5A4A013313705D4B7A
:10A9D8009B7803F00203DBB20BB1FDF717FF99F880
:10A9E80000302A2B0CD12B7853B1524A013B1370FB
:10A9F800544B9B7803F00203DBB20BB1FDF706FF63
:10AA080099F80030552B14D12368997C0F2910D957
:10AA18002A7808398A42474B01DA083200E00022D6
:10AA28001A70484B9B7803F00203DBB20BB1FDF7B9
:10AA3800EDFE99F80030442B42D123689A7C0F2A06
:10AA48003ED929783B4B072902D90839197001E00A
:10AA5800083A1A703B4B9B7803F00203DBB2002BD9
:10AA68002ED0FDF7D3FE2BE049F6556399420ED15F
:10AA7800314B1B78A3F13101C9B2032907D842F041
:10AA880006023A7007225343284A573B137023683B
:10AA98009A6843F609539A4212D133781B2B08D986
:10AAA800284B46F615629A809A7842F002029A700C
:10AAB80006E05901C918244B0020C918FDF7AAFF60
:10AAC800FFF75AF8214A2B7811789346994288BFA4
:10AAD800137012780F32934202DD1C4A0F3B137039
:10AAE80023684FF0000A93F81290B9F10F0F9ABF3C
:10AAF800C9F120095FFA89F94FF010099BF80000A5
:10AB08004FFA8AF318180FFA88F202EBE000019363
:10AB180007F002F99BF80020019B5FFA80FC9B1864
:10AB280003F007032BE000BF041D0020931D002045
:10AB3800E31D00209E1D0020CC1C0020AC1D002021
:10AB4800302C0020F41D0020F8620308951D002019
:10AB58004CFA03F06549013300F0010000280CBFEE
:10AB6800A520DB20DBB201F809000AF1010A09F18E
:10AB78000109082B5FFA8AFA5FFA89F903D0B9F15B
:10AB8800200FE5D109E0B9F1200F06D023684FFA6C
:10AB98008AF19B7C89189942B0DB3B7813F0010F4E
:10ABA80015D0236852499B7C09780F2B01F080014E
:10ABB80098BFC3F11003C9B294BFDBB2002331B10F
:10ABC800297810318A1A4949CB185F219954494F7D
:10ABD800BB7803F00203DBB2002B61D0FDF748FE1F
:10ABE8000346F8B9226846F6295192688A4206D087
:10ABF80024318A4203D043F6E5118A4204D13078E1
:10AC08003D496522002308E043F609518A4207D1ED
:10AC180030781C38C0B2F91D6522FDF747FE18E0F0
:10AC28002878F8E7236846F6E9429B68934203D000
:10AC380043F6FC22934202D1BA79317801E0BA791D
:10AC48002978BB882C4801FB0231BA7909B207F090
:10AC580074F823689A7C102A1DD89B6846F6E94246
:10AC680093420ED006DC43F6E512934209D043F630
:10AC7800FC2204E046F62952934202D02432934241
:10AC880002D11020072108E043F60952934202D16D
:10AC98000020102101E005200B21164AFDF772FE65
:10ACA800226846F68D5193688B421BD046F6474181
:10ACB8008B4217D043F6ED218B4202D10B4BDB219F
:10ACC8009977937C0B2B0DD9BB7803F00203DBB289
:10ACD80043B1297809480131022203B0BDE8F04F99
:10ACE800FDF7BEBE03B0BDE8F08F00BFF401002041
:10ACF800EC390020F41D0020FB1D0020F501002088
:10AD0800114B002270B50D461A7118B11B7803B9A2
:10AD180020234370BDB10D48F5F78CFD0446681C2F
:10AD28005CB10A492246F5F78DFA022C0BDC601C4F
:10AD380028182021C4F1030201E020210322BDE8E4
:10AD48007040F5F727BB70BD801D0020811D0020D5
:10AD580038B50546002408E0601906F0DDFF3038F4
:10AD6800C0B2092808D80134E4B2044B1B78303B40
:10AD78009C42F1DB012038BD002038BDE81C0020D2
:10AD880008B506F0C9FF0023C0B2064AD25C824269
:10AD980001D1202804D10133082BF6D1002008BDA9
:10ADA800012008BD98B2020870B506460D46002479
:10ADB8000DB12D232B55A0190021013406F0A2FF57
:10ADC800062CF5D170BD00002DE9F04F974C984F37
:10ADD800206839788368068A9AB201FB06260D46F0
:10ADE80048F6BC218B4287B0B6B20BD1914B1A788A
:10ADF8005B7802F00702C3F3420303EBC20306EBDE
:10AE0800C3062BE048F67C418B4212D1894B8A4815
:10AE18001A78597802F0070288235A43C1F342018D
:10AE2800773B03FB012320210822F618F5F7B2FA35
:10AE380014E049F234018B420BD17E4B1A785B78CF
:10AE480002F00702C3F3420303EBC2039B01F618A7
:10AE580004E0B3F5E97F08BF02EB4506774B784D70
:10AE68001A78984612F0010F53D123689A6847F26E
:10AE780089139A4204D046F689739A4240F0448175
:10AE8800704B1B782A2B3BD16F4B93F8009009F13C
:10AE9800010909F0010983F80090B9F1000F1AD0EF
:10AEA80046F689739A4208D1684B46F615629A802D
:10AEB8009A7842F002029A7026E120211022644812
:10AEC800F5F768FA3B7800205901C918614BC91891
:10AED800FDF7A0FD18E15D48FDF742FD23684846EF
:10AEE8009A6846F689739A420CBF5B495B49FDF73D
:10AEF80091FD39785A4801310222FDF7B1FD03E18D
:10AF0800552B02D0442B40F0FF804F4B00221A7083
:10AF1800FAE023685869F5F78DFC4A4B834693F8A5
:10AF280000A09946BAF1450F02D14E4B00221A7083
:10AF38005046FDF72BFE00284DD04B4B5FFA8BFB9C
:10AF48001A7852450ED15846FFF790FCFF2804D1D5
:10AF58005846FFF78BFCFF283DD0444B1A78013246
:10AF68001A7015E0DFF804A100228AF8002058467C
:10AF78000593FFF77BFCFF28059B04D09AF8002077
:10AF880001328AF8002099F80020FF281A7022D090
:10AF98002168374A4B6910601B5C886847F2891141
:10AFA8008842136092460FD1562B01D0542B0BD1F7
:10AFB8003B78123BDBB2022B06D82B7830B2C01894
:10AFC80006F0AAFECAF800002B7830B2C018DAF8EA
:10AFD800001006F097FE99F80030552B17D123681A
:10AFE800997C0F2913D92A7808398A42144B01DA37
:10AFF800083200E000221A70144B9B7803F0020319
:10B00800DBB20BB1FDF702FC184B00221A7099F85D
:10B018000030442B3BD123689A7C0F2A37D92978F2
:10B02800074B072926D90839197025E0041D002087
:10B03800931D0020991D002004020020E31D00201C
:10B048009E1D0020CC1C0020EE1D0020F41D0020B9
:10B05800F40100201B5B03082C5903086E590308F0
:10B06800F5010020E41C0020E61C0020121D002031
:10B07800AC1D0020083A1A70964B9B7803F0020327
:10B08800DBB20BB1FDF7C2FB934B00221A7099F8A3
:10B098000030432B0CD1236830B25B6919788F4B91
:10B0A80019602B78C01806F02DFE8B4B00221A7001
:10B0B80099F80030232B13D122682B78927C013A1F
:10B0C80093420DDA864A01331370834B00221A70BB
:10B0D800804B9B7803F00203DBB20BB1FDF796FBC4
:10B0E80099F800302A2B0FD12B786BB17C4A013BA1
:10B0F8001370794B00221A70764B9B7803F0020389
:10B10800DBB20BB1FDF782FBFEF736FD754A2B78F3
:10B1180011789246994288BF137012780F32934281
:10B1280002DD704A0F3B137023684FF0000B93F851
:10B138001290B9F10F0F9ABFC9F120095FFA89F986
:10B148004FF010099AF8000033B2181858440593C4
:10B1580006F0E2FD644A02F8090009F101095FFA04
:10B1680089F9B9F11F0F059B05D821680BF1010B6F
:10B17800897C8B45E6DB98F8001011F0010F16D09A
:10B1880021685A48897C00780F2900F0800098BF10
:10B19800C1F11001C0B294BFC9B2002138B12878FA
:10B1A8009AF8006010305218801B5F2111542268F1
:10B1B80090684AF6EA0290420AD14D4B1B78532B0D
:10B1C8002FD106F0A9FD4B4B187006F09FFE28E022
:10B1D800B0F5E97F25D1464A1278532A21D118467D
:10B1E800FFF7CEFD0646E0B93B78DA00D31A03F143
:10B1F8001200FFF7ADFD60B1FF2300933E4B0196AF
:10B208001B7879200133029331460422334606F035
:10B2180001FE3B780021DA00D31A03F11200FFF790
:10B22800C3FD2C4EB37803F00203DBB2002B6ED0C3
:10B23800FDF71EFB034680B9226849F23401926883
:10B248008A420AD046F689718A4214BF287838782B
:10B25800F11D6522FDF72AFB0FE02368B2799B6890
:10B268002648B3F5E97F0CBF39782978B38801FB04
:10B278000231B27909B206F060FD23689A7C032A8C
:10B2880008D99A6848F6BC218A4203D046F68971E3
:10B298008A4214D19B6848F6BC2293420CD198F894
:10B2A800003013F0010F01D010202CE020210722DC
:10B2B8001348F5F76FF82AE0B3F5E97F02D10520C6
:10B2C8000B2121E046F6897293421BD10020102100
:10B2D8001AE000BFF41D0020121D0020AC1D002044
:10B2E8009E1D0020951D0020F4010020EC3900204F
:10B2F800CC1C0020E81C0020931D0020FB1D002012
:10B308000402002000200721104AFDF73BFB2368B8
:10B318009A7C032A16D9B27802F00202D2B28AB114
:10B328009B6848F6BC2293420CD046F68972934239
:10B3380008D0297806480131022207B0BDE8F04F4D
:10B34800FDF78EBB07B0BDE8F08F00BFF41D0020ED
:10B35800F50100202DE9F04F794E8BB033689D68D8
:10B3680093F81290122D01D00B2D09D1754A122D88
:10B3780092F80090A9F130095FFA89F915D01DE01B
:10B388004BF267739D4203D028339D4240F05383AC
:10B398006D482821F5F77CF88046002800F04E8398
:10B3A80001302821F5F774F848E39F7B37B9674BDC
:10B3B800B846D879FEF7EAFB044615E00027B846F8
:10B3C800FF20FEF7E3FB4BF258539D4204460BD196
:10B3D8004BF2376006F0A0FCC0B2099020B15B4B7D
:10B3E8009B790BB1FDF7DAFB3368594D9A68122A3D
:10B3F8001AD19B7BC3B12B7813F0010F08D12046DB
:10B40800FFF7A6FC534B10B101221A7000E0187028
:10B418004E4B9B7943B12046FFF79AFC20B14D4B28
:10B428001B780BB1FDF7BAFB2978DFF844A111F0BE
:10B43800010100F087819AF80030DFF838B118462A
:10B448000793FDF7A3FB079B002800F0B58042494E
:10B45800002008704148424A90F800C013609C459B
:10B46800404940F0898033689B8903F00F03032B20
:10B478001ED13D4BACF1300C18784FF00A0E0590F8
:10B488003A480EFB0C00DDF814E000EB0E0C0EF150
:10B49800010E5FFA8EFE70449CF8ADC090F8AD00C6
:10B4A800C2F800C083F800E0002872D1187070E07C
:10B4B800082B2CD12C4BACF130001B7800EB800C06
:10B4C8000CEB030E294BDFF8A0C013F80E300893DD
:10B4D8000BB98CF800309CF800E000EB8000059078
:10B4E80070440EF1010E5FFA8EFE8CF800E01F4BDF
:10B4F800DDF814C01B5C08900CEB0E00DFF86CE064
:10B5080013601EF80030002B43D1174811E0072BB9
:10B5180011D1BCF1300F10D11348037823B14FF08B
:10B528002B0EC2F800E001E0C2F800C0013303F0BE
:10B53800010303702DE0062B2BD10B78013327E094
:10B54800041D0020E81C002004020020A21D002089
:10B55800E31D00206B130020AB580020E61C0020E0
:10B56800AC1D00209E1D0020121D0020F4B1020811
:10B57800CC1C0020E91C0020DFF898E203709BF83F
:10B5880000304FF0010C8EF800C013B10B78634403
:10B598000B7040238BF800300B784B4503D39B4B43
:10B5A80009F1FF30187008781168201806F0AAFB16
:10B5B8002B7843F004032B709AF80030232B2FD1FB
:10B5C800924B09F1FF311A788A4229DA72B9326846
:10B5D8004BF2677192688A4208D028318A4205D0B6
:10B5E8002046079306F098FB079BC8B118780130EE
:10B5F800C0B21870201806F08FFB28B9834B2021A1
:10B608001878201806F07EFB814B40221A702B78A0
:10B61800804A43F004032B7000238BF8003013702A
:10B628009AF800302A2B10D1784B1A786AB1013A6F
:10B638001A70774B40221A702B78764A43F004032D
:10B648002B7000238BF8003013709AF80030432BCE
:10B658001FD16E4B1878484505D220182021079332
:10B6680006F050FB079B9BF800203AB91B7809F1BC
:10B67800FF32934202DA654A013313702B78644A29
:10B6880043F004032B7000231370624A8BF80030D8
:10B6980013709BF8003013B15F4A013B13709BF89D
:10B6A8000030012B0ED1594B1A784A4501D201328C
:10B6B8001A70584A002313702A7842F004022A703C
:10B6C8008BF800302B7803F00402D2B2002A71D034
:10B6D800524A6FF382031370002111225048F4F785
:10B6E80059FE504A494B11781B78994288BF13700C
:10B6F80011780F318B4202DD4A490F3B0B701178EC
:10B7080047481022611806F018FB4548F5F792F8EB
:10B7180033684BF267719B68C2B28B4202D0283102
:10B728008B4205D122B94048F5F784F8421CD2B2C1
:10B738000F2A3FD83A4820218018C2F11002F4F7A6
:10B7480029FE37E0DFF8D8B011225846F4F722FE78
:10B7580033684BF267729B68934202D02832934257
:10B7680009D1214604222E4806F0E7FA4046394618
:10B77800FFF7C6FA1EE021461022584606F0DDFA09
:10B788005846F5F757F802462021C2F110025844EE
:10B79800F4F700FE21464A46244806F0CEFA244A29
:10B7A8001020937882F8069043F0020393700146C4
:10B7B800FDF7E8F89AF80030532B75D133689A688A
:10B7C8004BF258539A4208D1204606F0A5FA20B108
:10B7D8004BF23760012106F095FA3368DFF838A09C
:10B7E8009B68122B40D12046FFF7B2FA8346002807
:10B7F80030D0104BFF2219780F4BF9B90092019104
:10B808001B78782001330293FB3A1FE09E1D00202D
:10B81800AB580020121D0020E91C0020E31D002069
:10B82800801D0020951D0020811D00201B1D00206B
:10B83800141D00206B130020931D0020002100928E
:10B8480001911B787A200133029304220B4606F0FB
:10B85800E1FA09E08AF800007D492046FFF7A4FADA
:10B868007C4B83F800B0EFE020464946FDF7E0F84E
:10B87800794B0020187033688AF800009B684AF6F4
:10B88800FE02934202D10090013005E04BF27A5259
:10B89800934206D1012300930146024603460DF068
:10B8A800CDFD6E48FDF75CF8FEF766F92B7813F0CE
:10B8B800010F17D033684BF267729B68934202D02E
:10B8C8002832934204D140463946FFF719FA09E075
:10B8D8005F4B634A03F1100153F8040B8B4242F8A3
:10B8E800040BF9D133689A68122A1ED19B7BE3B105
:10B8F8002046FFF72DFAC0B12B7813F0010F14D1B1
:10B90800584B9A7922B9DA79574B1B789A420CD05E
:10B91800564B1A780023303A05E055492A20C918B1
:10B9280001330874DBB29342F7DB326893680B2B60
:10B9380001D0122B0AD14A4B991D13F8010B20286C
:10B9480002D10D3003F8010C8B42F6D192684BF20C
:10B9580058539A4214D1434B9B798BB1099878B1CB
:10B968004FF0000909EB040006F0D6F918B1404B76
:10B978002A224B441A7409F10109B9F1100FF1D1C7
:10B988002B7813F0010F25D03A4B1B7803F0800376
:10B99800DBB2FBB133689A684BF267739A422D4B5E
:10B9A80003D04BF28F718A420CD11B7833B9B8F1AE
:10B9B800000F0FD05F3388F801300BE057B15F22DA
:10B9C800FA5407E0244A1B78127810339B1A284A45
:10B9D8005F21D154284CA37803F00203DBB2002B7B
:10B9E80032D0FCF745FF2049034628B9087865227C
:10B9F800E11DFCF75BFF12E03068B4F90430A2796E
:10BA080084680978122C01FB023105D1807B18B9B2
:10BA18001449C97902FB0131184806F08EF93368D8
:10BA28009B68122B10D10820134A01460BB0BDE8C1
:10BA3800F04FFCF7A7BF0027B84600E0074609F11A
:10BA4800FF395FFA89F9BBE40BB0BDE8F08F00BF9E
:10BA5800801D00209E1D0020951D0020141D002023
:10BA680004020020A21D0020931D0020E81C0020D5
:10BA7800F4010020EC390020F41D0020FB1D0020FB
:10BA880024282DE9F041144626D16B4B43F63C326D
:10BA98001B686A4D9B686A4E934206D12B7813F057
:10BAA800010F0ED02438674909E04BF28F72934298
:10BAB8000AD12B7813F0010F03D063490020FCF75B
:10BAC800A9FF2978490800E02978301901310222B4
:10BAD800FCF7C6FF0234AAE0E72809D1574B5848BB
:10BAE8001978801801310322FCF7BAFF03349EE06D
:10BAF800A3282AD1514D2B783F2B15D810465349EE
:10BB0800FCF788FF5148F4F795FE2A2124184C4881
:10BB1800E4B2F4F7BDFC002800F08A8029780222FC
:10BB28000131FCF79DFF83E05901494DC918691897
:10BB380001F582411046DF31FCF76CFF05F59240B4
:10BB4800FE30F4F777FE241871E0F22821D13B4F3C
:10BB58003B4D3978072605EB0208B1FBF6F1404664
:10BB680001310222FCF77CFF39782D23B1FBF6F670
:10BB780088F80230F3009E1B8B1B364FDBB207EBB5
:10BB880083031988E21CA9529B78A818837006348D
:10BB98004DE025280BD1304B46F615629A80452298
:10BBA8009A719A78053842F002029A703CE05E2851
:10BBB8000BD1294B46F615729A8045229A719A78CC
:10BBC8003E3842F002029A702EE07C280BD1224BBC
:10BBD80046F248129A8011229A719A785C3842F09B
:10BBE80002029A7020E0EC280BD11B4B46F65972E2
:10BBF8009A8045229A719A78CC3842F002029A705B
:10BC080012E0A7280BD1144B46F679729A80452288
:10BC18009A719A78873842F002029A7004E0E02814
:10BC280001D1541C03E018B1054B18550134E4B296
:10BC38002046BDE8F08100BF041D0020931D0020B0
:10BC4800F4010020805303083E530308FA5A0308FE
:10BC5800FC100308753D0308F41D002038B50A4B95
:10BC680046F68A451B78002405FB030507E0074BC9
:10BC780022461978FFF704FF041B2D19044628787B
:10BC880008B11F2CF3D938BDE71C0020931D0020F4
:10BC980070B5002543F62064204606F03DF80646B8
:10BCA80004F1080006F038F816F0FF0F06D020F06F
:10BCB8007F0010F0FF0F01D00135ADB246F23F13FF
:10BCC8009C4201D00934E7E7284670BD70B5B0F949
:10BCD80000500E4605EBC50505F57855283528466C
:10BCE80006F01AF8C3B213F0800F064C08D03EB91C
:10BCF80022882846013A03F07F01228006F002F8E4
:10BD0800208870BDE21C0020454B2DE9F74F1B88A9
:10BD1800444A044689461788DFF80C8123B14FF05E
:10BD2800000A0AE09A4608E00529FBD198F8003095
:10BD380043F0040388F8003070E098F8003013F0FE
:10BD4800030F0BD013F0010F02D0B4F1FF3F05D160
:10BD580003F00203DBB21BB1012C01D03F19BFB2C3
:10BD68003BB2B3F1FF3F04D0B3F57A7F08BF002799
:10BD780001E040F2E7370FFA87FB0BEBCB0303F543
:10BD8800785303F12000019305F0C6FF10F0FF0F70
:10BD9800019B16D0B9F1050F09D103F1280005F070
:10BDA800BBFF20F07F0010F0FF0FC6D022E0B9F1F2
:10BDB800000F1FD003F1280005F0AEFF00F07F064A
:10BDC80018E00AF1010AB4F1FF3F1FFA8AFA04D118
:10BDD80098F8003043F0010305E0012C05D198F8EC
:10BDE800003043F0020388F80030BAF57A7F0DD0AE
:10BDF8003D46A2E74E4505D0B9F1000F02D0B9F192
:10BE0800050F9AD1BAF1000F05D000E03D46054A6A
:10BE18002DB2156002E0034BC3F800B0BDE8FE8FF9
:10BE2800E21C0020AC1D0020B01D00202DE9F041CF
:10BE3800037890465A1ED2B2792A9AB00F4600F279
:10BE4800CA805E01654AF3189B18654A46F68A4619
:10BE58001278457806FB0236E7213046F4F718FBDE
:10BE68000446F0B930467C21F4F712FB0446C0B909
:10BE780030462521F4F70CFB044690B930462421BE
:10BE8800F4F706FB044660B930464021F4F700FB9E
:10BE9800044630B93046F921F4F7FAFA0446002886
:10BEA80078D0A41B0FB14F4800E0404631462246E7
:10BEB800A619F4F745FD3046E721F4F7E9FA30B161
:10BEC80028466946652246F65973FCF7EFFC30466A
:10BED8007C21F4F7DDFA50B1691EC9B201EB0111FA
:10BEE80001F5C24168464831112205F026FF304667
:10BEF8002521F4F7CDFA38B1681EC0B2694665222B
:10BF080046F61563FCF7D2FC3046F921F4F7C0FA7F
:10BF180038B1681EC0B26946652246F61573FCF74B
:10BF2800C5FC30464021F4F7B3FA50B1691EC9B2D6
:10BF380001EB011101F5EA416846BB31112205F018
:10BF4800FCFE30462421F4F7A3FA58B117B125486E
:10BF5800201801E008EB040029460222FCF780FDC6
:10BF680002340CE017B11F48201801E008EB040068
:10BF78006946F4F701FC6846F4F75CFC0419002FE5
:10BF880029D0194A9378141943F0020393700023B7
:10BF9800E37116E03046F4F74DFC05461FB94046FC
:10BFA80031462A4615E0102810DD2A460D4831464C
:10BFB800F4F7C6FC0C4A9378551943F002039370C2
:10BFC800EC7110200146FCF7DDFC04E0074831461F
:10BFD8001022F4F7B5FC1AB0BDE8F081DF4203087F
:10BFE800E71C0020FB1D0020F41D00200402002097
:10BFF8000C4B1A7812F0010302D000200A4905E020
:10C0080002F00200C0B218B108491846FCF702BD98
:10C0180002F00402D2B20AB10549F7E70548012146
:10C02800FFF704BFB01D0020B818030897180308CD
:10C03800D9180308E51D002070B5124D124C0020D8
:10C048001249FCF7F7FB2846A1780222FCF708FD05
:10C05800E81CE1780222FCF703FD05F108002179CC
:10C068000222FCF7FDFC05F10B0061790222FCF7C6
:10C07800F7FCA17905F10E000222BDE87040FCF73B
:10C08800EFBC00BFF4010020E51D002005B3020845
:10C098002DE9F341544F554C3B689D7C237813F0B0
:10C0A800010F33D1022243F61E610DF1060005F09F
:10C0B80044FE4F4EBDF806304FF0FF30336029463E
:10C0C800FFF722FE237843F001032370494B1B78C6
:10C0D80013F0030F18D1B6F90010474801EBC1015E
:10C0E80001F578512031092205F027FE434B1B88C2
:10C0F8003BB1434B30461978C1F34001FFF7E6FDE9
:10C1080010B90020FAF784F8FFF796FF3D4E337810
:10C11800552B0DD1DFF8DC803B48FCF721FC98F863
:10C1280000304FF0FF306FF3410388F800300DE026
:10C13800442B2FD1DFF8BC803348FCF711FC98F86A
:10C14800003001206FF3000388F800302946FFF71C
:10C15800DBFD98F8003013F0030F19D1244D264861
:10C16800B5F90010092201EBC10101F57851203120
:10C1780005F0E3FD214B1B883BB1214B284619787C
:10C18800C1F34001FFF7A2FD10B90020FAF740F80B
:10C19800FFF752FFFFF72CFF3378232B22D1154BE3
:10C1A800194E1A7802F0FC026FF382021A70FCF73B
:10C1B800F5FCB3786FF34103B370144B1D7835B9B0
:10C1C800FCF724FB3046FCF7CBFB3D600AE0227805
:10C1D800013DEDB242F0060222701D700C4B53F87F
:10C1E80025303B60BDE8FC81041D0020E31D0020D4
:10C1F800AC1D0020B01D0020E51D0020E21C002021
:10C20800EF630020CC1C0020F41D0020C31D00207B
:10C21800D01D00202DE9F0411646104A0F465378EC
:10C228000E21C3F342034B43117803F50A434C3301
:10C238000B4D01F00701044603EB4101022205F012
:10C248007CFDE81921780222FCF70AFC6178A8191C
:10C258000222BDE8F041FCF703BC00BF991D002095
:10C26800F4010020044B02225978044BC1F3420127
:10C2780018180131FCF7F4BB991D0020F4010020C7
:10C2880010B5074B074C1B78074A03F0070304EB6C
:10C2980083031C88111814529B788B7010BD00BF43
:10C2A800991D0020753D0308F4010020084B1B78F8
:10C2B8009B0902D0012B06D102E01020054904E0B9
:10C2C8001020054901E005491020FCF7A3BB00BF79
:10C2D800991D00205A2503087B2503089C2503087F
:10C2E8002DE9F041DFF868800F4698F80010174DE7
:10C2F800C1F382010446164605F108000131022205
:10C30800FCF7AEFB98F80010042201F01C0101F5BF
:10C318001E413431204605F010FDE819217802222B
:10C32800FCF79EFBF81C281861780222FCF798FBA2
:10C33800A819A1780222FCF793FBF01CE1782818D1
:10C348000222BDE8F041FCF78BBB00BFF4010020DE
:10C35800E51C0020064B1B7803F08003DBB233B1E9
:10C36800435C04482021C0180222F4F713B8704730
:10C37800EC390020F40100202DE9F743654D664CA7
:10C388002B6821789B68022203EB41010DF106001E
:10C3980005F0D3FC2B68A9469A6843F6F4239A4221
:10C3A80008D100205D49FCF735FBBDF806804FF445
:10C3B800B46303E0BDF806804FF46163B8FBF3F1A2
:10C3C80003FB11883C221FFA88F8B8FBF2F302FB42
:10C3D8001388CFB2DEB2022251483946FCF740FB3F
:10C3E8005FFA88F802224F483146FCF739FB0222EF
:10C3F8004D484146FCF734FB4C4B1B7813F0010FBA
:10C408006ED04B4B4B4D1878232804D12B78012B39
:10C4180062D8013305E02A2805D12B78002B5BD0A0
:10C42800013B2B7058E0A0F13003DBB2092B01D996
:10C4380043284BD12B7873B9D9F8003039B29A68B0
:10C4480043F6F4239A4201D10A2200E01122FDF7B3
:10C45800B3FBC7B216E0012B0ED1D9F8003031B2C8
:10C468009A6843F6F4239A4201D1172200E03B224E
:10C47800FDF7A2FBC6B205E041463B22FDF79CFB57
:10C488005FFA80F8D9F800309A6843F6F4239A42A4
:10C4980009D13C235E434FF4B46303FB0767B844F8
:10C4A800ADF8068006E038463146424610F035FAC7
:10C4B800ADF80600D9F8003020789B680DF1060128
:10C4C80003EB4000022205F032FC05E0532803D1BB
:10C4D80000232B70FDF750FB17482978FFF73AFF28
:10C4E800D9F800309A6843F6F4239A4210D020789D
:10C4F800124965220023FCF7D9F905200B21104ABF
:10C50800FCF740FA21780F4801310222FCF7A8FA1B
:10C51800BDE8FE83041D0020931D00207F570308FB
:10C52800040200200A02002012020020E31D00205D
:10C53800CC1C00209E1D002016B30208FB1D002005
:10C54800F41D0020F501002073B59A4B9A4D1A7816
:10C5580012F0010F05D12A7812F0380204BF2A70B0
:10C568006A701A78934E42F001021A702B78924C36
:10C5780013F038023ED191490978552904D113F0B6
:10C58800070F2FD0DA1D0AE044290CD103F0070267
:10C5980001323D3992FBF1F1C800411A521A62F397
:10C5A800020323701EE053290AD1C3F3C2010131EB
:10C5B80061F3C5032370637862F34303637011E08A
:10C5C80023290FD1FCF7EAFA33787D4A43F00603B2
:10C5D80033701378013BDBB213707A4A52F8232088
:10C5E800794B1A6000207949FCF714FA1C20FFF7F0
:10C5F80047FEDDE0082A2ED175490020FCF70AFA2B
:10C608000620FFF72FFE0C20FFF73AFE152118220F
:10C6180001A8FFF7FFFD694B1B78552B06D16378FE
:10C6280003F0FE03C3F34202013A07E0442B0BD1A7
:10C63800637803F0FE03C3F34202013202F00302FF
:10C6480062F343036370B3E0532B28D0232B40F0ED
:10C65800AF802378A6E0102A51D15D490020FCF76D
:10C66800D9F90620FFF7FEFD0C20FFF709FE15217A
:10C67800182201A8FFF7CEFD6178564801F00101A4
:10C68800FFF768FE4D4B1878232801D02A2804D1DB
:10C698006378DA4362F30003D4E7532804D123789C
:10C6A800C3F3C202013280E0A0F13003DBB2092BF0
:10C6B80001D943287CD16B7802AA03F001033B21FE
:10C6C800D41883F001024B43172606FB023214F8F4
:10C6D800041CFDF771FA04F8040C6B780E22C3F3FE
:10C6E80042035343287803F50A434C3300F007000C
:10C6F80003EB400001A90C3A05F019FB58E0182A91
:10C708004DD133490020FCF785F90620FFF7AAFD33
:10C718000C20FFF7B5FDFFF7C9FD284B1B78552BFB
:10C7280007D1237813F0C00F42D0C3F38112013A26
:10C7380006E0442B07D123789A09012A38DC013214
:10C7480062F3871333E0232B04D12378C3F3C202A7
:10C75800023A2AE0532B2BD1FCF720FA33781E4AF1
:10C7680043F006033370164B1648197840F8212019
:10C77800013119702378C3F3C201013161F3C50394
:10C78800C3F381112370104B11B1012904D101E0C9
:10C798001C3202E0114A00E0114A1A6008E0114A0E
:10C7A80000211170C3F3C202013A62F3C50323707A
:10C7B8007CBD00BFE31D0020991D0020CC1C00207B
:10C7C800C31D0020D01D0020041D002018250308CB
:10C7D8003925030819B302081CB3020854B3020828
:10C7E80070B302089E1D002073B5494B494D1A7855
:10C7F80012F0010F04D12A7812F0030208BF2A7040
:10C808001A78434E42F001021A702B78414C13F00B
:10C8180003022ED1404A1278552A03D1C3F382026B
:10C82800013A04E0442A06D1C3F38202013262F3DA
:10C838008403237017E0532A03D15A1C62F30103BF
:10C84800F7E7232A0FD1FCF7A9F93378334A43F0E5
:10C85800060333701378013BDBB21370304A52F889
:10C868002320304B1A6001A810211B22FFF738FD46
:10C878004CE0012A4AD101A810211A32FFF730FDF5
:10C88800254B1878232804D12378C3F341120132A9
:10C8980005E02A2807D12378C3F34112013A62F34D
:10C8A800461323702CE0532804D12378DA1C62F352
:10C8B8000103F6E7A0F13003DBB2092B01D94328C5
:10C8C8001ED12B7802AAC3F34113D4180C215A1C89
:10C8D80003F001034B4302F001021F2614F8041C65
:10C8E80006FB0232FDF768F904F8040C287801A960
:10C8F80000F01C0000F51E403430042205F017FA41
:10C9080029780948C1F34111FFF724FD7CBD00BF18
:10C91800E31D0020E51C0020CC1C0020C31D0020C6
:10C92800D01D0020041D00208CB30208064B1B7884
:10C9380003F08003DBB233B1435C04482021C01804
:10C948000322F3F727BD7047EC390020F4010020DB
:10C958004328F8B504460D46174606D1104B002665
:10C968001A786FF3C3021A7000E00E462046FCF7EF
:10C978000DF990B10A4B303C1A780A2602F00801EA
:10C98800C9B2002918BF002506FB05466FF3C3028C
:10C9980036B21A70BE42A8BF3E4630B2F8BD00BFDC
:10C9A800E31D00202DE9F3416E4F6F4E3B7843F0B5
:10C9B80001033B70347844B94BF2AF5005F0ACF941
:10C9C8006A4B6B491860204617E0012C02D1002001
:10C9D800684912E0022C02D1002067490DE0032CBF
:10C9E80002D10020654908E0042C02D100206449E6
:10C9F80003E0052C03D163490020FCF70BF83178DC
:10CA0800D9B9614B1B78312B01D1013101E0302BB1
:10CA180005D1564B4BF2AF50196005F073F95B4BDB
:10CA28001A785B4B02F08002D2B20AB1202202E0EF
:10CA38004E4A12683032DA776EE001290BD00229AB
:10CA48000CD003290DD004290ED04BF2AB55052983
:10CA580018BF00250AE04BF29B5507E04BF29F55A3
:10CA680004E04BF2A35501E04BF2A75529460422F6
:10CA780001A805F062F9474B474A03F1100153F842
:10CA8800040B8B4242F8040BF9D1032243489DF86A
:10CA98000410FBF7E5FF032241489DF80510FBF75A
:10CAA800DFFF03223F489DF80610FBF7D9FF3E48F9
:10CAB80003229DF80710FBF7D3FF334B3B4C187844
:10CAC800232804D12378022B22D8013304E02A2812
:10CAD80004D12378E3B1013B237019E0A0F13003BE
:10CAE800DBB2092B01D9432812D194F8008002AA9D
:10CAF800904418F8041CFF22FFF72AFF08F8040CDA
:10CB0800207802AA131813F8041C281805F0FAF85C
:10CB180027482178FFF70AFF1B4B1B78532B1FD19F
:10CB2800224B00221A7033780133DBB2062B3370A4
:10CB380004D0012B14D10D4B1B688BB1FDF71CF8E9
:10CB4800002333703B781B4A43F006033B7013788D
:10CB5800013BDBB21370184A52F82320174B1A60B6
:10CB6800BDE8FC81E31D0020931D0020AC1D0020C2
:10CB7800057103082E7203084F72030870720308C8
:10CB880091720308B2720308CC1C0020EC39002013
:10CB9800F401002064A0030804020020050200201C
:10CBA800090200200D020020110200209E1D002015
:10CBB80090B30208C31D0020D01D0020041D0020D2
:10CBC80070B5174C0D460646002120464FF4C17239
:10CBD800F3F7E0FBFF2D0AD1B10001F5DC41204657
:10CBE8001531042205F0A9F823789BB970BDFE2DF4
:10CBF80001D1173E02E0FD2D02D10136267009E071
:10CC0800B60006F5DC401530401905F085F8C0B2CD
:10CC1800207020B10248BDE8704019F053B970BDCA
:10CC2800082000202DE9F04119F07EF960B11020AC
:10CC38008F49FBF7EFFE8F4B1B78432B40F0EE81BB
:10CC4800BDE8F04119F092B919F080F9002826D012
:10CC5800894C23786BB110208849FBF7DBFE8848A4
:10CC68002D211030F3F714FC002800F0D78121782B
:10CC780010E010208349FBF7CDFE81482D211030AC
:10CC8800F3F706FC0446002800F0C88119F076F98D
:10CC9800014620468222BDE8F041FBF7E1BE7A4C0E
:10CCA80043F6CC2223689B68934250D0774E744D4C
:10CCB800307803EB800005F02FF803220146744812
:10CCC800FBF7CEFE2368986846F6797398422BD016
:10CCD800203B984228D03378013000EB830005F0E0
:10CCE8001BF80322014605F11500FBF7B9FE23687E
:10CCF80030789B68023303EB800005F00DF80322BF
:10CD0800014605F11900FBF7ABFE236830789B68F4
:10CD1800033303EB800004F0FFFF0322014605F113
:10CD28001D00FBF79DFE0EE02D2103225948F3F765
:10CD380031FB2D2103225848F3F72CFB57482D21AE
:10CD48000322F3F727FB20232B772B762B75544BE5
:10CD58001B7813F0010F00F0BD80236843F6CC2246
:10CD68009B68444D934261D04E4E484F3278387894
:10CD7800D31803EB800004F0CFFF4B4B014618603B
:10CD880028789846A0F13002D2B2092A01D943285E
:10CD98000FD109B2BA22FCF70FFF236832789B68DB
:10CDA8000146C8F800003878D31803EB800004F077
:10CDB800A9FF2B782A2B04D1337813B1394A013BC8
:10CDC80013702B78232B0ED13378022B0BD82268C3
:10CDD80046F6597192688A4205D020318A4202D0BB
:10CDE800304A013313702B78552B01D0442B0FD1C7
:10CDF800236831789B68A3F5DC43B3F1150248BF7B
:10CE0800A3F112023B7803EBA202D0B2FFF7D8FEDF
:10CE1800264B1B7803F08003DBB23BB13278184B0A
:10CE280003EB820320225A749A74DA742B78532BFA
:10CE380006D023689A6843F6CC239A4240F0EE80E5
:10CE4800FBF7ACFE236846F615629B68934203D154
:10CE58000E4B0220197806E046F67972934227D1E4
:10CE68000A4B002019780131BDE8F0410CF0BABA3C
:10CE7800345A0308CC1C0020601500200B59030805
:10CE8800F4010020555A0308041D0020931D0020BA
:10CE980005020020090200200D02002011020020D6
:10CEA800E31D00209E1D0020AC1D0020EC39002051
:10CEB80046F65972934204D1594B01201978091842
:10CEC800D2E746F61572934240F0A880544B0320EF
:10CED8001978C8E723684AF6FE029B6893423ED158
:10CEE8004F4E10204F49FBF795FD31784E4D01EB21
:10CEF800011101F52841FE311022284604F01DFFDA
:10CF08002B4605F110012A461078474F78B9474952
:10CF1800FBF780FD3846E721F3F7BAFA78B13178A4
:10CF2800401B381801310322FBF79AFD07E013F87C
:10CF3800010B10B9203003F8010C8B42E4D13C4DB1
:10CF48002B782A2B03D13078FD21FFF739FE2B7877
:10CF5800432B63D1307823680130C0B259E043F6DF
:10CF6800CC229342324E1AD010203249FBF752FDA0
:10CF780033782A2B52D1304B1B689B68A3F5DC43CE
:10CF8800B3F1150248BFA3F11202254BFF211B780C
:10CF980003EBA202D0B2BDE8F041FFF711BE33782F
:10CFA8001F4D552B04D12B78142B01D1033B2B702B
:10CFB8003378442B05D12B78122B02D1184B15222C
:10CFC8001A702B78DFF874805901C918414401F5AB
:10CFD800944100201F31FBF71DFD08F592411020F8
:10CFE80017312F78FBF716FD3378112F8CBF0327E5
:10CFF80000272A2B05D12878FE21C01BC0B2FFF7D5
:10D00800DFFD3378432B09D12B78173BDF1B2368CF
:10D01800F8B2997CBDE8F04118F06EBFBDE8F08128
:10D02800931D0020135A0308F4010020233B030832
:10D03800CC1C0020D1590308041D0020FC10030853
:10D0480010B50E4B1B78452B17D10D4B1A7842F0B3
:10D0580006021A700B4A1378032B0ED80A490B4C98
:10D06800086844F823000133137083680B60FBF7EA
:10D07800D9FBBDE81040FBF791BD10BDCC1C0020CA
:10D08800E31D0020C31D0020041D0020D01D00202A
:10D0980010B50C4B04462146D8790FF002FC60B15C
:10D0A800204655210FF05CFA48B120460FF0EEFA01
:10D0B800D0F1010038BF002010BD022010BD0220B1
:10D0C80010BD00BFA21D002008B50FF0D9FBC0B2EB
:10D0D80008BD00002DE9F047634B644C1A78994667
:10D0E80012F0010F624D65D02078FFF7D1FF614A39
:10D0F8002B181178604F93F8A031604E442938708E
:10D10800336090460AD12D2B08D038B995F8A11173
:10D1180001233B7031602078FFF7D6FF98F8003084
:10D12800552B10D133682D2B0DD03B785BB1013BCB
:10D13800514ADBB21370EB1893F8A0114F4B2078CB
:10D148001960FFF7C1FF98F80030232B19D14C4B19
:10D1580020781B689B7C013B984212DA434B0130D4
:10D16800C0B21870FFF794FF3870281890F8A031F3
:10D178003360444B9B7803F00203DBB20BB1FBF73F
:10D1880045FB98F800302A2B14D1207890B1374B02
:10D198000138C0B21870FFF77BFF3870281890F874
:10D1A800A0313360374B9B7803F00203DBB20BB13D
:10D1B800FBF72CFB344EFCF7DFFC237832789A42DD
:10D1C80088BF337032780F32934202DD2E4A0F3B0C
:10D1D8001370DFF8C480002730783818C0B2FFF722
:10D1E80057FF281890F8A0310137102F08F8013F91
:10D1F80007D0254B1A78224BBA181B689B7C9A4299
:10D20800EADB99F8003013F0010F13D01F4B1A789E
:10D218001F4B02F08002D2B22AB122783178103244
:10D22800521A5F2105E0227831781032521A1349D8
:10D2380009689954134DAB7803F00203DBB25BB174
:10D248002078E91D652246F61573FBF72FFB0520AC
:10D258000B212A46FBF796FB21780E480131022262
:10D26800BDE8F047FBF7FCBBE31D00209E1D002036
:10D27800F4B10208CC1C0020E41C0020AC1D0020E6
:10D28800041D0020F41D0020951D0020EC3900200D
:10D29800F4010020F5010020030200202DE9F041EF
:10D2A800002480460D4616462346012717FA04F245
:10D2B80098F80010E0B2914206D146F65973294613
:10D2C8003246FBF7F3FA3B460134042CEDD1043C1B
:10D2D8000A4AE0B2A218917898F800208A4207D149
:10D2E80032B146F6797329463246FBF7DFFA012355
:10D2F8000134042CECD11846BDE8F081A21D0020B1
:10D308002DE9F041074610460D461446F3F792FA08
:10D31800C3B28046B3B1AB4214D80B4E20212A4683
:10D32800F019F3F737F82046F3F784FAC8EB050548
:10D338006D08EDB2EF1902462146F019BDE8F0413B
:10D34800F2F780BFBDE8F081F4010020312200230C
:10D358000178194111F0010F02D00449C9188A75E2
:10D3680001330132042BD2B2F2D17047F40100200C
:10D378002DE9F04F87B09DF840408146072C0D46B7
:10D3880005929A4637D1073C27462B78234113F05C
:10D39800010F2CD0012623B24FF000080293512030
:10D3A8003146324633460096CDF8048004F032FD0B
:10D3B8001B204146A2194346CDF80080F5F7A0F995
:10D3C80037B9112039463A4633460097F5F798F9A8
:10D3D800534B204613F8242001276FF3000203F86B
:10D3E80024201199F6F750F82046F6F74BFA013445
:10D3F800042CCAD10DE2012C03780CD10BB90B789F
:10D4080023B3FF2300930021464B01911B780C2086
:10D418000133029316E0022C09D10BB90B78ABB19A
:10D428000021FF2300930191029134200AE0062C89
:10D438000CD10BB90B784BB10021FF23009301915C
:10D448000291652004220B4604F0E4FCBAF1010FB6
:10D4580099F800302BD13BB1334B0020D9790246E3
:10D4680053460090F5F74CF92B783BB12E4B012031
:10D47800D979002203460092F5F742F90020F5F722
:10D48800B9FF99F80030002B5BD0284B1978002998
:10D4980057D1274B5B78002B53D0FF2300933A20BA
:10D4A80001220B460191029104F0B4FC49E063B1FA
:10D4B800052C4FF0000102D100910F2001E00091EE
:10D4C8000B200A460123F5F71BF92B7883B1052CAD
:10D4D8004FF0000106D110200A4601230091F5F70C
:10D4E8000FF912E00C200A4601230091F5F708F91C
:10D4F800022C25D0032C01D10E4B02E0042C02D1C2
:10D508000D4B1F781DE0052C01D10C4BF9E7012CC0
:10D5180001D1044BF5E7062C0CBFFF27002710E0CC
:10D52800A9190020761A0020A21D002094190020B5
:10D538006B130020BC1F0020835700200B3C0020E9
:10D54800FF2799F80030002B00F0B580934B944EDC
:10D558001A78984602F02002D2B262B1317811F0FE
:10D56800010108D1FF230093282001220B460191D5
:10D57800029104F04FFC98F8003003F01003DBB27E
:10D588006BB1317801F00201C9B241B9FF230093B0
:10D59800292001220B460191029104F03BFC98F8E6
:10D5A800033013F0010F0DD0317801F00401C9B236
:10D5B80041B9FF2300932A2001220B4601910291D1
:10D5C80004F028FC98F8033003F00203DBB26BB1D7
:10D5D800317801F00801C9B241B9FF2300932B202B
:10D5E80001220B460191029104F014FC98F80330D3
:10D5F80003F00403DBB26BB1317801F01001C9B25A
:10D6080041B9FF2300932C2001220B46019102917E
:10D6180004F000FC98F8033003F00803DBB26BB1A8
:10D62800317801F02001C9B241B9FF2300932D20C0
:10D6380001220B460191029104F0ECFB11F01AFF54
:10D6480068B1317801F04001C9B241B9FF230093B4
:10D65800492001220B460191029104F0DBFB98F866
:10D66800033003F04003DBB26BB1317801F0800185
:10D67800C9B241B9FF2300934E2001220B46019104
:10D68800029104F0C7FB767816F0010613D14548DD
:10D69800314617F068FE58B1FF230093731C002130
:10D6A8001BB20293752001220B46019104F0B2FBD4
:10D6B8000136702EEBD1119B3B4A19783B4B51B187
:10D6C80099F8001011702A781A702B780BB1542031
:10D6D80005E0522003E011702A7853201A7004F0F4
:10D6E8006BFF119B00261A78314B1A7099F800309D
:10D6F800334113F0010F2DD03146059817F033FE52
:10D708000122014628B933B20190009202931046D3
:10D7180005E0002133B200920191029324200B46C8
:10D7280004F078FBBAF1010F05D1224B8020DA7999
:10D738000521013208E0022C07F1010202D1802004
:10D74800072101E0802006213346F6F7FBFB30462F
:10D75800F6F76CF82B78334113F0010F55D0002100
:10D768004FF0010B33B2029302205A460B46CDF814
:10D7780000B0019104F04EFBDA45DFF83C801DD182
:10D7880018F8263013EA0B0332D10A4A0520D1795A
:10D798000093594406EB0B0228E000BFEC39002047
:10D7A800681B002084190020E1190020E2190020DC
:10D7B800861B0020A21D0020A919002018F8263079
:10D7C80013F0010314D1022C0CD1134B1B7803F076
:10D7D8002403042B04BF114B83F800B000230093EB
:10D7E800072001E000930620791C721CF4F788FFDB
:10D7F80011993046F5F748FE3046F6F743F818F821
:10D8080026306FF3000308F826300136042E7FF423
:10D818006DAF07B0BDE8F08F901B002064130020A7
:10D828002DE9F04180460E46174646F63F1500247E
:10D838003846214617F097FD88B1294608220B483B
:10D8480004F07BFA0948414617F03AFD074817F0FB
:10D858005DFD20B90123A3403278134333700134AE
:10D868000835042CE4D1BDE8F08100BF7E1B002000
:10D878002DE9F04387B08046894604A847F269310C
:10D88800082204F05AFA002440462146E7B217F06D
:10D898006AFD002843D03846F4F76AFC0025661C68
:10D8A8000246314611202B460095F4F729FF012343
:10D8B80021462A460420FF080095F4F721FF4BF281
:10D8C8005F70381804F028FA04F00703C1B2194150
:10D8D80011F001014FF002024FF001030AD000924B
:10D8E800019336B27720294692182B46029604F007
:10D8F80091FA14E00092019336B2232004220B46D9
:10D90800029604F087FAB9F1000F08D004A821465E
:10D9180017F029FD18B10548214617F00EFD01340E
:10D92800402CB1D107B0BDE8F08300BFBE1900207C
:10D938002DE9F74F9846137805460C4617469DF88B
:10D9480030909DF834B09DF83800DFF8C8A073B166
:10D958002A4A51786FF3820151703B7800EA030339
:10D968003B7021789AF800208A18D31A2B702378F4
:10D9780083B123482146F5F731FF2249204817F0A3
:10D988009FFC1F480121FFF773FF1D4841462246AF
:10D99800FFF746FF1C4B00261E70297843F6FB2034
:10D9A80004F0B0F9494646F64D0004F0ABF92046BC
:10D9B80039464A46F5F7D4FC144B42469E70394620
:10D9C8004B462046CDF800B00195FFF7D1FC28461C
:10D9D800F8F756FC2B780E480E498AF80030F5F710
:10D9E800FDFE12F095FD88F800603E7026702E70DE
:10D9F80003B0BDE8F04F04F0E9BC00BF073C0020CD
:10DA0800871B0020D9190020E01D00206B1300207F
:10DA18006A1B00209419002010B50B4B0B4C0246D2
:10DA280003CB206061600A48114617F06AFC214662
:10DA3800074817F045FC064817F068FCD0F10100CC
:10DA480038BF002010BD00BFC02D0020741B00206F
:10DA58007E1B002010B50A4C637C4BB1002009499D
:10DA6800FAF7D8FF084B1B78432B01D1433B63746B
:10DA7800607C20B90549BDE81040FAF7CBBF10BD5E
:10DA8800CE1C0020653B0308CC1C0020443B030847
:10DA9800034B1A7801321A7001230370704700BFD4
:10DAA800E01D002010B50C48FAF75AFF0B4A002475
:10DAB80014700B4A0B4B14700B4ADC7014700B4A31
:10DAC8009C7014700A4A1C7114700A4A1470FBF78F
:10DAD80065F8094B1C6010BDF41D0020A21D002034
:10DAE800CD1C00206B130020E41D0020F11D002038
:10DAF800081D0020E01D0020041D00202DE9F04F26
:10DB08009C4B9D4F93F800903B68DFF8C0829C7C4B
:10DB18009A4BF0221A7098F800308BB00D2B3D46C6
:10DB2800464645D1202196486FF02F02F2F732FC85
:10DB3800944B93F803C0BCF1010F04D903225A7126
:10DB4800002091492FE01AD10024DC708F4A904BB5
:10DB580090499148914D04701C7014700C70CDF868
:10DB680000C001942D780295FFF7E2FEFBF716F846
:10DB78008B483C600BB0BDE8F04FFAF7F1BE89481E
:10DB88008449F5F72BFE884B884A03CB884B1060F5
:10DB98001B785160532B5FD198F8003085490133C9
:10DBA80088F8003000200BB0BDE8F04FFAF732BF1C
:10DBB800092B0FD17E4B1B78532B3DD17E4B002276
:10DBC8001A700D2388F800307C4B1A7842F0060250
:10DBD8001A7089E20E2B37D1754B1B78532B2BD13A
:10DBE8007749704817F06CFB6E48FFF715FF04463D
:10DBF80040B198F800300522013B88F80030614BAD
:10DC0800DA7071E2082246F64E01684804F095F889
:10DC180066496C4817F075FB012300935F4B01942C
:10DC28001B785D4802935B49584A594BFFF780FEC1
:10DC3800FAF7B4FF3C6057E2232B40F055820BB053
:10DC4800BDE8F04FFFF72EBF33B95F4B1A781AB90A
:10DC580001321A7012F05CFC631E48BFA31DDB1072
:10DC6800013303FB09F91FFA89F909F5D047A9F52A
:10DC78009049A9F1A109514BCDF81C901A784E375B
:10DC880012F0010F4C4C00F02381494B1A78994649
:10DC9800432A40F0CC8033780D2B40F0C8804148AF
:10DCA800217817F060FB002800F0C1803F482178F8
:10DCB80017F059FB002840F0BA80079920780FFA2E
:10DCC80081FB0BEBD00004F027F823784FF0010A12
:10DCD80003F007020AFA02FADFF8F4805FFA8AFA18
:10DCE80010EA0A0FC8F8000027D0264B5B78002BF3
:10DCF80040F09D80294BD879F8F720FA002800F0E9
:10DD08009680D8F80010CAF1FF0A20780AEA0101C3
:10DD1800C8F800100BEBD00003F0F4FF20780FFADE
:10DD280087FB0BEBD00003F0F7FF00EA0A0120782D
:10DD3800C8F800100BEBD00064E00FFA87FC0CEB7E
:10DD4800D300CDF814C003F0E7FF10EA0A0FC8F8B3
:10DD580000003FD140EA0A01059A2078C8F800106F
:10DD680002EBD00003F0CEFF2178164817F0E5FA51
:10DD78005DE000BF931D0020041D0020EF1D002062
:10DD8800040200206B1300200A3C0308E41D002055
:10DD9800CD1C0020F11D0020081D0020A21D002020
:10DDA800F41D0020871B0020C02D00207C190020B6
:10DDB800CC1C0020D03C03089E1D0020E31D002041
:10DDC800CE190020D919002030140020E01D0020B1
:10DDD800AC1D0020914B5B7823B9914BD879F8F7AB
:10DDE800ADF9B0B9059B2078CAF1FF0A03EBD00062
:10DDF80003F092FF8B4A00EA0A01059B2078116024
:10DE080003EBD00003F07EFF2178874817F0A0FAD3
:10DE18000DE020780BEBD00003F07EFF40EA0A010A
:10DE28002078C8F800100BEBD00003F06BFF99F8CE
:10DE38000030232B10D12A682378927C013A934230
:10DE48000ADA7A4A01331370794B9B7803F002039C
:10DE5800DBB20BB1FAF7DAFC99F800302A2B0CD1B7
:10DE6800237853B1714A013B1370714B9B7803F0CF
:10DE78000203DBB20BB1FAF7C9FC99F80030552B55
:10DE880012D129682278897C684B08398A4201DADC
:10DE9800083200E000221A70654B9B7803F00203F9
:10DEA800DBB20BB1FAF7B2FC99F80030442B0FD172
:10DEB80022785E4B072A9CBF2A68927C083A1A701F
:10DEC8005B4B9B7803F00203DBB20BB1FAF79EFCC5
:10DED800FBF752FE574A237811789246994288BF39
:10DEE800137012780F32934202DD524A0F3B1370BF
:10DEF8002B684FF0000B93F81280CDF818B0B8F1EA
:10DF08000F0F9ABFC8F120085FFA88F84FF0100881
:10DF180031784FFA8BF30D2905D19AF800209B1818
:10DF2800DB10454A04E09AF800209B18434ADB10AE
:10DF3800D35C9AF8002005934FFA8BF39A180D29B1
:10DF480002F007094FEAE20202D13D49895C0691D5
:10DF5800DDF81CC004930FFA8CF0101803F0DCFEF7
:10DF6800C0B2049B08909AF800003AB2181802EB65
:10DF7800E00003F0D1FE3278049B09929AF8002061
:10DF8800C0B29A1846E0059BDDF824C043FA09F1AF
:10DF98002C4B01F0010100290CBFA521DB21BCF1AC
:10DFA8000D0F03F8081014D127494FEAE20C11F8B5
:10DFB8000C1041FA09F111F0010F08D0DDF818C072
:10DFC8004CFA09F111F0010F03D0582110E02D216E
:10DFD8000EE0DDF820C04CFA09F111F0010F01D074
:10DFE800502105E040FA09F111F0010F02D0542147
:10DFF80003F8081009F101095FFA89F90BF1010B1F
:10E0080008F101080132B9F1080F5FFA8BFB5FFADA
:10E0180088F81BD0B8F1200FB5D124E06B1300208D
:10E02800A21D0020AC1D0020D91900209E1D002033
:10E03800F41D0020951D0020CE1900202E1A002066
:10E048007C190020F4010020871B0020B8F1200F64
:10E0580009D09AF800304FFA8BF2D2182B689B7CC3
:10E068009A42FFF655AF22490B7813F0010F17D0EB
:10E078002B68204A9B7C12780F2B02F0800298BFF5
:10E08800C3F11003D2B294BFDBB2002342B12278AD
:10E098009AF800101032521A1749CB185F21995478
:10E0A800164EB37803F00203DBB25BB12078F11DA2
:10E0B800652246F61563FAF7F9FB05200B2132466F
:10E0C800FAF760FC2B689B7C0B2B0DD9B37803F017
:10E0D8000203DBB243B121780948013102220BB0B7
:10E0E800BDE8F04FFAF7BCBC0BB0BDE8F08F00BF3D
:10E0F800E31D0020EC390020F4010020F41D00206D
:10E10800F501002088234B43054A03EBD003D35C79
:10E1180000F0070053FA00F000F00100704700BF5C
:10E12800840D002070B504461646157839B912E0FA
:10E138000135EDB228462146FFF7E4FF48B9202D06
:10E14800F6D970BD013DEDB228462146FFF7DAFF4A
:10E1580008B1356070BD002DF4D170BD064B382173
:10E168001B78032201FB0031044844230370C9B221
:10E17800173BC370FAF774BC9E1D0020F401002001
:10E18800012802D0022806D102E01D20044904E03B
:10E198001D20044901E004491D20FAF73BBC00BFDB
:10E1A800B134030890340308D234030803780968AB
:10E1B8000F4A03EB0310401802EBC00050F8240C80
:10E1C8000C4988420FD1882101FB03239A68A0F5E6
:10E1D8009C63063B9A4208D0A0F598600538101A4F
:10E1E80018BF01207047002070470020704700BF0B
:10E1F800840D00206F34030803780A6803EB0313C7
:10E20800D318084A053B02EBC3035968064A9142F2
:10E2180005D1187A09288CBF0020012070470020FA
:10E22800704700BF840D00206F3403082DE9F04FBC
:10E23800984B994FF0221A703B6889B09C6847F652
:10E248007313E11A4C4244EB0104CC3A6243934BFA
:10E258009D5C03EB0208C5F30005EEB23A46002EBA
:10E268002CD130468E49FAF7D5FB8E4B1B78232BE1
:10E2780041F02A8298F8013066F3041388F80130D7
:10E28800FAF78CFC884B1A7842F006021A70874A13
:10E298001378013BDBB21370854A52F823303B6098
:10E2A800844B1D70844B1D70844B1D70844B1E6005
:10E2B800844B1D70844B1D7001F006BA814D95F892
:10E2C8000090B9F1000F0CD04FF43661614309F1A9
:10E2D800FF30342303FB00137C49CB181B798DF8DE
:10E2E8001F307B4B1E787EB17A4E2046317811F074
:10E2F800A5FF002840F05C84754930700870074617
:10E308000646804600F05BBC6D490B688B46A3F15E
:10E318001200032809D9A3F11601032909D9A3F189
:10E328001A01032909D9374605E037464FF0010895
:10E3380005E037460126B84601E00127B0465949AD
:10E348000978532940F0D581B9F1000F3AD17222EA
:10E3580062436149885C10F0020F0AD0002B41F03B
:10E36800B381013363F383008854CBF8003001F0A4
:10E37800ABB95A4B997989B120464A4611F046FF04
:10E38800FF2801F0A18101302870CBF80090FAF73E
:10E3980005FC2046FFF7E2FE01F096B9DFF8FCC065
:10E3A800242202FB04C25178204669F304115170FB
:10E3B8004B4A022182F80090039311F0CDFE01220E
:10E3C800039BCDE209F1FF312046C9B211F036FFB7
:10E3D800002840F08B80DFF810B1DFF8EC909BF854
:10E3E8000020012332B98BF80030324B89F8002025
:10E3F8001A70E4E305900393FAF7D0FB05988BF8BD
:10E408000000039B89F80030364A835C9246A3F1EA
:10E418003001C9B2092904D9413BDBB2052B01F20D
:10E42800538101300A28EFD14FF0000847460AEB24
:10E43800480016F0CDFF7B080237FFB20A2F294E9D
:10E448000AF8030008F10108F1D1304612F0FCFB8C
:10E45800002801F03981304612F064F90746002897
:10E4680041F032811D4B3046997912F0FCFB0028AF
:10E4780001F02A812978337901392046C9B202226C
:10E488000097019612F042FC022389F8003001F04F
:10E498001BB900BFEF1D0020041D0020F339002028
:10E4A800FF250308CC1C0020E31D0020C31D00200D
:10E4B800D01D0020E91C0020121D0020931D002003
:10E4C800AC1D00209E1D0020951D0020643E0020EC
:10E4D800E01C0020941D0020245500206B13002010
:10E4E800E21D0020C41D00209F1D0020DBF8003025
:10E4F800DFF80893202B27D0212B23D14FF4366245
:10E50800624329783420013900FB0122AC489DF888
:10E518001F3012184FF0000B20460192C9B2032297
:10E52800CDF800B012F0F2FBFAF738FB2A78A54BC9
:10E53800013AA5481A701423C9F800B085F800B04C
:10E5480003703CE31E2B03D10133C9F8003019E3F3
:10E558001F2B18D14FF436626243297834200139D1
:10E5680000FB012296484FF0000B121801929DF80B
:10E578001F302046C9B20622CDF800B012F0C6FB03
:10E58800C9F800B0FEE29A1F062A0ED88F4B1A78F7
:10E5980019462AB901321A708D4B1A788D4B00E34F
:10E5A800012A40F00C830223A1E1A3F10D02042A01
:10E5B8003AD88949D3B291F800C095F800E080486C
:10E5C800864ABCF1000F1ED04FF0000C81F800C045
:10E5D80011784FF4366262430EF1FF3E0CF1340CB1
:10E5E8000CFB0E228018C0184174382000FB04EE82
:10E5F8005FFA8EF000EB800000F5FA409B30C018FF
:10E6080003F080FBDBE24FF0010C81F800C04FF40F
:10E61800366161430EF1FF3E0CF1330C0CFB0E1E0C
:10E628007044C3185B7C59E0A3F112020B2A4CD842
:10E638006B4A29781078002845D000201070A3F183
:10E64800120938224B1E02FB0433203ADBB2534333
:10E6580003F5FE435FFA89F9DFF894B1CB3303EB96
:10E6680049039BF800101846039303F04BFB5D4ADF
:10E678004FF4B66C0CFB04FC11781A22013902FB2A
:10E6880001C14F48494400EB41019BF80000DFF805
:10E6980070B18875039B9BF80010581C0492CDF844
:10E6A80014C003F02FFB4F49049A0B78DDF814C00F
:10E6B800013B02FB03C2424B4A4403EB42029BF874
:10E6C8000030D3757BE2012308E0DFF8209199F848
:10E6D80000302BB9012289F80020434A13706EE2FA
:10E6E800FAF75CFA002389F800302046FFF736FD78
:10E6F80065E243294BD1354A1278002A40F05F82FF
:10E70800354A1278002A40F05A82B9F1000F00F019
:10E718005682364A1278002A40F05182212B30D096
:10E728001F2B30D02E4B1978012919D9B8F1000FB9
:10E7380002D1002F00F043822D4B02391A7852FA89
:10E7480001F010F0010F4FF0010004D010FA01F1B0
:10E7580022EA010225E210FA01F141EA020220E26E
:10E7680000F02D8209F1FF312046C9B211F066FD93
:10E7780020B9204B1B78002B40F0218200232B70FE
:10E7880000E2202300E01E23CBF80030FAE1232921
:10E7980040F096800D4B1B78002B40F010820E4BFA
:10E7A8001978002940F00B82104BB9F1000F50D0B6
:10E7B8001A783AB30C480F2A01700F48017042E1E9
:10E7C800643E0020941D0020E01C0020E21D002073
:10E7D800921D0020F01D0020AB1D0020601E0020AF
:10E7E800971D00209E1D0020E91C0020931D00207D
:10E7F800911D00209F1D0020121D0020AC1D00202F
:10E80800E11D002009F1FF312046C9B211F016FDC3
:10E81800B0B19A4A13787BB1B8F1000F01D0042B3C
:10E8280008D90EB1012B05D9002F00F0C881042B9F
:10E8380000F2C281013351E79DF81F000121F6E083
:10E848008F4B1A78511EC9B208296FD801321A7035
:10E858006CE0DFF86CC2242101FB04C1487869F33D
:10E8680004104870022120460492039311F074FCAE
:10E8780009F004FCFAF792F98249087840F006009A
:10E888000870814801780139C9B201707F48049A3B
:10E8980050F8211011607E4A82F800907D4A82F873
:10E8A8000090039BCBF8009083F800907A4B85F892
:10E8B800009083F80690794B83F8009000F004BF2D
:10E8C8002A2936D1764B1B78002B40F07881754B7E
:10E8D8001A78002A40F0738173490B784BB16C4861
:10E8E800012B02706B48027040F26981013B0B708A
:10E8F80065E1B9F1000F00F0628109F1FF312046AE
:10E90800C9B211F09BFC58B15C4A137823B1012BB2
:10E9180040F25581013BE1E69DF81F00002186E0A9
:10E92800574A1378012B01D9013B13700022584B29
:10E9380037E1442940F08D80594A1278002A40F086
:10E948003E81B9F1000F0DD1534B9A79511EC9B2CE
:10E95800012901D8013203E0032A40F03081023A4C
:10E968009A712CE1504A1278002A40F02881444AD2
:10E978001278002A40F023814A4A1278002A58D196
:10E988003E4B1B78012B09D9002E00F01881474B0C
:10E998001A78072A00F212810132AAE019D1B8F1D7
:10E9A800000F0BD0424A032011789846013191FBA1
:10E9B800F0F000EB4000091A117000E1002E00F0A1
:10E9C800FE803B4A1E461178013101F003011170A7
:10E9D800F5E0314B204699794A4611F017FCFF289B
:10E9E80000F0ED80DBF80030212B00F0E8801F2BD1
:10E9F80000F0E580013028702046FFF7AFFB4FF4A8
:10EA08003662624329783423013903FB0123294AFA
:10EA18009BF80000D31893F8049049468DF81F908E
:10EA2800FFF770FB0146002840F0AC804846224AB8
:10EA3800A6E00D2B0BD19DF81F0011F0B1FA30B1F3
:10EA48001E4B1A781F2A00F2BA800132A9E0012071
:10EA5800AAE0552940F0B380114A1278002A40F004
:10EA6800AE80B9F1000F2DD10B4B9A79012A01D94B
:10EA7800013A75E740F0A380032271E7971D002053
:10EA88009F1D0020E31D0020C31D0020D01D002075
:10EA9800E91C0020121D00206B130020951D00208A
:10EAA800E21D0020AB1D0020931D0020911D0020B9
:10EAB800E11D0020643E0020AC1D0020601E0020E7
:10EAC800F3390020894A1278002A78D1884A1278C6
:10EAD800002A74D1874A1278002A56D1864B1A78B0
:10EAE800012A08D9002E6AD0844B1A78012A65D9E0
:10EAF800013A1A7062E012D1814B197811B10139CB
:10EB080019705CE0B8F1000F03D00221197090462B
:10EB180055E0002E53D00321197016464FE0B9F185
:10EB2800010F4CD9774BA9F1020220469979D2B24C
:10EB380011F07AFBFF2842D0DBF80030DFF8D091E3
:10EB4800212B3CD01F2B3AD0013028702046FFF7EC
:10EB580005FB4FF43662624329783423013903FBFD
:10EB68000123694A99F80000D31893F804B059466C
:10EB78008DF81FB0FFF7C6FA014618B958464A463D
:10EB8800FFF7D0FAFAF70AF819E00D2B0BD19DF828
:10EB98001F0011F005FA30B15C4B1A78012A0ED922
:10EBA800013A1A700BE0FF20584911F017F906E0F6
:10EBB80000273E46B84602E0012700E001262978F2
:10EBC800DFF89891002940F0CB8099F8003013F0D5
:10EBD800010205D143F0010389F800304C4B1A605B
:10EBE80000252046294611F0C3FD30B17223634346
:10EBF800484AD15C41F00201D1540135382DF0D199
:10EC08003A356543434E735D13F0020F43F34000FA
:10EC180015D03F4C206810B93F4900F0C1BC002016
:10EC28003E49F9F7F7FE735D13F00C0F43F38105C6
:10EC380040F04A85F9F7B2FF256000F045BD314D37
:10EC4800AB79A3B1012B01D1354906E0022B01D1E3
:10EC5800344902E0032B02D13349F9F7DBFEA979E5
:10EC6800204611F01DFB022201463048EDE114B99F
:10EC780020462F4901E02F491846F9F7CBFE2E48C8
:10EC880003786BB92D490A222D48F1F759FE2D4911
:10EC9800242303FB04135A7842F010025A7004E04C
:10ECA800274829490A22F1F74BFE284D382102222C
:10ECB80005F11E00F9F7D4FE204611F015FB0222DB
:10ECC800014605F11900F9F7CBFE214B00221A7015
:10ECD800204B1B7803F08003DBB2002B00F0F48498
:10ECE8001D4B1B88EB8100F0EFBC00BF931D00207B
:10ECF8009F1D0020AB1D0020971D0020911D0020A6
:10ED0800E11D00206B130020643E0020601E0020DF
:10ED1800AC1D002024550020412603086226030864
:10ED28006A2703088B270308AC2703081202002070
:10ED3800A426030828270308E01C0020CD27030881
:10ED4800FA010020F3390020EE270308F40100201F
:10ED5800951D0020EC39002071A00308E31D002058
:10ED680001392046C9B211F069FA002800F0F4838D
:10ED7800954B93F800B038230BF1FF3B03FB04BB22
:10ED880099F800305FFA8BFB13F0010F03D08F4A1C
:10ED98001378002B41D08E48F9F7E2FD0BEB0B11ED
:10EDA80001F5EA4110228B48BB3102F0C6FF884BBF
:10EDB80011229A71884B1B6813B91020874921E0EA
:10EDC800012B02D1102086491CE0022B02D1102011
:10EDD800844917E0052B02D11020834912E01E2B2D
:10EDE80002D1102081490DE01F2B02D1102080494B
:10EDF80008E0202B02D110207E4903E0212B03D10B
:10EE08007D491020F9F706FE99F800306F4843F065
:10EE1800010389F8003000230370784B1A78002A20
:10EE280000F0AB800BEB0B1B0BF5EA4909F1BB09B2
:10EE380010227348494602F080FF00229346704B27
:10EE4800995C41B10BF1010B5FFA8BFB0132BBF10D
:10EE5800100FF4D107E06A49C2F1100201EB0B0070
:10EE68002021F1F797FA654A107858450BD90138EF
:10EE7800484402F051FF30B9604B2021187801381E
:10EE8800484402F03FFFDFF894B19BF80030184681
:10EE98000393F9F77BFEDC46039BDFF878B110B9E2
:10EEA800432B44D101E0432B05D100238BF80030DC
:10EEB8004FF0200A30E05348534A90F800E0534995
:10EEC8009E450ED1AEF1300E0A20137800FB0E1EBF
:10EED8000133DBB21370734493F8AD307BB9137010
:10EEE8000DE003709BF800304FF0000E82F800E050
:10EEF8002BB1424803780F2B01D80133037040230C
:10EF08008BF8003013789CF800200A20303A00FB78
:10EF18000211C91891F8ADA03849394A0878514604
:10EF2800013802F800A0484402F0ECFE0FE0384B2C
:10EF38001B7803F08003DBB24BB19BF8003033B988
:10EF48002E482F490378FF22CB1803F8012C9BF891
:10EF5800003013B12F4A013B13709BF80030012B8E
:10EF680010D1264A13780F2B01D801331370264A83
:10EF780000238BF80030137004E004200C21144A9D
:10EF8800F9F700FD144A13689346002B48D14FF453
:10EF98003662624329783424013904FB01241E4A6D
:10EFA800A4186178164AC1F3C30109B93F2004E0E7
:10EFB800994201D9DB2000E0A5200133DBB290752E
:10EFC80001320A2BF1D17FE39E1D0020951D002000
:10EFD800F41D0020FB1D0020AC1D0020EB330308AE
:10EFE800D528030817290308DD290308822A0308FE
:10EFF800A32A0308C42A0308E52A0308931D00204E
:10F00800F4010020E61C0020121D0020F4B10208C3
:10F01800EC390020E91C00206C3E0020CC1C0020AC
:10F02800012B15D14FF4366363432A783424013A0F
:10F0380004FB0234AB4BE418637813F0070300F0C9
:10F04800438314215943A8488322F9F709FD3BE378
:10F05800022B26D1A54A9DF81F30882101FB0323E6
:10F068002978A34AD87901390623202502F80159BD
:10F0780050FA03F515F0010F10D04FF436656543CB
:10F08800342606FB01559B4E7519ED791D4115F087
:10F09800010F01D0DB2500E0A5255570013BE4D226
:10F0A80012E3032B13D14FF4366363432A783424D5
:10F0B800013A04FB02348F4B1C19237A13F0010F19
:10F0C80002D010208C496BE210208C4968E2042B96
:10F0D80013D14FF4366363432A783424013A04FB8E
:10F0E8000234844B1C19237A13F0020F02D010202B
:10F0F800834955E21020834952E2052B15D1162782
:10F1080000262B783422013B53434FF4366202FB2E
:10F118000433784A7C49D318985DC919013616F02A
:10F128003DF90237052EECD1CEE2991F062900F2EF
:10F13800FF809DF81F206D4F02EB0210411807EB6E
:10F14800C101C968714801F1100651F804CBB142F8
:10F1580040F804CBF9D19E1FF6B202EB02129219C5
:10F16800013207EBC202507A92F80AC0684A29783D
:10F178001378904673B94FF43663634334220139E8
:10F1880002FB0131634BCA5E634B024102EA0C0287
:10F198001A7011E0022B0FD1604B01391B784FF028
:10F1A800000900932046C9B204223346CDF80490E2
:10F1B80011F0ACFD88F8009098F80030012B29D1A7
:10F1C800574BDFF8589193F800A05046F9F7DEFC4A
:10F1D80010B9BAF1430F1AD10DF11F005149FFF7C9
:10F1E8000BF810B1002389F800309DF81F30DBF8C8
:10F1F800002003EB03139B1807EBC303504699F851
:10F20800001013F8202CFAF7D7FC89F8000099F8B9
:10F2180000A003E013B9404B93F800A0BAF1090F1E
:10F2280007D9BAF1630F8CBF4FF003094FF00209F9
:10F2380001E04FF001099DF81F3003EB03139E19FD
:10F2480007EBC607FB685A7BE02A02D12E4A202129
:10F2580051779A7BE02A02D12B4A20219177DA7BD9
:10F26800E02A02D1284A2021D17798F800200ABB49
:10F278004FF43662624329783424013904FB0124AF
:10F28800184AA418A27812F0080F1BD05A7BE02A5B
:10F2980002D11D4A3F2151779A7BE02A02D11A4AAE
:10F2A8003F219177DB7BE02B40F00E82164B3F220B
:10F2B800DA7709E21C4B1B7803F08003DBB2002BE2
:10F2C80040F002820DF11F001649FEF76FFF18B1DA
:10F2D8005046FEF755FFF7E114485146C9EB0000C8
:10F2E8004A46B2E66C3E00200F020020840D002042
:10F2F80013020020643E00207A2903089B29030892
:10F30800402A03081F2A0308F401002004020020F1
:10F31800E21D0020693E0020921D0020F01D002003
:10F32800CC1C0020AC1D0020EC3900201402002069
:10F33800A3F10D02042A31D89DF81F30D6B222223B
:10F3480002FB0363984A02EB83035F6C3846F1F7CC
:10F3580071FA394602469548F1F7F2FA944B1B7850
:10F368006BB1944B1B7803F08003DBB21BB192485E
:10F3780020210222EDE0914B8F4819780CE04FF4E0
:10F38800366363432A783424013A04FB02348C4BF5
:10F3980089481C19A619717C822256E6123B0B2B50
:10F3A80000F292819DF81F20DBB2222101FB02317D
:10F3B8007D4A163152F821207C4902F110008A4614
:10F3C80052F804CB824241F804CBF9D1DFF83092ED
:10F3D800DFF830B22FB199F80020012A15D1013297
:10F3E80009E096B199F80020012A07D975490978EA
:10F3F80003290AD1013A89F8002006E005D17149AC
:10F408000978032908BF8BF8002099F800209AB9D9
:10F418004FF4B6614C432A781A21013A01FB0244A1
:10F42800674AE318083302EB43039A798BF8002004
:10F43800DA79644B1A7047E1634C202104F1180013
:10F448000822F0F7A7FFB8F1000F00D1AEB15D4D6B
:10F458002B78012B01D15D4A01E04BB95C4A136856
:10F4680023615368CAF80430B8F1000F21D00BE0CB
:10F47800022B0CBF574A584AF1E7584A13682361D0
:10F488005368CAF8043019E19BF800004E4A31214C
:10F49800002350FA03F515F0010F01D0117701E0B0
:10F4A8002D251577013301310132042BC9B2F0D172
:10F4B8002FE0002E00F00281202108224848F0F7B2
:10F4C80069FF3D489BF800108222F9F7C9FA394BC9
:10F4D8001B7803F08003DBB21BB199F80030012BD5
:10F4E80002D82B78032B21D1202102223248F0F7B1
:10F4F80051FF1BE050FA03F515F0010F01D0117709
:10F5080001E02D251577013301310132042BC9B2F1
:10F51800F0D1284B1B7803F08003DBB233B199F8A4
:10F528000030012B02D9E4182023A376214B1B7845
:10F5380003F08003DBB2002B00F0C68099F800309E
:10F54800012B40F0C180002F40F0BE8017482021D9
:10F558000822F0F71FFFB7E099F80030214D13F0AB
:10F56800010F04BF43F0010389F800302E78002E04
:10F578004AD12D210A221C48F0F70CFF04201B4910
:10F58800F9F748FA1A4B1B78012B02D110201949B8
:10F5980006E0022B02D11020174901E0174910207C
:10F5A800F9F738FA90E000BF840D0020040200202B
:10F5B800AB1D0020EC39002012020020601E002044
:10F5C800643E0020E11D0020F401002025330308DB
:10F5D800463303086733030888330308A132030856
:10F5E8000C0200209F1D0020C41D002014350308B4
:10F5F800951D0020FE290308BC290308DD290308FE
:10F60800971D0020911D0020314B1C782046F9F7EA
:10F61800BDFA304B304A00282AD0304F304938786C
:10F62800A04216D130380C782E4E00EB80073C19DA
:10F63800345D04B90C700F7800EB8000C4190137F1
:10F64800FFB2C0190F70315C345D59B9244801709C
:10F6580008E00120087019783C7019B1092E9CBF88
:10F6680036182E702978511801F8014C402119706C
:10F67800197811B11748013901701978012909D190
:10F688002978092902D81848013101700021197018
:10F69800134B19701168154BC3F816105168C3F84D
:10F6A8001A101289DA83124A127802F08002D2B252
:10F6B80052B12A789B1820225A7505E09BF8000061
:10F6C8000A4A3121002315E709B0BDE8F08F00BFD1
:10F6D800CC1C0020E91C0020C41D0020E61C0020D2
:10F6E800121D0020F4B102089F1D0020F401002023
:10F6F800EC39002010B5002386B004468DF814308C
:10F7080011B118460C4901E008460C49F9F782F98D
:10F71800217810220139C9B201EB011101F5C2416A
:10F72800483101A802F009FB1020014601AAFDF7A3
:10F73800E7FD06B010BD00BF0C1303084E13030805
:10F748000B4B1B78442B06D0552B037801D013B1F3
:10F758007047013B01E003780133037003780BB96C
:10F76800203302E0212B01D1203B0370FFF7C2BFF9
:10F77800CC1C00202DE9F74FDFF8CC91DFF8D8A199
:10F7880099F80030554643F0010389F800309AF89B
:10F798000130644C23F07F039B46D3B100206249BB
:10F7A800F9F738F961482A21F0F772FE18B1217883
:10F7B8008222F9F755F92278002A40F0AF802B68A9
:10F7C80062F3CF332B605A4B1A7842F003021A7057
:10F7D800A4E0574F23703B783E4603F00202D2B2B2
:10F7E8000192DFF87881002A44D013F001092BD068
:10F7F80058465049F9F70EF998F80030232B0CD1E8
:10F808004D4B4E4A4E481A600121FFF773FF3B7873
:10F8180003F0FE036BF341033B7098F800302A2B8A
:10F828007CD1337803F0FE036FF3410333702B6808
:10F8380043F400432B600F232370414B187803B027
:10F84800BDE8F04F0FF030B848463E49F9F7E2F806
:10F8580098F80030232B61D1374B384A38481A6062
:10F868000121FFF747FF3B7869F3000369F3410380
:10F878003B7053E00EF069FF054600282FD00121A8
:10F888002F48FFF75DFF98F80030532B12D13B78D3
:10F89800019A03F0F10362F300033B70DAF80030D9
:10F8A80043F40043CAF800300F232370244B187820
:10F8B8000EF0FAFF98F80030232B2FD1337800226E
:10F8C80003F0FD036FF3000333701D4B1A70F9F753
:10F8D80065F91D4A137843F00603137014E01B49B9
:10F8E800F9F798F898F80030232B17D13B7865F38F
:10F8F800410365F300033B70F9F750F999F80030BC
:10F9080043F0060389F80030114A1378013BDBB253
:10F918001370104A52F82320074B1A6003B0BDE851
:10F92800F08F00BF8E58002090130308F4010020C8
:10F938001B3C0020B1130308041D002098B30208E3
:10F948009E1D0020D2130308E31D0020F3130308B3
:10F95800C31D0020D01D0020EC390020CC1C002045
:10F968002DE9FF41364C374D237843F001032370CE
:10F97800297801F00401C9B211B93348FFF7E0FE54
:10F988002B7803F00402D2B232B1304A12781AB995
:10F998002C4A43F0080313702D4E3378232B26D1BD
:10F9A8002B782A4A6FF3C303002113F004082B7045
:10F9B800284F117009D0234A61F382031370264B34
:10F9C80021483B60FFF796FE11E0F9F7E7F8237846
:10F9D800224A43F0060323701378013BDBB213700D
:10F9E8001F4A52F823303B60174B83F80080337866
:10F9F800532B23D12B780424144A03F0F403234314
:10FA080014702B70104B0B221D781649013DEDB276
:10FA180002FB05F000F5CA40883002F088F90020A2
:10FA28001149F8F7F7FFFF2300210093013516204D
:10FA380022460B460191029502F0ECF9BDE8FF81E0
:10FA4800E31D00201B3C00209E1D00208E58002036
:10FA5800CC1C0020041D0020B4B30208C31D0020E4
:10FA6800D01D0020103C00206F1303082DE9F04141
:10FA7800984B04469A7812F0010F00F017811B8802
:10FA8800002B40F01381944D95F820303F2B40F225
:10FA9800D780012C14D1914B1B7803F00203DBB201
:10FAA800002B00F0C48095F820208B4B402A03D10E
:10FAB800013283F82020FBE0482283F82020B6E0BA
:10FAC800022C03D1482385F82030B0E0844E3378E7
:10FAD80003F02002D2B28AB195F82020402A0DD135
:10FAE800032C0BD07F4B804A03F1100153F8040B11
:10FAF8008B4242F8040BF9D1412395E003F010033F
:10FB0800DBB28BB195F82030412B0DD1032C0BD0F3
:10FB1800764B754A03F1100153F8040B8B4242F8F7
:10FB2800040BF9D142237FE0F37813F0010F0FD0D3
:10FB380095F82020422A0BD16D4B6B4A03F1100136
:10FB480053F8040B8B4242F8040BF9D143236BE0C2
:10FB580003F00202D2B27AB195F82020432A0BD1E1
:10FB6800644B614A03F1100153F8040B8B4242F8CD
:10FB7800040BF9D1442357E003F00402D2B27AB15E
:10FB880095F82020442A0BD15B4B574A03F110010A
:10FB980053F8040B8B4242F8040BF9D1452343E098
:10FBA80003F00803DBB28BB195F82030452B0DD15B
:10FBB800032C0BD0514B4C4A03F1100153F8040BA2
:10FBC8008B4242F8040BF9D146232DE00FF052FC8A
:10FBD800A0B14B4B1B788BB195F82030462B0DD13B
:10FBE800032C0BD0474B404A03F1100153F8040B88
:10FBF8008B4242F8040BF9D1472315E0F37803F060
:10FC08004003DBB29BB195F82030472B0FD1032C72
:10FC18000DD03D4B344A03F1100153F8040B8B42CD
:10FC280042F8040BF9D1482385F8203078E095F89C
:10FC380020300133DBB2472B85F820307FF629AF1F
:10FC480095F82060472E04D9234B002683F82060BE
:10FC580001E00136F6B206F14007FFB212E02B4888
:10FC6800314615F080FB08B1032C04D1284B9B5D6D
:10FC780023B1032C02D185F820600FE00136F6B2DB
:10FC8800BE4203D03F2EEAD9402E07D1214B1E2277
:10FC98001A70402385F82030BDE8F08195F82000DF
:10FCA8001149652246F61563F8F700FE012C37D195
:10FCB800194B0D4A03F1100153F8040B8B4242F81B
:10FCC800040BF9D1044B93F820303F2B3CD900208A
:10FCD80012493EE0F41D0020F4010020981900208C
:10FCE800EC390020441A0308FB1D0020651A03089C
:10FCF800861A0308A71A0308C81A0308E91A03088A
:10FD0800583E00200A1B03084C1B03082E1A00202B
:10FD1800E4190020A01D0020447D0308021A0308EE
:10FD2800104BD87800F02000C0B220B1022C06D0C9
:10FD380000200D490DE0032C01D10C4909E00C4BC2
:10FD480093F820303F2B02D800200A4901E00A49E5
:10FD58000020F8F75FFE1020084A0146BDE8F04190
:10FD6800F8F710BEEC3900201D110308231A030808
:10FD7800F4010020C01903082B1B0308F41D002000
:10FD880010B5F8F70BFF084B1B7803F00403DBB240
:10FD98002BB106490020BDE81040F8F73BBE022011
:10FDA800BDE81040FFF762BE98190020F21703085B
:10FDB80070B5224B06461B78214CF3B9257819E01B
:10FDC8002048294615F0CFFA78B123689D4202D918
:10FDD800FF2E02D007E0FF2E02D19D4208D202E09A
:10FDE80036B91DB913B9256012E00EB9013500E026
:10FDF800AD19EDB23F2DE3D90AE0013B20211248AD
:10FE080010222360F0F7C6FA00201049F8F702FE26
:10FE18000F48F8F7A5FD46F6156320780D496522C9
:10FE2800F8F744FD084D216805F110000131022260
:10FE3800F8F716FE2D23AB7470BD00BF931D00208C
:10FE4800AC1D00200A1D0020F4010020C05B03083F
:10FE5800F41D0020FB1D0020F8B5594BF02259482D
:10FE68001A700378044613F00E051DD1564A43F064
:10FE78000203156000F8013B15F01AFA2C46534BA3
:10FE8800E35C1BB15248214615F057FA0134402C67
:10FE9800F5D1504B01221A7010F03AFB4E4B1A78EC
:10FEA80042F001021A70F8BD13F00C0543D12E463A
:10FEB8004748294615F057FA08B10136F6B2013518
:10FEC800402DF5D11EB9237843F0040331E0002515
:10FED80042482946EFB215F046FA68B13B4BEB5C55
:10FEE80053B13F4B01371F700020FFF761FF2378A4
:10FEF80043F00803237002E00135402DE8D1394D65
:10FF08003A212846F0F7C4FA38B1401BC0B2013094
:10FF1800281831460222F8F7A3FD334B1B78532BE0
:10FF28004CD12F4B00201870FFF742FF237843F085
:10FF380008032370F8BD6FF34103037003F0040353
:10FF4800DBB2294D23B100202849F8F763FD0EE004
:10FF58002B78552B01D1FF2002E0442B02D1012040
:10FF6800FFF726FF13200D21214AF8F70BFD2B7808
:10FF7800232B23D12478134E04F00204F4B9154B33
:10FF88001C7010F0C5FA337803F0FB0364F3C30365
:10FF980033700D4B1C60F8F701FE0F4B1A7842F0D6
:10FFA80006021A70134A1378013BDBB21370124A27
:10FFB80052F82320114B1A60094B1C70F8BD00BF82
:10FFC800EF1D0020091D0020AC1D0020302C002052
:10FFD8000A1D002030140020E31D0020991900207C
:10FFE800931D0020F4010020CC1C0020066D03089E
:08FFF800F41D0020C31D0020D0
:020000040801F1
:10000000D01D0020041D002070B505460C46164684
:100010003BB1400000F5364039304018114601F040
:1000200075FE054B292202FB0535F3092C1906F054
:100030007F066370E67070BDE23A002038B510B3F9
:10004000A0F14103DBB2432B1FD9C50900F07F04A7
:100050000BD0052C19D90021601E0A460BF0AAFA14
:10006000D0F1010038BF002038BD042C0FD9601E2C
:10007000C0B229462A460AF015FF50B9102C8CBF91
:100080000020012038BD012038BD002038BD2846A1
:1000900038BD284638BD0000F7B5604F604C387851
:1000A00031234000237400F5364001332376393084
:1000B000053B6374637601F033FEC0B220F07F022B
:1000C00000F07F01D2B28DF804108DF8002004F109
:1000D000120359B9534A04F11500118892786182CC
:1000E0009A7020210222F0F759F90CE0D20904EBB2
:1000F0008202526A10886082927804F115009A7028
:100100000222F8F7B1FC3878400000F536403A306A
:1001100001F006FEC0B220F07F0300F07F01DBB2E9
:100120008DF805108DF801303F4851B93D4B203115
:100130001A889B786283837002220330F0F72EF9CD
:100140000BE0DB0904EB83035B6A1A8862839B780C
:10015000022283700330F8F787FC344B1B7813F0CE
:10016000010F5AD0324D02A92A788B1813F8041CBB
:1001700013F8086C2F4B1B78232B04D1002A41D194
:10018000223B2B703EE02A2B04D1002A3AD0013AC0
:100190002A7037E0552B46EA010611D10DE02B7885
:1001A00002AAD318013E13F8081CF6B23046C9095A
:1001B00013F8042CFFF742FF98B9002EEFD121E08D
:1001C000442B19D115E02B7802A9CB18013613F86E
:1001D000081CF6B23046C90913F8042CFFF72EFFAD
:1001E00038B1134B3878197832460123FFF70CFFEA
:1001F00008E0872EE7D905E0532B03D1533B2B7042
:10020000F9F7BEFC0C4B1B7803F08003DBB223B183
:100210002B782022023304F83320FEBD931D0020EA
:10022000F4010020037903080E020020E31D0020E2
:100230009E1D0020CC1C0020EC390020024800212B
:100240000922F0F7ABB800BFB11D002070B50A4617
:10025000002405E01B19811A2A2501345D54E4B2FB
:100260000F4D104B295D09B19442F3D1801A00194A
:1002700018182021121BF0F791F80B4B1E7876B15D
:10028000432E07D114B1013CE4B201E0074B1C70CE
:1002900000232B553046F8F77DFC00B12E5570BD7C
:1002A000B11D0020F4010020CC1C0020F21D002014
:1002B00038B5184C184DA07800F01000C0B250B9F5
:1002C0001649F8F7ABFBFFF7B9FF236843F4801337
:1002D00023600F232B702A782AB92368FF2062F34A
:1002E0001453236038BD0E48C5792DB91C20082150
:1002F000FFF7ACFF284638BD23680A496FF3145353
:1003000008222360F0F7CAFA00280CBF0120FF2062
:1003100038BD00BFEC390020F21D0020551803083D
:10032000B11D00205C980308F0B55C4C85B0667880
:1003300006F01006F6B2002E3ED1594B1A78594BF2
:10034000013A53F82230584A934204D1574B1A7855
:1003500042F0020207E002F11C018B4208D1534B2C
:100360001A7842F00402022161F3C7021A7019E000
:100370003832934216D1FFF79BFF002800F08C80A3
:1003800001284A4D06D12B78022243F0010362F383
:10039000C70306E030464649F8F740FB2B7866F382
:1003A000C7032B70434B1A7842F001021A7023687E
:1003B00043F4805323606FE03C4D2B7813F0F80634
:1003C00006D03D49002005B0BDE8F040F8F726BB57
:1003D00013F0070F41D003F00202D7B24FB1122041
:1003E000314611F0DBF9FF2300930196029643207A
:1003F0002AE003F00406F6B2A6B13946384611F0F9
:10040000CDF9382102200FF08DFD0AF01BFB0EF014
:10041000C7F9FF230093019702974420394604222D
:100420003B4614E013F0010F13D0012143F6206086
:1004300011F0B4F93046F5F7EFFE204B45201E8051
:10044000FF2300930196029631460422334601F0C1
:10045000E5FC00201A49F8F7E1FA2B7803F0FA03DB
:100460006FF341032B70174B1B78232B14D1236898
:100470006FF30C332360F8F795FB0E4B1A7842F0BC
:1004800006021A70064A1378013BDBB21370054A64
:1004900052F823200C4B1A6005B0F0BDEC39002057
:1004A000C31D0020D01D0020D0B302080856002034
:1004B00076180308E31D0020A2700308E21C002048
:1004C00081700308CC1C0020041D00201FB50446C9
:1004D000F5F78EFFA8B14B2002F072F8FF230093CE
:1004E0000121FF3B0193392004220B460134029481
:1004F00001F094FC064B01205A7842F004025A7035
:1005000004E0044B1888003818BF012004B010BD67
:10051000F03B0020A4580020F0B5204E0024337A90
:100520000546013385B00F46337210202146012263
:1005300023460094F2F7E8F855B9FF2300934F20C3
:10054000294604222B460195029701F067FC0EE034
:10055000012D0CD1FF230093502023462146042275
:100560000194029701F05AFC337A013B3372337ADB
:10057000052B11D1FA3301210024009327200B46CB
:1005800004220194029401F049FC044B1C7205B052
:10059000BDE8F04001F0E6BF05B0F0BDA21D0020AF
:1005A000074B292202FB00335B7913F0100F05D0B3
:1005B000044B283ADA711A7109321A72704700BF77
:1005C000E23A00206B130020044B1878A0F1010CD4
:1005D000DCF1000040EB0C00704700BF001D002064
:1005E000034B1878A0F10202504240EB0200704722
:1005F000001D0020034B1878012894BF0020012023
:10060000704700BF001D0020064B1A7802F0F70269
:100610006FF304121A70044B00221A70034B03325A
:100620001A707047B01D0020F21D0020001D002030
:1006300010B52148214903680A789C7B944203D96C
:100640009C8914F0200F18D09A8912F0800F01D1E4
:1006500005E01C3B9A8912F0400FFAD000E01C33F1
:10066000036000230B7003689B8913F0200F16D0E2
:10067000134BDA79114B1A7011E00132D2B20A70C1
:10068000986843F60953984209D101E00132D2B289
:10069000162A03D80B4853B29840F7D40A700A4A76
:1006A000136843F480731360F8F7C0F8074B1A78A7
:1006B00042F006021A7010BD041D0020931D002098
:1006C000A21D002000060088EC390020E31D002058
:1006D00010B52349234A0B78D3B11068848914F0EC
:1006E000200F15D1013BDBB20B70846843F6095231
:1006F000944228D104E013B1013BDBB200E0837BDC
:10070000162B03D8184C5AB29440F4D40B701AE04C
:100710001368988910F0400F01D106E01C339889C6
:1007200010F0800FFAD0136002E00E481C3B03600B
:1007300013689A7B0A709B8913F0200F03D00B4B30
:10074000DA79074B1A700A4A136843F4807313600E
:10075000F8F76CF8074B1A7842F006021A7010BDD1
:10076000931D0020041D002000060088A21D00200B
:10077000EC390020E31D0020074B084A1B68934218
:1007800002D01C32934205D1054B1878003818BFAF
:100790000120704700207047041D002024B4020887
:1007A00094190020074B084A1B68934202D01C3260
:1007B000934205D1054B1878003818BF01207047C7
:1007C00000207047041D00205CB40208941900202A
:1007D00070B50A4C0546E07100F56A507C3001F0B6
:1007E0009FFA207005F5D840E93001F099FA607061
:1007F0002046BDE87040F5F727BD00BFA21D0020D0
:100800002DE9F0479A4B86B01A7806460F461C46EB
:100810001AB1012A40F0DA812FE0964B1A68964B04
:100820009A4200F0D581F5F763FA944B5B7803F0B8
:100830000203DBB253B9924B5B7803F08003DBB267
:1008400023B901F0B5FE08B90AF0FCF88D4B1A681F
:100850006FF310421A6037B98B4B1878F8F79AF992
:10086000002800F0B581FFF7E9FC884B3C221A70A4
:10087000F7F7DCFF237801332370844B1B7813B91F
:10088000FFF7C2FEA4E1012130460AF0FDF8F7F7B8
:10089000C1FF00207E49F8F7C1F806211B20FFF7B1
:1008A000D5FC7C4B7C491A7898468A1812F8312C72
:1008B000002A00F08D81794A7949137891F80090E7
:1008C000C3F3C00AC3F3001503F0F7036FF3041377
:1008D00009F00109137017B10223237000E027709B
:1008E0000B21062204A801F02CFA98F8002004A895
:1008F0006949303AEFF778FC044610B1122700241A
:1009000029E04AF6EB0001F00BFA0028F6D0654D1D
:100910002C72F5F753FB0446002840F05981624AD7
:10092000544B21461A60FF23009301900290042249
:100930000820234601F072FA012223460E202146A8
:100940000094F1F7E1FE594B1A7842F004021A7054
:100950000123AB713CE13946062204A801F0F1F90C
:1009600098F8002004A84C49303AEFF73DFC0028E5
:1009700040F020812046FFF7A9FD002840F02881A3
:10098000DFF82081012188F808002046F5F724FBD4
:1009900049EA0A090746F5F711FB002840F0BF8035
:1009A00038464349EFF7FEFDC0B901F013FD314B66
:1009B000B9F1000F02D115B93E4A24E035B13E4AE3
:1009C0001A603E4B1A786FF3410205E03C4A1A6008
:1009D0003A4B1A7865F341021A70E5E03846394916
:1009E000EFF7E0FD20B138463749EFF7DBFD78B986
:1009F000B9F1000F40F0EC80002D40F0E98001F0EB
:100A0000E9FC324A1B4B1A603046FFF7C9FDCBE0C8
:100A100038462F49EFF7C6FD50B94AF6E9000121E3
:100A200001F074F9174A136843F400531360DFE7C9
:100A300038462849EFF7B6FD40B9B9F1000F40F04C
:100A4000C780002D40F0C480234A0DE0384623497A
:100A5000EFF7A8FD002845D1B9F1000F40F0B880AC
:100A6000002D40F0B5801E4A024B1A609CE000BF8A
:100A7000001D0020041D002024B40208D6330020ED
:100A8000FF3B0020EC390020CC1C0020F21D002090
:100A9000FC100308E81C0020B11D0020B01D002040
:100AA000EF630020A21D002094B40208FE25002060
:100AB000BDA00308E0B6020868B80208E31D0020E4
:100AC00040B4020839A00308C9A2030884B8020888
:100AD00074A0030876A00308BCB8020886A2030825
:100AE0005CB4020838463C49EFF75CFD00285BD156
:100AF00001F070FCB9F1000F07D0384A384B1A608A
:100B0000384B1A786FF3410261E0002D60D0364A0D
:100B1000334B1A60334B1A7869F3410257E0384679
:100B20002D49EFF73FFD054628B901F053FCB9F117
:100B3000000F4DD01EE038462C49EFF733FD00285A
:100B400046D038462A49EFF72DFD40B9B9F1000FDC
:100B50003ED1284A224B88F807401A6038E03846D0
:100B60002549EFF71FFD054660B9B9F1000F16D012
:100B700001F030FC194A1A4B1A601A4B1A7865F3C7
:100B8000410224E038461D49EFF70CFD20B13846FC
:100B90001B49EFF707FD10B9B9F1000F18D1194A39
:100BA0000F4B1A6001F016FC2046FFF711FE202CB7
:100BB0000ED105E00134E4B20737202C7FF4CBAE30
:100BC000711C0020C9B2FFF7A7FC01E000221A70D7
:100BD00006B0BDE8F08700BF78A0030840B4020863
:100BE000041D0020E31D002068B8020876A0030859
:100BF00086A203085CB40208BDA0030839A003085C
:100C000074A0030810B90208034B1B7853FA00F0D4
:100C100000F00100704700BFA21D0020034B1B180D
:100C20009878003818BF0120704700BFA21D00202F
:100C3000F8B504460D460E78FFF7F0FF18B3144AD6
:100C400013199F7810460023021992781A4112F066
:100C5000010F4FF001020DD0BE42297803D09A4017
:100C600042EA010104E09A40C2F10F0202EA0101E6
:100C7000297005E09A402978C2F10F020A402A70D3
:100C80000133042BE0D12B7803B92E70F8BD00BFDF
:100C9000A21D002070B57E4B044631B11B78532B4A
:100CA00040F0F580533B037070BD1A78302A33D181
:100CB000784B1A795AB1784A78491278292000FB82
:100CC0000212527912F0100F01D001221A71744AE7
:100CD00025781278154012D01D7A002D40F0D7806B
:100CE000E8B2FFF791FF30B10123AB402278C3F1A6
:100CF0000F03134023700135042DF1D141E0E8B218
:100D0000FFF782FF20B10123AB4022781343237009
:100D10000135042DF3D134E0A2F13101C9B2032928
:100D20003BD85C4E32795AB15B4A5C491278292033
:100D300000FB0212527912F0100F01D00122327121
:100D40001D78313DEDB22846FFF75EFF002800F028
:100D50009E80237853FA05F212F0010F0BD0327AFD
:100D6000002A40F09480013212FA05F5C5F10F0512
:100D700005EA030304E0012212FA05F545EA03033C
:100D80002370002112224748EFF708FB454920460F
:100D90001022BDE87040FCF785BA132A0CD0552A02
:100DA00018D13D4B3D4A1B78292101FB03235B7978
:100DB00013F0200F03D170BD364B01221A710020B1
:100DC0002146FFF735FF0020FFF728FF00285ED0FF
:100DD000002054E0142A0CD02A2A18D12E4B2F4A76
:100DE0001B78292101FB03235B7913F0200F03D12A
:100DF00070BD284B01221A7101202146FFF718FF10
:100E00000120FFF70BFF002841D0012037E0152A11
:100E10000CD0232A18D1204B204A1B78292101FB12
:100E200003235B7913F0200F03D170BD194B01220E
:100E30001A7102202146FFF7FBFE0220FFF7EEFEAB
:100E4000002824D002201AE0162A0CD0442A1ED1F1
:100E5000114B124A1B78292101FB03235B7913F004
:100E6000200F03D170BD0B4B01221A7103202146C4
:100E7000FFF7DEFE0320FFF7D1FE40B10320094952
:100E8000102246F67973BDE87040F7F713BD70BDC8
:100E9000CC1C00206B130020961D0020E23A00209D
:100EA000A21D0020CE1C00202DE9F043002387B0B6
:100EB0008DF81730804B1B78012B00F07E827F4C21
:100EC000227872B17E4B5B78002B40F076827D4DAC
:100ED0002B78002B40F0B980F7F764FE09232B70C4
:100EE000B3E0784B19781D46082900F2AE807649A8
:100EF0000978232913D11A70F7F754FE7349744AFD
:100F00000B7853B17348013B0478DBB244F006041C
:100F100004700B70704951F823301360C1E26D4BBF
:100F20001A7812F0010F04D101210A438DF817102D
:100F30001A70F2F71BF828B92B781BB90DF11700BE
:100F4000FCF7AAFDF2F720F830B92B78012B03D17A
:100F50000DF11700FCF7A0FDF2F724F830B92B785B
:100F6000022B03D10DF11700FCF796FDF2F726F8DE
:100F700030B92B78032B03D10DF11700FCF78CFD52
:100F8000F2F72AF848B9F2F753F830B92B78042B66
:100F900003D10DF11700FCF77FFDF2F77DF830B9B2
:100FA0002B78052B03D10DF11700FCF775FDF2F737
:100FB00067F830B92B78062B03D10DF11700FCF739
:100FC0006BFDF2F717F830B92B78072B03D10DF131
:100FD0001700FCF761FDF2F71BF830B92B78082BEE
:100FE00003D10DF11700FCF757FD9DF81730002BCA
:100FF0002BD02B78082B23D8DFE803F005080D1041
:101000001316191C1F000020344901E03449002048
:10101000F7F704FD16E000203249F9E700203249D5
:10102000F6E700203149F3E700203149F0E70020DE
:101030003049EDE700203049EAE700202F49E7E793
:10104000F7F7B0FD2A782E4B1A701E4F3B783D46BD
:10105000092B40F0BD801F4B1B4F1978984611F0AB
:1010600001015CD1274E12223046EFF797F9012398
:10107000737415F067FA10B92278234B1A7023782D
:1010800003B97374737C13B1204B00221A70FCF700
:10109000E5FC1D48717CFFF7FDFD98F8003003F07A
:1010A000FD0343F0010388F80030194B1A788AB326
:1010B0003A7000221A7032E0EF1D002094190020CF
:1010C0006B130020E01D0020CC1C0020C31D00205D
:1010D000041D0020E31D0020D01D0020B6410308A0
:1010E00095410308D7410308F84103081942030852
:1010F0003A4203085B4203087C4203089D4203080E
:1011000085630020CE1C0020081D002064130020F1
:10111000981D002015F016FA08B930233B703B7873
:10112000884E13B93379112B4ED1DFF86892FCF752
:1011300095FC854899F81110FFF7ACFD824B1A78A1
:10114000984622B1002010214A46FCF7DDF82378AA
:1011500098F800407D4A24EA030111707C4A23EA92
:10116000040111703A78A2F15200C0B2012803D9EB
:101170003079744F11280CD1002333711CB911B18F
:101180000133009311E10423F3702B7801332B70AA
:101190001AE0432A18D1BBB97C78ACB96D4BD87929
:1011A000F4F7D0FF38B96C49F7F738FC0523FB702A
:1011B00008332B7004E020466849F7F72FFCFC70D9
:1011C000674A684B1A606CE15F48FCF7C3F868E156
:1011D0000A2B31D15D4807F0A7F8C6B2594C36B397
:1011E000E378042B02D100205F4903E0022B04D1F5
:1011F0005E490020F7F712FC02E00BB90433E370FC
:10120000314602225A48F7F72FFC5A4B1E78232EFC
:1012100000F0D3803046F7F7BDFC002800F0418194
:10122000312E40F03E812B7801332B7002E03B7869
:1012300001333B70042332E00B2B32D1434807F0DB
:1012400059F8C6B23F4C36B3E378042B02D10020E4
:10125000494903E0022B04D148490020F7F7DEFB9F
:1012600002E00BB90433E370314602224048F7F73D
:10127000FBFB404B1E78232E00F09F803046F7F793
:1012800089FC002800F00D81312E40F00A812B7876
:1012900001332B7002E03B7801333B700823E3708D
:1012A000FFE00C2B40F0FD80284807F009F80021F2
:1012B000C4B2264806F0DAFF002C6DD0214EB37878
:1012C0002BB9BE2014F078FEB3780133B370F378F5
:1012D0001C4A092B02D900201F4915E010D11D4BD3
:1012E00000241C70D470264B194A18491648012551
:1012F0001C7014700C7004700095019402949EE0B0
:10130000082B04D11F490020F7F788FB11E0062BBA
:1013100002D100201C49F7E7042B02D100201B4911
:10132000F2E7022B02D100201949EDE70BB908338F
:10133000D370F378082B3CD80D4821460222F7F7EA
:1013400093FB36E06B130020081D0020F11D0020E8
:10135000E41D0020A21D00200A3C0308863B030870
:101360002CB90208041D00208E3C0308AF3C030882
:10137000F4010020CC1C00204C3C03086D3C030809
:10138000CD1C0020A73B0308C83B0308E93B03082A
:101390002B3C0308CE1C0020012543484349444A06
:1013A0002B460095F2F7D0FB0095424B01941B7839
:1013B00040E0414F3C78232C02D1FCF777FB70E0F2
:1013C0002046F7F7E7FB00286BD0303CE4B2631E01
:1013D000DBB2012B3C7039D8022C364D1ED1E87996
:1013E000F4F7B0FE002838D02F48FCF719FB00288E
:1013F00033D1082246F64E01304800F0A2FC2A49BB
:101400002E4813F06CFF2D49082246F64E0000F0DE
:1014100092FC2A492A4813F078FF06E0012322486B
:101420002249234A0093F2F78FFB01230024009303
:1014300001942B78029323481D49234A1B4BFCF748
:101440007BFAF7F7AFFB214B1C602AE0032C28D175
:10145000184BD879F4F776FE10B90C23F37020E01E
:1014600015F070F870B904460F48214613F07FFF5D
:1014700028B1E02014F0A0FD204614F0D9FD01347D
:10148000402CF1D1124A00231370F3702B78114ACB
:1014900001332B700D4B1A600F4B1A7842F0060285
:1014A0001A7007B0BDE8F083871B0020CD1C002018
:1014B000F11D0020A21D0020CC1C00207C19002062
:1014C000D9190020081D0020E41D0020041D002063
:1014D0009E1D00202CB90208E31D0020194A00239C
:1014E0001360194A19481370194A1178037001F0F2
:1014F000F60163F307111170164A1748117863F368
:1015000001011170154A117863F3C5011170144A75
:101510001370144A117801F0FC0163F38201117019
:10152000114A1168037021F4805163F3CF311160C7
:101530000E4A117801F0F40163F3820111700C4A34
:1015400093717047041D0020C31D00209E1D0020C4
:10155000E31D0020E51C0020EE1D0020991D002049
:10156000A11D0020B01D0020EC3900201B3C0020F4
:101570006B1300202DE9F04F6A4B6B4D1970A0F1F1
:101580001103DBB2012B87B00E46287006D8122853
:1015900001D1113800E00020F4F79CFE2B78522B8B
:1015A0000DD1F1F7C9FD28B9F1F7BAFD10B9F1F77E
:1015B000DBFD20B15D4B1A7842F008021A705C4BDB
:1015C0005C4C1B782BB922685B4B9A4201D0FFF729
:1015D00085FF2368002B40F04081584F7B7803F053
:1015E0002003DBB273B1564B93F80080B8F1000FC3
:1015F00008D14AF6E900414600F088FB3B6868F3F1
:101600004D333B604F4B187810F01E0002D0002085
:101610004D4907E04D4B93F805909846B9F1000FFE
:1016200005D04B4907B0BDE8F04FF7F7F7B9494F80
:1016300097F801B0BA46BBF1000F2DD0BBF1070FF0
:1016400015D94548F7F790F94449B878652246F628
:101650001573F7F72FF93878072310F003007B7024
:101660000EBF3F4948463F49F7F7D8F90CE0BBF1B8
:10167000020F09D83848437823B1F7F775F987F88E
:10168000019093E202237B701020334A014607B099
:10169000BDE8F04FF7F77AB9334B9A795AB183F82E
:1016A00006B000F09FFC8E20594601225B46CDF823
:1016B00000B0F1F729F80020F1F7A0FE2B4A2C49E1
:1016C00013782C4843F00603137000230B702A494B
:1016D00023600B7088F8013088F8043003702933D8
:1016E0007343264F9146F95C8346C1F3C00111B99B
:1016F0003046FFF785F8292303FB06777B7913F043
:10170000100F04D02A78133AD2B2032A3AD913F030
:10171000200F5DD02B78442B34D031D8232B31D0FF
:101720002A2B2EE0961D0020CC1C0020D61900206C
:10173000EF1D0020041D00202CB90208EC39002008
:10174000941900208D5800205F1103086B130020AE
:10175000BE4203089B1D0020F41D0020FB1D00203D
:101760006712030846120308A21D0020E31D002093
:10177000C31D0020981D0020931D0020E23A002088
:10178000552B25D1844B1B7813BB844B1F78FFB995
:1017900043F6DB2000F0C4FA0128014618D188F88E
:1017A00001001F200591FFF713F899F8003030462B
:1017B00067F3410389F80030059909F065F9F7F7F7
:1017C000F1F9774B2360774B1F602B788BF8003053
:1017D0002B78432B0AD1714B1B783BB90121724BFB
:1017E00088F801103046236009F04EF92878173840
:1017F000C3B2072B27D86D49FF220BF0B7F89AF830
:1018000000106B4B60F301018AF8001001F0030136
:10181000022918D00122032041B1009001929B7847
:1018200068309B1802930021033206E00090019279
:101830009B786C200133029304220B4600F0EEFAF1
:10184000FF238AF8013098F80730002B00F0AE81B2
:1018500052232B70574B0022DA712268524B9A4266
:1018600050D12878A0F14303DAB2122A22D8524A82
:101870005BB29A401ED5432840F09881464B1B78B6
:10188000002B40F0938100F0AFFD4C4B48B11A782B
:1018900003201109013191FBF0F000EB4000091A1F
:1018A00004E01A781109013101F0070161F3071210
:1018B0001A707BE1F7F76EF9002823D03F4F3B7891
:1018C00013F0F00108D161F307133B703C4B21602A
:1018D0001A7842F008020EE0102913D100F084FDBE
:1018E00080B13B7800216FF307133B70344B2160CC
:1018F0001A7842F0100230461A7007B0BDE8F04F77
:10190000FEF77EBF2F4B1E211A78254F61F346024A
:101910001A702B78232B1CD12368BB4219D12A4B78
:10192000292202FB0636737913F0100F11D0274BD2
:101930001B7873B1264EF7F735F9FCF7B7F8F07955
:1019400000F56A507C3000F0EBF93070AA20F1F716
:1019500055FD1A4E337813F0010F41D02368BB4276
:101960000BD01C4A934208D0FEF706FF28B9FEF7B9
:1019700019FF10B9AA30F1F741FD2268164B9A42BF
:1019800002D10020F1F73AFD2B78522B40F0D380A2
:101990005322124BC7E000BF94190020001D002005
:1019A00010B90208D01D002024B402089D1D00209B
:1019B0009B1D00206B130020002000C0E31D0020B1
:1019C000B01D0020611E0020E23A0020C31D00204F
:1019D000A21D00202CB9020848B90208CC1C002026
:1019E0002368BB420BD0734A934208D0FEF7C4FE73
:1019F00028B9FEF7D7FE10B9AA30F1F7FFFC2B7813
:101A0000552B1ED1FEF764FE33786B4843F0060376
:101A100033708378694F03F00203DBB24BB1F6F702
:101A2000A3FF23681868FAF71DF93B786FF34103A9
:101A30003B706348837803F00203DBB20BB1F6F727
:101A400093FF2B78442B1ED1FEF7F2FD33785A48D2
:101A500043F0060333708378584F03F00203DBB280
:101A60004BB1F6F781FF23681868FAF7FBF83B786B
:101A70006FF341033B705248837803F00203DBB2FB
:101A80000BB1F6F771FF2B78522B09D13378002276
:101A900043F0010333704B4B1A704B4B45321A70B5
:101AA0004A4B00271F702B78232B44D1484B4248C8
:101AB0001F70484B1F70F6F757FF4148F6F754FF69
:101AC0003378454943F0060333700B783B4A002BCB
:101AD0002BD0424A013B1770414ADBB20B7052F8DF
:101AE000233023603F4B1A7812B11F700EF014FDA3
:101AF00023683D4A9B68934202D10AF073F81AE0CA
:101B000002F59A718B4203D002F5E0718B4204D149
:101B10000120014607F0F0F80DE002F5EE72934265
:101B200009D1324B00221A7005E0117863F30711D6
:101B3000117023603AE02E4B5B7813B10020F1F76F
:101B40005DFC23681F7B17F00F0702D1FBF77CFABF
:101B50001BE0012F02D1F8F7BFF916E0022F02D1E6
:101B6000F9F736F911E0082F05D84FF09C53BB4028
:101B700001D5F9F7F3FB042F03D123689B6998473C
:101B800003E0052F01D1F8F7A1FE337803F002033B
:101B9000DBB21BB123681868FAF764F833786FF387
:101BA000410333702B780BB1084A137007B0BDE8BE
:101BB000F08F00BF2CB90208F41D0020E31D0020A7
:101BC000141D00209E1D0020CC1C0020E61C0020BF
:101BD000A11D0020EE1D0020C31D0020931D00202C
:101BE000D01D00203014002064B90208131D00200D
:101BF0006B130020034B1868034BC11A484240EB9B
